Archive member included to satisfy reference by file (symbol)

c:/renesas/ra/e2studio_v2022-10_fsp_v4.2.0/toolchains/gcc_arm/gcc-arm-none-eabi-10.3-2021.10/bin/../lib/gcc/arm-none-eabi/10.3.1/thumb/v8-m.main+fp/hard\libgcc.a(_arm_muldf3.o)
                              ./src/udp_printf.o (__aeabi_dmul)
c:/renesas/ra/e2studio_v2022-10_fsp_v4.2.0/toolchains/gcc_arm/gcc-arm-none-eabi-10.3-2021.10/bin/../lib/gcc/arm-none-eabi/10.3.1/thumb/v8-m.main+fp/hard\libgcc.a(_arm_addsubdf3.o)
                              ./src/udp_printf.o (__aeabi_dsub)
c:/renesas/ra/e2studio_v2022-10_fsp_v4.2.0/toolchains/gcc_arm/gcc-arm-none-eabi-10.3-2021.10/bin/../lib/gcc/arm-none-eabi/10.3.1/thumb/v8-m.main+fp/hard\libgcc.a(_arm_muldivdf3.o)
                              ./src/udp_printf.o (__aeabi_ddiv)
c:/renesas/ra/e2studio_v2022-10_fsp_v4.2.0/toolchains/gcc_arm/gcc-arm-none-eabi-10.3-2021.10/bin/../lib/gcc/arm-none-eabi/10.3.1/thumb/v8-m.main+fp/hard\libgcc.a(_arm_cmpdf2.o)
                              ./src/udp_printf.o (__aeabi_dcmpeq)
c:/renesas/ra/e2studio_v2022-10_fsp_v4.2.0/toolchains/gcc_arm/gcc-arm-none-eabi-10.3-2021.10/bin/../lib/gcc/arm-none-eabi/10.3.1/thumb/v8-m.main+fp/hard\libgcc.a(_arm_unorddf2.o)
                              ./src/udp_printf.o (__aeabi_dcmpun)
c:/renesas/ra/e2studio_v2022-10_fsp_v4.2.0/toolchains/gcc_arm/gcc-arm-none-eabi-10.3-2021.10/bin/../lib/gcc/arm-none-eabi/10.3.1/thumb/v8-m.main+fp/hard\libgcc.a(_arm_fixdfsi.o)
                              ./src/udp_printf.o (__aeabi_d2iz)
c:/renesas/ra/e2studio_v2022-10_fsp_v4.2.0/toolchains/gcc_arm/gcc-arm-none-eabi-10.3-2021.10/bin/../lib/gcc/arm-none-eabi/10.3.1/../../../../arm-none-eabi/lib/thumb/v8-m.main+fp/hard\libg_nano.a(lib_a-aeabi_memcpy.o)
                              ./src/udp_cdc.o (__aeabi_memcpy4)
c:/renesas/ra/e2studio_v2022-10_fsp_v4.2.0/toolchains/gcc_arm/gcc-arm-none-eabi-10.3-2021.10/bin/../lib/gcc/arm-none-eabi/10.3.1/../../../../arm-none-eabi/lib/thumb/v8-m.main+fp/hard\libg_nano.a(lib_a-errno.o)
                              ./ra/fsp/src/bsp/mcu/all/bsp_sbrk.o (__errno)
c:/renesas/ra/e2studio_v2022-10_fsp_v4.2.0/toolchains/gcc_arm/gcc-arm-none-eabi-10.3-2021.10/bin/../lib/gcc/arm-none-eabi/10.3.1/../../../../arm-none-eabi/lib/thumb/v8-m.main+fp/hard\libg_nano.a(lib_a-exit.o)
                              c:/renesas/ra/e2studio_v2022-10_fsp_v4.2.0/toolchains/gcc_arm/gcc-arm-none-eabi-10.3-2021.10/bin/../lib/gcc/arm-none-eabi/10.3.1/../../../../arm-none-eabi/lib/thumb/v8-m.main+fp/hard/rdimon-crt0.o (exit)
c:/renesas/ra/e2studio_v2022-10_fsp_v4.2.0/toolchains/gcc_arm/gcc-arm-none-eabi-10.3-2021.10/bin/../lib/gcc/arm-none-eabi/10.3.1/../../../../arm-none-eabi/lib/thumb/v8-m.main+fp/hard\libg_nano.a(lib_a-impure.o)
                              c:/renesas/ra/e2studio_v2022-10_fsp_v4.2.0/toolchains/gcc_arm/gcc-arm-none-eabi-10.3-2021.10/bin/../lib/gcc/arm-none-eabi/10.3.1/../../../../arm-none-eabi/lib/thumb/v8-m.main+fp/hard\libg_nano.a(lib_a-exit.o) (_global_impure_ptr)
c:/renesas/ra/e2studio_v2022-10_fsp_v4.2.0/toolchains/gcc_arm/gcc-arm-none-eabi-10.3-2021.10/bin/../lib/gcc/arm-none-eabi/10.3.1/../../../../arm-none-eabi/lib/thumb/v8-m.main+fp/hard\libg_nano.a(lib_a-init.o)
                              c:/renesas/ra/e2studio_v2022-10_fsp_v4.2.0/toolchains/gcc_arm/gcc-arm-none-eabi-10.3-2021.10/bin/../lib/gcc/arm-none-eabi/10.3.1/../../../../arm-none-eabi/lib/thumb/v8-m.main+fp/hard/rdimon-crt0.o (__libc_init_array)
c:/renesas/ra/e2studio_v2022-10_fsp_v4.2.0/toolchains/gcc_arm/gcc-arm-none-eabi-10.3-2021.10/bin/../lib/gcc/arm-none-eabi/10.3.1/../../../../arm-none-eabi/lib/thumb/v8-m.main+fp/hard\libg_nano.a(lib_a-memcpy-stub.o)
                              ./ra/fsp/src/bsp/cmsis/Device/RENESAS/Source/system.o (memcpy)
c:/renesas/ra/e2studio_v2022-10_fsp_v4.2.0/toolchains/gcc_arm/gcc-arm-none-eabi-10.3-2021.10/bin/../lib/gcc/arm-none-eabi/10.3.1/../../../../arm-none-eabi/lib/thumb/v8-m.main+fp/hard\libg_nano.a(lib_a-memset.o)
                              c:/renesas/ra/e2studio_v2022-10_fsp_v4.2.0/toolchains/gcc_arm/gcc-arm-none-eabi-10.3-2021.10/bin/../lib/gcc/arm-none-eabi/10.3.1/../../../../arm-none-eabi/lib/thumb/v8-m.main+fp/hard/rdimon-crt0.o (memset)
c:/renesas/ra/e2studio_v2022-10_fsp_v4.2.0/toolchains/gcc_arm/gcc-arm-none-eabi-10.3-2021.10/bin/../lib/gcc/arm-none-eabi/10.3.1/../../../../arm-none-eabi/lib/thumb/v8-m.main+fp/hard\libg_nano.a(lib_a-strlen.o)
                              ./src/hal_entry.o (strlen)
c:/renesas/ra/e2studio_v2022-10_fsp_v4.2.0/toolchains/gcc_arm/gcc-arm-none-eabi-10.3-2021.10/bin/../lib/gcc/arm-none-eabi/10.3.1/../../../../arm-none-eabi/lib/thumb/v8-m.main+fp/hard\librdimon_nano.a(rdimon-syscalls.o)
                              c:/renesas/ra/e2studio_v2022-10_fsp_v4.2.0/toolchains/gcc_arm/gcc-arm-none-eabi-10.3-2021.10/bin/../lib/gcc/arm-none-eabi/10.3.1/../../../../arm-none-eabi/lib/thumb/v8-m.main+fp/hard/rdimon-crt0.o (initialise_monitor_handles)
c:/renesas/ra/e2studio_v2022-10_fsp_v4.2.0/toolchains/gcc_arm/gcc-arm-none-eabi-10.3-2021.10/bin/../lib/gcc/arm-none-eabi/10.3.1/../../../../arm-none-eabi/lib/thumb/v8-m.main+fp/hard\librdimon_nano.a(rdimon-_exit.o)
                              c:/renesas/ra/e2studio_v2022-10_fsp_v4.2.0/toolchains/gcc_arm/gcc-arm-none-eabi-10.3-2021.10/bin/../lib/gcc/arm-none-eabi/10.3.1/../../../../arm-none-eabi/lib/thumb/v8-m.main+fp/hard\libg_nano.a(lib_a-exit.o) (_exit)
c:/renesas/ra/e2studio_v2022-10_fsp_v4.2.0/toolchains/gcc_arm/gcc-arm-none-eabi-10.3-2021.10/bin/../lib/gcc/arm-none-eabi/10.3.1/../../../../arm-none-eabi/lib/thumb/v8-m.main+fp/hard\librdimon_nano.a(rdimon-_kill.o)
                              c:/renesas/ra/e2studio_v2022-10_fsp_v4.2.0/toolchains/gcc_arm/gcc-arm-none-eabi-10.3-2021.10/bin/../lib/gcc/arm-none-eabi/10.3.1/../../../../arm-none-eabi/lib/thumb/v8-m.main+fp/hard\librdimon_nano.a(rdimon-_exit.o) (_kill_shared)
c:/renesas/ra/e2studio_v2022-10_fsp_v4.2.0/toolchains/gcc_arm/gcc-arm-none-eabi-10.3-2021.10/bin/../lib/gcc/arm-none-eabi/10.3.1/../../../../arm-none-eabi/lib/thumb/v8-m.main+fp/hard\libc_nano.a(lib_a-findfp.o)
                              c:/renesas/ra/e2studio_v2022-10_fsp_v4.2.0/toolchains/gcc_arm/gcc-arm-none-eabi-10.3-2021.10/bin/../lib/gcc/arm-none-eabi/10.3.1/../../../../arm-none-eabi/lib/thumb/v8-m.main+fp/hard\librdimon_nano.a(rdimon-syscalls.o) (__sinit)
c:/renesas/ra/e2studio_v2022-10_fsp_v4.2.0/toolchains/gcc_arm/gcc-arm-none-eabi-10.3-2021.10/bin/../lib/gcc/arm-none-eabi/10.3.1/../../../../arm-none-eabi/lib/thumb/v8-m.main+fp/hard\libc_nano.a(lib_a-fwalk.o)
                              c:/renesas/ra/e2studio_v2022-10_fsp_v4.2.0/toolchains/gcc_arm/gcc-arm-none-eabi-10.3-2021.10/bin/../lib/gcc/arm-none-eabi/10.3.1/../../../../arm-none-eabi/lib/thumb/v8-m.main+fp/hard\libc_nano.a(lib_a-findfp.o) (_fwalk)
c:/renesas/ra/e2studio_v2022-10_fsp_v4.2.0/toolchains/gcc_arm/gcc-arm-none-eabi-10.3-2021.10/bin/../lib/gcc/arm-none-eabi/10.3.1/../../../../arm-none-eabi/lib/thumb/v8-m.main+fp/hard\libc_nano.a(lib_a-lock.o)
                              c:/renesas/ra/e2studio_v2022-10_fsp_v4.2.0/toolchains/gcc_arm/gcc-arm-none-eabi-10.3-2021.10/bin/../lib/gcc/arm-none-eabi/10.3.1/../../../../arm-none-eabi/lib/thumb/v8-m.main+fp/hard\libc_nano.a(lib_a-findfp.o) (__retarget_lock_init_recursive)
c:/renesas/ra/e2studio_v2022-10_fsp_v4.2.0/toolchains/gcc_arm/gcc-arm-none-eabi-10.3-2021.10/bin/../lib/gcc/arm-none-eabi/10.3.1/../../../../arm-none-eabi/lib/thumb/v8-m.main+fp/hard\libc_nano.a(lib_a-nano-mallocr.o)
                              c:/renesas/ra/e2studio_v2022-10_fsp_v4.2.0/toolchains/gcc_arm/gcc-arm-none-eabi-10.3-2021.10/bin/../lib/gcc/arm-none-eabi/10.3.1/../../../../arm-none-eabi/lib/thumb/v8-m.main+fp/hard\libc_nano.a(lib_a-findfp.o) (_malloc_r)
c:/renesas/ra/e2studio_v2022-10_fsp_v4.2.0/toolchains/gcc_arm/gcc-arm-none-eabi-10.3-2021.10/bin/../lib/gcc/arm-none-eabi/10.3.1/../../../../arm-none-eabi/lib/thumb/v8-m.main+fp/hard\libc_nano.a(lib_a-sbrkr.o)
                              c:/renesas/ra/e2studio_v2022-10_fsp_v4.2.0/toolchains/gcc_arm/gcc-arm-none-eabi-10.3-2021.10/bin/../lib/gcc/arm-none-eabi/10.3.1/../../../../arm-none-eabi/lib/thumb/v8-m.main+fp/hard\libc_nano.a(lib_a-nano-mallocr.o) (_sbrk_r)
c:/renesas/ra/e2studio_v2022-10_fsp_v4.2.0/toolchains/gcc_arm/gcc-arm-none-eabi-10.3-2021.10/bin/../lib/gcc/arm-none-eabi/10.3.1/../../../../arm-none-eabi/lib/thumb/v8-m.main+fp/hard\libc_nano.a(lib_a-stdio.o)
                              c:/renesas/ra/e2studio_v2022-10_fsp_v4.2.0/toolchains/gcc_arm/gcc-arm-none-eabi-10.3-2021.10/bin/../lib/gcc/arm-none-eabi/10.3.1/../../../../arm-none-eabi/lib/thumb/v8-m.main+fp/hard\libc_nano.a(lib_a-findfp.o) (__sread)
c:/renesas/ra/e2studio_v2022-10_fsp_v4.2.0/toolchains/gcc_arm/gcc-arm-none-eabi-10.3-2021.10/bin/../lib/gcc/arm-none-eabi/10.3.1/../../../../arm-none-eabi/lib/thumb/v8-m.main+fp/hard\libc_nano.a(lib_a-writer.o)
                              c:/renesas/ra/e2studio_v2022-10_fsp_v4.2.0/toolchains/gcc_arm/gcc-arm-none-eabi-10.3-2021.10/bin/../lib/gcc/arm-none-eabi/10.3.1/../../../../arm-none-eabi/lib/thumb/v8-m.main+fp/hard\libc_nano.a(lib_a-stdio.o) (_write_r)
c:/renesas/ra/e2studio_v2022-10_fsp_v4.2.0/toolchains/gcc_arm/gcc-arm-none-eabi-10.3-2021.10/bin/../lib/gcc/arm-none-eabi/10.3.1/../../../../arm-none-eabi/lib/thumb/v8-m.main+fp/hard\libc_nano.a(lib_a-closer.o)
                              c:/renesas/ra/e2studio_v2022-10_fsp_v4.2.0/toolchains/gcc_arm/gcc-arm-none-eabi-10.3-2021.10/bin/../lib/gcc/arm-none-eabi/10.3.1/../../../../arm-none-eabi/lib/thumb/v8-m.main+fp/hard\libc_nano.a(lib_a-stdio.o) (_close_r)
c:/renesas/ra/e2studio_v2022-10_fsp_v4.2.0/toolchains/gcc_arm/gcc-arm-none-eabi-10.3-2021.10/bin/../lib/gcc/arm-none-eabi/10.3.1/../../../../arm-none-eabi/lib/thumb/v8-m.main+fp/hard\libc_nano.a(lib_a-fflush.o)
                              c:/renesas/ra/e2studio_v2022-10_fsp_v4.2.0/toolchains/gcc_arm/gcc-arm-none-eabi-10.3-2021.10/bin/../lib/gcc/arm-none-eabi/10.3.1/../../../../arm-none-eabi/lib/thumb/v8-m.main+fp/hard\libc_nano.a(lib_a-findfp.o) (_fflush_r)
c:/renesas/ra/e2studio_v2022-10_fsp_v4.2.0/toolchains/gcc_arm/gcc-arm-none-eabi-10.3-2021.10/bin/../lib/gcc/arm-none-eabi/10.3.1/../../../../arm-none-eabi/lib/thumb/v8-m.main+fp/hard\libc_nano.a(lib_a-lseekr.o)
                              c:/renesas/ra/e2studio_v2022-10_fsp_v4.2.0/toolchains/gcc_arm/gcc-arm-none-eabi-10.3-2021.10/bin/../lib/gcc/arm-none-eabi/10.3.1/../../../../arm-none-eabi/lib/thumb/v8-m.main+fp/hard\libc_nano.a(lib_a-stdio.o) (_lseek_r)
c:/renesas/ra/e2studio_v2022-10_fsp_v4.2.0/toolchains/gcc_arm/gcc-arm-none-eabi-10.3-2021.10/bin/../lib/gcc/arm-none-eabi/10.3.1/../../../../arm-none-eabi/lib/thumb/v8-m.main+fp/hard\libc_nano.a(lib_a-mlock.o)
                              c:/renesas/ra/e2studio_v2022-10_fsp_v4.2.0/toolchains/gcc_arm/gcc-arm-none-eabi-10.3-2021.10/bin/../lib/gcc/arm-none-eabi/10.3.1/../../../../arm-none-eabi/lib/thumb/v8-m.main+fp/hard\libc_nano.a(lib_a-nano-mallocr.o) (__malloc_lock)
c:/renesas/ra/e2studio_v2022-10_fsp_v4.2.0/toolchains/gcc_arm/gcc-arm-none-eabi-10.3-2021.10/bin/../lib/gcc/arm-none-eabi/10.3.1/../../../../arm-none-eabi/lib/thumb/v8-m.main+fp/hard\libc_nano.a(lib_a-nano-freer.o)
                              c:/renesas/ra/e2studio_v2022-10_fsp_v4.2.0/toolchains/gcc_arm/gcc-arm-none-eabi-10.3-2021.10/bin/../lib/gcc/arm-none-eabi/10.3.1/../../../../arm-none-eabi/lib/thumb/v8-m.main+fp/hard\libc_nano.a(lib_a-fflush.o) (_free_r)
c:/renesas/ra/e2studio_v2022-10_fsp_v4.2.0/toolchains/gcc_arm/gcc-arm-none-eabi-10.3-2021.10/bin/../lib/gcc/arm-none-eabi/10.3.1/../../../../arm-none-eabi/lib/thumb/v8-m.main+fp/hard\libc_nano.a(lib_a-readr.o)
                              c:/renesas/ra/e2studio_v2022-10_fsp_v4.2.0/toolchains/gcc_arm/gcc-arm-none-eabi-10.3-2021.10/bin/../lib/gcc/arm-none-eabi/10.3.1/../../../../arm-none-eabi/lib/thumb/v8-m.main+fp/hard\libc_nano.a(lib_a-stdio.o) (_read_r)
c:/renesas/ra/e2studio_v2022-10_fsp_v4.2.0/toolchains/gcc_arm/gcc-arm-none-eabi-10.3-2021.10/bin/../lib/gcc/arm-none-eabi/10.3.1/../../../../arm-none-eabi/lib/thumb/v8-m.main+fp/hard\libc_nano.a(lib_a-reent.o)
                              c:/renesas/ra/e2studio_v2022-10_fsp_v4.2.0/toolchains/gcc_arm/gcc-arm-none-eabi-10.3-2021.10/bin/../lib/gcc/arm-none-eabi/10.3.1/../../../../arm-none-eabi/lib/thumb/v8-m.main+fp/hard\libc_nano.a(lib_a-sbrkr.o) (errno)

Discarded input sections

 .text          0x00000000        0x0 c:/renesas/ra/e2studio_v2022-10_fsp_v4.2.0/toolchains/gcc_arm/gcc-arm-none-eabi-10.3-2021.10/bin/../lib/gcc/arm-none-eabi/10.3.1/thumb/v8-m.main+fp/hard/crti.o
 .data          0x00000000        0x0 c:/renesas/ra/e2studio_v2022-10_fsp_v4.2.0/toolchains/gcc_arm/gcc-arm-none-eabi-10.3-2021.10/bin/../lib/gcc/arm-none-eabi/10.3.1/thumb/v8-m.main+fp/hard/crti.o
 .bss           0x00000000        0x0 c:/renesas/ra/e2studio_v2022-10_fsp_v4.2.0/toolchains/gcc_arm/gcc-arm-none-eabi-10.3-2021.10/bin/../lib/gcc/arm-none-eabi/10.3.1/thumb/v8-m.main+fp/hard/crti.o
 .data          0x00000000        0x4 c:/renesas/ra/e2studio_v2022-10_fsp_v4.2.0/toolchains/gcc_arm/gcc-arm-none-eabi-10.3-2021.10/bin/../lib/gcc/arm-none-eabi/10.3.1/thumb/v8-m.main+fp/hard/crtbegin.o
 .rodata        0x00000000       0x24 c:/renesas/ra/e2studio_v2022-10_fsp_v4.2.0/toolchains/gcc_arm/gcc-arm-none-eabi-10.3-2021.10/bin/../lib/gcc/arm-none-eabi/10.3.1/thumb/v8-m.main+fp/hard/crtbegin.o
 .text          0x00000000       0xf8 c:/renesas/ra/e2studio_v2022-10_fsp_v4.2.0/toolchains/gcc_arm/gcc-arm-none-eabi-10.3-2021.10/bin/../lib/gcc/arm-none-eabi/10.3.1/../../../../arm-none-eabi/lib/thumb/v8-m.main+fp/hard/rdimon-crt0.o
 .data          0x00000000      0x118 c:/renesas/ra/e2studio_v2022-10_fsp_v4.2.0/toolchains/gcc_arm/gcc-arm-none-eabi-10.3-2021.10/bin/../lib/gcc/arm-none-eabi/10.3.1/../../../../arm-none-eabi/lib/thumb/v8-m.main+fp/hard/rdimon-crt0.o
 .bss           0x00000000        0x0 c:/renesas/ra/e2studio_v2022-10_fsp_v4.2.0/toolchains/gcc_arm/gcc-arm-none-eabi-10.3-2021.10/bin/../lib/gcc/arm-none-eabi/10.3.1/../../../../arm-none-eabi/lib/thumb/v8-m.main+fp/hard/rdimon-crt0.o
 .ARM.extab     0x00000000        0x0 c:/renesas/ra/e2studio_v2022-10_fsp_v4.2.0/toolchains/gcc_arm/gcc-arm-none-eabi-10.3-2021.10/bin/../lib/gcc/arm-none-eabi/10.3.1/../../../../arm-none-eabi/lib/thumb/v8-m.main+fp/hard/rdimon-crt0.o
 .ARM.exidx     0x00000000       0x10 c:/renesas/ra/e2studio_v2022-10_fsp_v4.2.0/toolchains/gcc_arm/gcc-arm-none-eabi-10.3-2021.10/bin/../lib/gcc/arm-none-eabi/10.3.1/../../../../arm-none-eabi/lib/thumb/v8-m.main+fp/hard/rdimon-crt0.o
 .ARM.attributes
                0x00000000       0x20 c:/renesas/ra/e2studio_v2022-10_fsp_v4.2.0/toolchains/gcc_arm/gcc-arm-none-eabi-10.3-2021.10/bin/../lib/gcc/arm-none-eabi/10.3.1/../../../../arm-none-eabi/lib/thumb/v8-m.main+fp/hard/rdimon-crt0.o
 .text          0x00000000        0x0 ./src/hal_entry.o
 .data          0x00000000        0x0 ./src/hal_entry.o
 .bss           0x00000000        0x0 ./src/hal_entry.o
 .text          0x00000000        0x0 ./src/udp_cdc.o
 .data          0x00000000        0x0 ./src/udp_cdc.o
 .bss           0x00000000        0x0 ./src/udp_cdc.o
 .text.udp_tx_buff
                0x00000000       0x14 ./src/udp_cdc.o
 .text.udp_tx_purge
                0x00000000       0x10 ./src/udp_cdc.o
 .rodata.udp_gets.str1.4
                0x00000000        0x4 ./src/udp_cdc.o
 .text.udp_gets
                0x00000000       0xc0 ./src/udp_cdc.o
 .text          0x00000000        0x0 ./src/udp_printf.o
 .data          0x00000000        0x0 ./src/udp_printf.o
 .bss           0x00000000        0x0 ./src/udp_printf.o
 .text          0x00000000        0x0 ./src/usb_desc.o
 .data          0x00000000        0x0 ./src/usb_desc.o
 .bss           0x00000000        0x0 ./src/usb_desc.o
 .text          0x00000000        0x0 ./ra_gen/common_data.o
 .data          0x00000000        0x0 ./ra_gen/common_data.o
 .bss           0x00000000        0x0 ./ra_gen/common_data.o
 .text.g_common_init
                0x00000000        0x4 ./ra_gen/common_data.o
 .rodata.g_ioport
                0x00000000        0xc ./ra_gen/common_data.o
 .text          0x00000000        0x0 ./ra_gen/hal_data.o
 .data          0x00000000        0x0 ./ra_gen/hal_data.o
 .bss           0x00000000        0x0 ./ra_gen/hal_data.o
 .text.g_hal_init
                0x00000000        0x4 ./ra_gen/hal_data.o
 .bss.g_rtc0_ctrl
                0x00000000       0x18 ./ra_gen/hal_data.o
 .rodata.g_basic0
                0x00000000        0xc ./ra_gen/hal_data.o
 .rodata.g_flash0
                0x00000000        0xc ./ra_gen/hal_data.o
 .rodata.g_rtc0
                0x00000000        0xc ./ra_gen/hal_data.o
 .rodata.g_rtc0_cfg
                0x00000000       0x20 ./ra_gen/hal_data.o
 .rodata.g_rtc0_err_cfg
                0x00000000        0x8 ./ra_gen/hal_data.o
 .text          0x00000000        0x0 ./ra_gen/main.o
 .data          0x00000000        0x0 ./ra_gen/main.o
 .bss           0x00000000        0x0 ./ra_gen/main.o
 .text          0x00000000        0x0 ./ra_gen/pin_data.o
 .data          0x00000000        0x0 ./ra_gen/pin_data.o
 .bss           0x00000000        0x0 ./ra_gen/pin_data.o
 .text          0x00000000        0x0 ./ra_gen/vector_data.o
 .data          0x00000000        0x0 ./ra_gen/vector_data.o
 .bss           0x00000000        0x0 ./ra_gen/vector_data.o
 .text          0x00000000        0x0 ./ra/fsp/src/r_usb_pcdc/src/r_usb_pcdc_driver.o
 .data          0x00000000        0x0 ./ra/fsp/src/r_usb_pcdc/src/r_usb_pcdc_driver.o
 .bss           0x00000000        0x0 ./ra/fsp/src/r_usb_pcdc/src/r_usb_pcdc_driver.o
 .text          0x00000000        0x0 ./ra/fsp/src/r_usb_basic/src/hw/r_usb_creg_abs.o
 .data          0x00000000        0x0 ./ra/fsp/src/r_usb_basic/src/hw/r_usb_creg_abs.o
 .bss           0x00000000        0x0 ./ra/fsp/src/r_usb_basic/src/hw/r_usb_creg_abs.o
 .text          0x00000000        0x0 ./ra/fsp/src/r_usb_basic/src/hw/r_usb_creg_access.o
 .data          0x00000000        0x0 ./ra/fsp/src/r_usb_basic/src/hw/r_usb_creg_access.o
 .bss           0x00000000        0x0 ./ra/fsp/src/r_usb_basic/src/hw/r_usb_creg_access.o
 .text.hw_usb_get_fifosel_adr.isra.0
                0x00000000       0x64 ./ra/fsp/src/r_usb_basic/src/hw/r_usb_creg_access.o
 .text.hw_usb_set_dcfm
                0x00000000       0x2c ./ra/fsp/src/r_usb_basic/src/hw/r_usb_creg_access.o
 .text.hw_usb_clear_dcfm
                0x00000000       0x34 ./ra/fsp/src/r_usb_basic/src/hw/r_usb_creg_access.o
 .text.hw_usb_set_usbe
                0x00000000       0x3c ./ra/fsp/src/r_usb_basic/src/hw/r_usb_creg_access.o
 .text.hw_usb_clear_usbe
                0x00000000       0x34 ./ra/fsp/src/r_usb_basic/src/hw/r_usb_creg_access.o
 .text.hw_usb_set_dclrm
                0x00000000       0x6c ./ra/fsp/src/r_usb_basic/src/hw/r_usb_creg_access.o
 .text.hw_usb_clear_dclrm
                0x00000000       0x6c ./ra/fsp/src/r_usb_basic/src/hw/r_usb_creg_access.o
 .text.hw_usb_set_dreqe
                0x00000000       0x40 ./ra/fsp/src/r_usb_basic/src/hw/r_usb_creg_access.o
 .text.hw_usb_clear_dreqe
                0x00000000       0x6c ./ra/fsp/src/r_usb_basic/src/hw/r_usb_creg_access.o
 .text.hw_usb_set_curpipe
                0x00000000       0x74 ./ra/fsp/src/r_usb_basic/src/hw/r_usb_creg_access.o
 .text.hw_usb_write_intenb
                0x00000000       0x2c ./ra/fsp/src/r_usb_basic/src/hw/r_usb_creg_access.o
 .text.hw_usb_set_intenb
                0x00000000       0x38 ./ra/fsp/src/r_usb_basic/src/hw/r_usb_creg_access.o
 .text.hw_usb_set_sofcfg
                0x00000000       0x10 ./ra/fsp/src/r_usb_basic/src/hw/r_usb_creg_access.o
 .text.hw_usb_write_intsts
                0x00000000       0x30 ./ra/fsp/src/r_usb_basic/src/hw/r_usb_creg_access.o
 .text.hw_usb_set_sqset
                0x00000000       0x74 ./ra/fsp/src/r_usb_basic/src/hw/r_usb_creg_access.o
 .text          0x00000000        0x0 ./ra/fsp/src/r_usb_basic/src/hw/r_usb_dma.o
 .data          0x00000000        0x0 ./ra/fsp/src/r_usb_basic/src/hw/r_usb_dma.o
 .bss           0x00000000        0x0 ./ra/fsp/src/r_usb_basic/src/hw/r_usb_dma.o
 .debug_info    0x00000000       0x6b ./ra/fsp/src/r_usb_basic/src/hw/r_usb_dma.o
 .debug_abbrev  0x00000000       0x26 ./ra/fsp/src/r_usb_basic/src/hw/r_usb_dma.o
 .debug_aranges
                0x00000000       0x18 ./ra/fsp/src/r_usb_basic/src/hw/r_usb_dma.o
 .debug_line    0x00000000       0x1d ./ra/fsp/src/r_usb_basic/src/hw/r_usb_dma.o
 .debug_str     0x00000000      0x1c2 ./ra/fsp/src/r_usb_basic/src/hw/r_usb_dma.o
 .comment       0x00000000       0x4a ./ra/fsp/src/r_usb_basic/src/hw/r_usb_dma.o
 .ARM.attributes
                0x00000000       0x3a ./ra/fsp/src/r_usb_basic/src/hw/r_usb_dma.o
 .text          0x00000000        0x0 ./ra/fsp/src/r_usb_basic/src/hw/r_usb_hostelectrical.o
 .data          0x00000000        0x0 ./ra/fsp/src/r_usb_basic/src/hw/r_usb_hostelectrical.o
 .bss           0x00000000        0x0 ./ra/fsp/src/r_usb_basic/src/hw/r_usb_hostelectrical.o
 .debug_info    0x00000000       0x6b ./ra/fsp/src/r_usb_basic/src/hw/r_usb_hostelectrical.o
 .debug_abbrev  0x00000000       0x26 ./ra/fsp/src/r_usb_basic/src/hw/r_usb_hostelectrical.o
 .debug_aranges
                0x00000000       0x18 ./ra/fsp/src/r_usb_basic/src/hw/r_usb_hostelectrical.o
 .debug_line    0x00000000       0x1d ./ra/fsp/src/r_usb_basic/src/hw/r_usb_hostelectrical.o
 .debug_str     0x00000000      0x1cd ./ra/fsp/src/r_usb_basic/src/hw/r_usb_hostelectrical.o
 .comment       0x00000000       0x4a ./ra/fsp/src/r_usb_basic/src/hw/r_usb_hostelectrical.o
 .ARM.attributes
                0x00000000       0x3a ./ra/fsp/src/r_usb_basic/src/hw/r_usb_hostelectrical.o
 .text          0x00000000        0x0 ./ra/fsp/src/r_usb_basic/src/hw/r_usb_hreg_abs.o
 .data          0x00000000        0x0 ./ra/fsp/src/r_usb_basic/src/hw/r_usb_hreg_abs.o
 .bss           0x00000000        0x0 ./ra/fsp/src/r_usb_basic/src/hw/r_usb_hreg_abs.o
 .debug_info    0x00000000       0x6b ./ra/fsp/src/r_usb_basic/src/hw/r_usb_hreg_abs.o
 .debug_abbrev  0x00000000       0x26 ./ra/fsp/src/r_usb_basic/src/hw/r_usb_hreg_abs.o
 .debug_aranges
                0x00000000       0x18 ./ra/fsp/src/r_usb_basic/src/hw/r_usb_hreg_abs.o
 .debug_line    0x00000000       0x1d ./ra/fsp/src/r_usb_basic/src/hw/r_usb_hreg_abs.o
 .debug_str     0x00000000      0x1c7 ./ra/fsp/src/r_usb_basic/src/hw/r_usb_hreg_abs.o
 .comment       0x00000000       0x4a ./ra/fsp/src/r_usb_basic/src/hw/r_usb_hreg_abs.o
 .ARM.attributes
                0x00000000       0x3a ./ra/fsp/src/r_usb_basic/src/hw/r_usb_hreg_abs.o
 .text          0x00000000        0x0 ./ra/fsp/src/r_usb_basic/src/hw/r_usb_hreg_access.o
 .data          0x00000000        0x0 ./ra/fsp/src/r_usb_basic/src/hw/r_usb_hreg_access.o
 .bss           0x00000000        0x0 ./ra/fsp/src/r_usb_basic/src/hw/r_usb_hreg_access.o
 .debug_info    0x00000000       0x6b ./ra/fsp/src/r_usb_basic/src/hw/r_usb_hreg_access.o
 .debug_abbrev  0x00000000       0x26 ./ra/fsp/src/r_usb_basic/src/hw/r_usb_hreg_access.o
 .debug_aranges
                0x00000000       0x18 ./ra/fsp/src/r_usb_basic/src/hw/r_usb_hreg_access.o
 .debug_line    0x00000000       0x1d ./ra/fsp/src/r_usb_basic/src/hw/r_usb_hreg_access.o
 .debug_str     0x00000000      0x1ca ./ra/fsp/src/r_usb_basic/src/hw/r_usb_hreg_access.o
 .comment       0x00000000       0x4a ./ra/fsp/src/r_usb_basic/src/hw/r_usb_hreg_access.o
 .ARM.attributes
                0x00000000       0x3a ./ra/fsp/src/r_usb_basic/src/hw/r_usb_hreg_access.o
 .text          0x00000000        0x0 ./ra/fsp/src/r_usb_basic/src/hw/r_usb_mcu.o
 .data          0x00000000        0x0 ./ra/fsp/src/r_usb_basic/src/hw/r_usb_mcu.o
 .bss           0x00000000        0x0 ./ra/fsp/src/r_usb_basic/src/hw/r_usb_mcu.o
 .text.usb_check_use_usba_module
                0x00000000        0x4 ./ra/fsp/src/r_usb_basic/src/hw/r_usb_mcu.o
 .text.usbhs_interrupt_handler
                0x00000000       0x24 ./ra/fsp/src/r_usb_basic/src/hw/r_usb_mcu.o
 .text.usbhs_d0fifo_handler
                0x00000000       0x24 ./ra/fsp/src/r_usb_basic/src/hw/r_usb_mcu.o
 .text.usbhs_d1fifo_handler
                0x00000000       0x24 ./ra/fsp/src/r_usb_basic/src/hw/r_usb_mcu.o
 .text          0x00000000        0x0 ./ra/fsp/src/r_usb_basic/src/hw/r_usb_preg_abs.o
 .data          0x00000000        0x0 ./ra/fsp/src/r_usb_basic/src/hw/r_usb_preg_abs.o
 .bss           0x00000000        0x0 ./ra/fsp/src/r_usb_basic/src/hw/r_usb_preg_abs.o
 .text.usb_pstd_remote_wakeup
                0x00000000       0x48 ./ra/fsp/src/r_usb_basic/src/hw/r_usb_preg_abs.o
 .text.usb_pstd_self_clock
                0x00000000       0x20 ./ra/fsp/src/r_usb_basic/src/hw/r_usb_preg_abs.o
 .text          0x00000000        0x0 ./ra/fsp/src/r_usb_basic/src/hw/r_usb_preg_access.o
 .data          0x00000000        0x0 ./ra/fsp/src/r_usb_basic/src/hw/r_usb_preg_access.o
 .bss           0x00000000        0x0 ./ra/fsp/src/r_usb_basic/src/hw/r_usb_preg_access.o
 .text.hw_usb_pset_wkup
                0x00000000       0x28 ./ra/fsp/src/r_usb_basic/src/hw/r_usb_preg_access.o
 .text.hw_usb_pcontrol_dprpu
                0x00000000       0x30 ./ra/fsp/src/r_usb_basic/src/hw/r_usb_preg_access.o
 .text          0x00000000        0x0 ./ra/fsp/src/r_usb_basic/src/driver/r_usb_cdataio.o
 .data          0x00000000        0x0 ./ra/fsp/src/r_usb_basic/src/driver/r_usb_cdataio.o
 .bss           0x00000000        0x0 ./ra/fsp/src/r_usb_basic/src/driver/r_usb_cdataio.o
 .text.usb_cstd_debug_hook
                0x00000000        0x4 ./ra/fsp/src/r_usb_basic/src/driver/r_usb_cdataio.o
 .text.usb_ctrl_stop
                0x00000000       0x24 ./ra/fsp/src/r_usb_basic/src/driver/r_usb_cdataio.o
 .text.usb_get_usepipe
                0x00000000       0x1c ./ra/fsp/src/r_usb_basic/src/driver/r_usb_cdataio.o
 .text          0x00000000        0x0 ./ra/fsp/src/r_usb_basic/src/driver/r_usb_clibusbip.o
 .data          0x00000000        0x0 ./ra/fsp/src/r_usb_basic/src/driver/r_usb_clibusbip.o
 .bss           0x00000000        0x0 ./ra/fsp/src/r_usb_basic/src/driver/r_usb_clibusbip.o
 .text.usb_class_task
                0x00000000        0x4 ./ra/fsp/src/r_usb_basic/src/driver/r_usb_clibusbip.o
 .text.usb_cstd_remote_wakeup
                0x00000000       0x30 ./ra/fsp/src/r_usb_basic/src/driver/r_usb_clibusbip.o
 .text          0x00000000        0x0 ./ra/fsp/src/r_usb_basic/src/driver/r_usb_cstd_rtos.o
 .data          0x00000000        0x0 ./ra/fsp/src/r_usb_basic/src/driver/r_usb_cstd_rtos.o
 .bss           0x00000000        0x0 ./ra/fsp/src/r_usb_basic/src/driver/r_usb_cstd_rtos.o
 .debug_info    0x00000000       0x6b ./ra/fsp/src/r_usb_basic/src/driver/r_usb_cstd_rtos.o
 .debug_abbrev  0x00000000       0x26 ./ra/fsp/src/r_usb_basic/src/driver/r_usb_cstd_rtos.o
 .debug_aranges
                0x00000000       0x18 ./ra/fsp/src/r_usb_basic/src/driver/r_usb_cstd_rtos.o
 .debug_line    0x00000000       0x1d ./ra/fsp/src/r_usb_basic/src/driver/r_usb_cstd_rtos.o
 .debug_str     0x00000000      0x1cc ./ra/fsp/src/r_usb_basic/src/driver/r_usb_cstd_rtos.o
 .comment       0x00000000       0x4a ./ra/fsp/src/r_usb_basic/src/driver/r_usb_cstd_rtos.o
 .ARM.attributes
                0x00000000       0x3a ./ra/fsp/src/r_usb_basic/src/driver/r_usb_cstd_rtos.o
 .text          0x00000000        0x0 ./ra/fsp/src/r_usb_basic/src/driver/r_usb_hbc.o
 .data          0x00000000        0x0 ./ra/fsp/src/r_usb_basic/src/driver/r_usb_hbc.o
 .bss           0x00000000        0x0 ./ra/fsp/src/r_usb_basic/src/driver/r_usb_hbc.o
 .debug_info    0x00000000       0x6b ./ra/fsp/src/r_usb_basic/src/driver/r_usb_hbc.o
 .debug_abbrev  0x00000000       0x26 ./ra/fsp/src/r_usb_basic/src/driver/r_usb_hbc.o
 .debug_aranges
                0x00000000       0x18 ./ra/fsp/src/r_usb_basic/src/driver/r_usb_hbc.o
 .debug_line    0x00000000       0x1d ./ra/fsp/src/r_usb_basic/src/driver/r_usb_hbc.o
 .debug_str     0x00000000      0x1c6 ./ra/fsp/src/r_usb_basic/src/driver/r_usb_hbc.o
 .comment       0x00000000       0x4a ./ra/fsp/src/r_usb_basic/src/driver/r_usb_hbc.o
 .ARM.attributes
                0x00000000       0x3a ./ra/fsp/src/r_usb_basic/src/driver/r_usb_hbc.o
 .text          0x00000000        0x0 ./ra/fsp/src/r_usb_basic/src/driver/r_usb_hcontrolrw.o
 .data          0x00000000        0x0 ./ra/fsp/src/r_usb_basic/src/driver/r_usb_hcontrolrw.o
 .bss           0x00000000        0x0 ./ra/fsp/src/r_usb_basic/src/driver/r_usb_hcontrolrw.o
 .debug_info    0x00000000       0x6b ./ra/fsp/src/r_usb_basic/src/driver/r_usb_hcontrolrw.o
 .debug_abbrev  0x00000000       0x26 ./ra/fsp/src/r_usb_basic/src/driver/r_usb_hcontrolrw.o
 .debug_aranges
                0x00000000       0x18 ./ra/fsp/src/r_usb_basic/src/driver/r_usb_hcontrolrw.o
 .debug_line    0x00000000       0x1d ./ra/fsp/src/r_usb_basic/src/driver/r_usb_hcontrolrw.o
 .debug_str     0x00000000      0x1cd ./ra/fsp/src/r_usb_basic/src/driver/r_usb_hcontrolrw.o
 .comment       0x00000000       0x4a ./ra/fsp/src/r_usb_basic/src/driver/r_usb_hcontrolrw.o
 .ARM.attributes
                0x00000000       0x3a ./ra/fsp/src/r_usb_basic/src/driver/r_usb_hcontrolrw.o
 .text          0x00000000        0x0 ./ra/fsp/src/r_usb_basic/src/driver/r_usb_hdriver.o
 .data          0x00000000        0x0 ./ra/fsp/src/r_usb_basic/src/driver/r_usb_hdriver.o
 .bss           0x00000000        0x0 ./ra/fsp/src/r_usb_basic/src/driver/r_usb_hdriver.o
 .debug_info    0x00000000       0x6b ./ra/fsp/src/r_usb_basic/src/driver/r_usb_hdriver.o
 .debug_abbrev  0x00000000       0x26 ./ra/fsp/src/r_usb_basic/src/driver/r_usb_hdriver.o
 .debug_aranges
                0x00000000       0x18 ./ra/fsp/src/r_usb_basic/src/driver/r_usb_hdriver.o
 .debug_line    0x00000000       0x1d ./ra/fsp/src/r_usb_basic/src/driver/r_usb_hdriver.o
 .debug_str     0x00000000      0x1ca ./ra/fsp/src/r_usb_basic/src/driver/r_usb_hdriver.o
 .comment       0x00000000       0x4a ./ra/fsp/src/r_usb_basic/src/driver/r_usb_hdriver.o
 .ARM.attributes
                0x00000000       0x3a ./ra/fsp/src/r_usb_basic/src/driver/r_usb_hdriver.o
 .text          0x00000000        0x0 ./ra/fsp/src/r_usb_basic/src/driver/r_usb_hhubsys.o
 .data          0x00000000        0x0 ./ra/fsp/src/r_usb_basic/src/driver/r_usb_hhubsys.o
 .bss           0x00000000        0x0 ./ra/fsp/src/r_usb_basic/src/driver/r_usb_hhubsys.o
 .debug_info    0x00000000       0x6b ./ra/fsp/src/r_usb_basic/src/driver/r_usb_hhubsys.o
 .debug_abbrev  0x00000000       0x26 ./ra/fsp/src/r_usb_basic/src/driver/r_usb_hhubsys.o
 .debug_aranges
                0x00000000       0x18 ./ra/fsp/src/r_usb_basic/src/driver/r_usb_hhubsys.o
 .debug_line    0x00000000       0x1d ./ra/fsp/src/r_usb_basic/src/driver/r_usb_hhubsys.o
 .debug_str     0x00000000      0x1ca ./ra/fsp/src/r_usb_basic/src/driver/r_usb_hhubsys.o
 .comment       0x00000000       0x4a ./ra/fsp/src/r_usb_basic/src/driver/r_usb_hhubsys.o
 .ARM.attributes
                0x00000000       0x3a ./ra/fsp/src/r_usb_basic/src/driver/r_usb_hhubsys.o
 .text          0x00000000        0x0 ./ra/fsp/src/r_usb_basic/src/driver/r_usb_hintfifo.o
 .data          0x00000000        0x0 ./ra/fsp/src/r_usb_basic/src/driver/r_usb_hintfifo.o
 .bss           0x00000000        0x0 ./ra/fsp/src/r_usb_basic/src/driver/r_usb_hintfifo.o
 .debug_info    0x00000000       0x6b ./ra/fsp/src/r_usb_basic/src/driver/r_usb_hintfifo.o
 .debug_abbrev  0x00000000       0x26 ./ra/fsp/src/r_usb_basic/src/driver/r_usb_hintfifo.o
 .debug_aranges
                0x00000000       0x18 ./ra/fsp/src/r_usb_basic/src/driver/r_usb_hintfifo.o
 .debug_line    0x00000000       0x1d ./ra/fsp/src/r_usb_basic/src/driver/r_usb_hintfifo.o
 .debug_str     0x00000000      0x1cb ./ra/fsp/src/r_usb_basic/src/driver/r_usb_hintfifo.o
 .comment       0x00000000       0x4a ./ra/fsp/src/r_usb_basic/src/driver/r_usb_hintfifo.o
 .ARM.attributes
                0x00000000       0x3a ./ra/fsp/src/r_usb_basic/src/driver/r_usb_hintfifo.o
 .text          0x00000000        0x0 ./ra/fsp/src/r_usb_basic/src/driver/r_usb_hinthandler_usbip0.o
 .data          0x00000000        0x0 ./ra/fsp/src/r_usb_basic/src/driver/r_usb_hinthandler_usbip0.o
 .bss           0x00000000        0x0 ./ra/fsp/src/r_usb_basic/src/driver/r_usb_hinthandler_usbip0.o
 .debug_info    0x00000000       0x6b ./ra/fsp/src/r_usb_basic/src/driver/r_usb_hinthandler_usbip0.o
 .debug_abbrev  0x00000000       0x26 ./ra/fsp/src/r_usb_basic/src/driver/r_usb_hinthandler_usbip0.o
 .debug_aranges
                0x00000000       0x18 ./ra/fsp/src/r_usb_basic/src/driver/r_usb_hinthandler_usbip0.o
 .debug_line    0x00000000       0x1d ./ra/fsp/src/r_usb_basic/src/driver/r_usb_hinthandler_usbip0.o
 .debug_str     0x00000000      0x1d5 ./ra/fsp/src/r_usb_basic/src/driver/r_usb_hinthandler_usbip0.o
 .comment       0x00000000       0x4a ./ra/fsp/src/r_usb_basic/src/driver/r_usb_hinthandler_usbip0.o
 .ARM.attributes
                0x00000000       0x3a ./ra/fsp/src/r_usb_basic/src/driver/r_usb_hinthandler_usbip0.o
 .text          0x00000000        0x0 ./ra/fsp/src/r_usb_basic/src/driver/r_usb_hinthandler_usbip1.o
 .data          0x00000000        0x0 ./ra/fsp/src/r_usb_basic/src/driver/r_usb_hinthandler_usbip1.o
 .bss           0x00000000        0x0 ./ra/fsp/src/r_usb_basic/src/driver/r_usb_hinthandler_usbip1.o
 .debug_info    0x00000000       0x6b ./ra/fsp/src/r_usb_basic/src/driver/r_usb_hinthandler_usbip1.o
 .debug_abbrev  0x00000000       0x26 ./ra/fsp/src/r_usb_basic/src/driver/r_usb_hinthandler_usbip1.o
 .debug_aranges
                0x00000000       0x18 ./ra/fsp/src/r_usb_basic/src/driver/r_usb_hinthandler_usbip1.o
 .debug_line    0x00000000       0x1d ./ra/fsp/src/r_usb_basic/src/driver/r_usb_hinthandler_usbip1.o
 .debug_str     0x00000000      0x1d5 ./ra/fsp/src/r_usb_basic/src/driver/r_usb_hinthandler_usbip1.o
 .comment       0x00000000       0x4a ./ra/fsp/src/r_usb_basic/src/driver/r_usb_hinthandler_usbip1.o
 .ARM.attributes
                0x00000000       0x3a ./ra/fsp/src/r_usb_basic/src/driver/r_usb_hinthandler_usbip1.o
 .text          0x00000000        0x0 ./ra/fsp/src/r_usb_basic/src/driver/r_usb_hlibusbip.o
 .data          0x00000000        0x0 ./ra/fsp/src/r_usb_basic/src/driver/r_usb_hlibusbip.o
 .bss           0x00000000        0x0 ./ra/fsp/src/r_usb_basic/src/driver/r_usb_hlibusbip.o
 .debug_info    0x00000000       0x6b ./ra/fsp/src/r_usb_basic/src/driver/r_usb_hlibusbip.o
 .debug_abbrev  0x00000000       0x26 ./ra/fsp/src/r_usb_basic/src/driver/r_usb_hlibusbip.o
 .debug_aranges
                0x00000000       0x18 ./ra/fsp/src/r_usb_basic/src/driver/r_usb_hlibusbip.o
 .debug_line    0x00000000       0x1d ./ra/fsp/src/r_usb_basic/src/driver/r_usb_hlibusbip.o
 .debug_str     0x00000000      0x1cc ./ra/fsp/src/r_usb_basic/src/driver/r_usb_hlibusbip.o
 .comment       0x00000000       0x4a ./ra/fsp/src/r_usb_basic/src/driver/r_usb_hlibusbip.o
 .ARM.attributes
                0x00000000       0x3a ./ra/fsp/src/r_usb_basic/src/driver/r_usb_hlibusbip.o
 .text          0x00000000        0x0 ./ra/fsp/src/r_usb_basic/src/driver/r_usb_hmanager.o
 .data          0x00000000        0x0 ./ra/fsp/src/r_usb_basic/src/driver/r_usb_hmanager.o
 .bss           0x00000000        0x0 ./ra/fsp/src/r_usb_basic/src/driver/r_usb_hmanager.o
 .debug_info    0x00000000       0x6b ./ra/fsp/src/r_usb_basic/src/driver/r_usb_hmanager.o
 .debug_abbrev  0x00000000       0x26 ./ra/fsp/src/r_usb_basic/src/driver/r_usb_hmanager.o
 .debug_aranges
                0x00000000       0x18 ./ra/fsp/src/r_usb_basic/src/driver/r_usb_hmanager.o
 .debug_line    0x00000000       0x1d ./ra/fsp/src/r_usb_basic/src/driver/r_usb_hmanager.o
 .debug_str     0x00000000      0x1cb ./ra/fsp/src/r_usb_basic/src/driver/r_usb_hmanager.o
 .comment       0x00000000       0x4a ./ra/fsp/src/r_usb_basic/src/driver/r_usb_hmanager.o
 .ARM.attributes
                0x00000000       0x3a ./ra/fsp/src/r_usb_basic/src/driver/r_usb_hmanager.o
 .text          0x00000000        0x0 ./ra/fsp/src/r_usb_basic/src/driver/r_usb_hscheduler.o
 .data          0x00000000        0x0 ./ra/fsp/src/r_usb_basic/src/driver/r_usb_hscheduler.o
 .bss           0x00000000        0x0 ./ra/fsp/src/r_usb_basic/src/driver/r_usb_hscheduler.o
 .debug_info    0x00000000       0x6b ./ra/fsp/src/r_usb_basic/src/driver/r_usb_hscheduler.o
 .debug_abbrev  0x00000000       0x26 ./ra/fsp/src/r_usb_basic/src/driver/r_usb_hscheduler.o
 .debug_aranges
                0x00000000       0x18 ./ra/fsp/src/r_usb_basic/src/driver/r_usb_hscheduler.o
 .debug_line    0x00000000       0x1d ./ra/fsp/src/r_usb_basic/src/driver/r_usb_hscheduler.o
 .debug_str     0x00000000      0x1cd ./ra/fsp/src/r_usb_basic/src/driver/r_usb_hscheduler.o
 .comment       0x00000000       0x4a ./ra/fsp/src/r_usb_basic/src/driver/r_usb_hscheduler.o
 .ARM.attributes
                0x00000000       0x3a ./ra/fsp/src/r_usb_basic/src/driver/r_usb_hscheduler.o
 .text          0x00000000        0x0 ./ra/fsp/src/r_usb_basic/src/driver/r_usb_hsignal.o
 .data          0x00000000        0x0 ./ra/fsp/src/r_usb_basic/src/driver/r_usb_hsignal.o
 .bss           0x00000000        0x0 ./ra/fsp/src/r_usb_basic/src/driver/r_usb_hsignal.o
 .debug_info    0x00000000       0x6b ./ra/fsp/src/r_usb_basic/src/driver/r_usb_hsignal.o
 .debug_abbrev  0x00000000       0x26 ./ra/fsp/src/r_usb_basic/src/driver/r_usb_hsignal.o
 .debug_aranges
                0x00000000       0x18 ./ra/fsp/src/r_usb_basic/src/driver/r_usb_hsignal.o
 .debug_line    0x00000000       0x1d ./ra/fsp/src/r_usb_basic/src/driver/r_usb_hsignal.o
 .debug_str     0x00000000      0x1ca ./ra/fsp/src/r_usb_basic/src/driver/r_usb_hsignal.o
 .comment       0x00000000       0x4a ./ra/fsp/src/r_usb_basic/src/driver/r_usb_hsignal.o
 .ARM.attributes
                0x00000000       0x3a ./ra/fsp/src/r_usb_basic/src/driver/r_usb_hsignal.o
 .text          0x00000000        0x0 ./ra/fsp/src/r_usb_basic/src/driver/r_usb_hstdfunction.o
 .data          0x00000000        0x0 ./ra/fsp/src/r_usb_basic/src/driver/r_usb_hstdfunction.o
 .bss           0x00000000        0x0 ./ra/fsp/src/r_usb_basic/src/driver/r_usb_hstdfunction.o
 .debug_info    0x00000000       0x6b ./ra/fsp/src/r_usb_basic/src/driver/r_usb_hstdfunction.o
 .debug_abbrev  0x00000000       0x26 ./ra/fsp/src/r_usb_basic/src/driver/r_usb_hstdfunction.o
 .debug_aranges
                0x00000000       0x18 ./ra/fsp/src/r_usb_basic/src/driver/r_usb_hstdfunction.o
 .debug_line    0x00000000       0x1d ./ra/fsp/src/r_usb_basic/src/driver/r_usb_hstdfunction.o
 .debug_str     0x00000000      0x1cf ./ra/fsp/src/r_usb_basic/src/driver/r_usb_hstdfunction.o
 .comment       0x00000000       0x4a ./ra/fsp/src/r_usb_basic/src/driver/r_usb_hstdfunction.o
 .ARM.attributes
                0x00000000       0x3a ./ra/fsp/src/r_usb_basic/src/driver/r_usb_hstdfunction.o
 .text          0x00000000        0x0 ./ra/fsp/src/r_usb_basic/src/driver/r_usb_pbc.o
 .data          0x00000000        0x0 ./ra/fsp/src/r_usb_basic/src/driver/r_usb_pbc.o
 .bss           0x00000000        0x0 ./ra/fsp/src/r_usb_basic/src/driver/r_usb_pbc.o
 .debug_info    0x00000000       0x6b ./ra/fsp/src/r_usb_basic/src/driver/r_usb_pbc.o
 .debug_abbrev  0x00000000       0x26 ./ra/fsp/src/r_usb_basic/src/driver/r_usb_pbc.o
 .debug_aranges
                0x00000000       0x18 ./ra/fsp/src/r_usb_basic/src/driver/r_usb_pbc.o
 .debug_line    0x00000000       0x1d ./ra/fsp/src/r_usb_basic/src/driver/r_usb_pbc.o
 .debug_str     0x00000000      0x1c6 ./ra/fsp/src/r_usb_basic/src/driver/r_usb_pbc.o
 .comment       0x00000000       0x4a ./ra/fsp/src/r_usb_basic/src/driver/r_usb_pbc.o
 .ARM.attributes
                0x00000000       0x3a ./ra/fsp/src/r_usb_basic/src/driver/r_usb_pbc.o
 .text          0x00000000        0x0 ./ra/fsp/src/r_usb_basic/src/driver/r_usb_pcontrolrw.o
 .data          0x00000000        0x0 ./ra/fsp/src/r_usb_basic/src/driver/r_usb_pcontrolrw.o
 .bss           0x00000000        0x0 ./ra/fsp/src/r_usb_basic/src/driver/r_usb_pcontrolrw.o
 .text          0x00000000        0x0 ./ra/fsp/src/r_usb_basic/src/driver/r_usb_pdriver.o
 .data          0x00000000        0x0 ./ra/fsp/src/r_usb_basic/src/driver/r_usb_pdriver.o
 .bss           0x00000000        0x0 ./ra/fsp/src/r_usb_basic/src/driver/r_usb_pdriver.o
 .text.usb_pstd_clr_alt
                0x00000000       0x10 ./ra/fsp/src/r_usb_basic/src/driver/r_usb_pdriver.o
 .text.usb_pstd_change_device_state
                0x00000000       0x70 ./ra/fsp/src/r_usb_basic/src/driver/r_usb_pdriver.o
 .text.usb_pstd_driver_registration
                0x00000000       0x48 ./ra/fsp/src/r_usb_basic/src/driver/r_usb_pdriver.o
 .text.usb_pstd_device_information
                0x00000000       0x40 ./ra/fsp/src/r_usb_basic/src/driver/r_usb_pdriver.o
 .text.usb_pstd_set_stall_clr_feature
                0x00000000       0x30 ./ra/fsp/src/r_usb_basic/src/driver/r_usb_pdriver.o
 .bss.g_usb_is_otg_attach_interrupt
                0x00000000        0x2 ./ra/fsp/src/r_usb_basic/src/driver/r_usb_pdriver.o
 .bss.g_usb_paud_iso_pipe
                0x00000000        0x8 ./ra/fsp/src/r_usb_basic/src/driver/r_usb_pdriver.o
 .bss.g_usb_pstd_remote_wakeup_state
                0x00000000        0x2 ./ra/fsp/src/r_usb_basic/src/driver/r_usb_pdriver.o
 .text          0x00000000        0x0 ./ra/fsp/src/r_usb_basic/src/driver/r_usb_pintfifo.o
 .data          0x00000000        0x0 ./ra/fsp/src/r_usb_basic/src/driver/r_usb_pintfifo.o
 .bss           0x00000000        0x0 ./ra/fsp/src/r_usb_basic/src/driver/r_usb_pintfifo.o
 .text          0x00000000        0x0 ./ra/fsp/src/r_usb_basic/src/driver/r_usb_pinthandler_usbip0.o
 .data          0x00000000        0x0 ./ra/fsp/src/r_usb_basic/src/driver/r_usb_pinthandler_usbip0.o
 .bss           0x00000000        0x0 ./ra/fsp/src/r_usb_basic/src/driver/r_usb_pinthandler_usbip0.o
 .text          0x00000000        0x0 ./ra/fsp/src/r_usb_basic/src/driver/r_usb_plibusbip.o
 .data          0x00000000        0x0 ./ra/fsp/src/r_usb_basic/src/driver/r_usb_plibusbip.o
 .bss           0x00000000        0x0 ./ra/fsp/src/r_usb_basic/src/driver/r_usb_plibusbip.o
 .text.usb_pstd_get_pipe_no
                0x00000000       0x68 ./ra/fsp/src/r_usb_basic/src/driver/r_usb_plibusbip.o
 .text          0x00000000        0x0 ./ra/fsp/src/r_usb_basic/src/driver/r_usb_psignal.o
 .data          0x00000000        0x0 ./ra/fsp/src/r_usb_basic/src/driver/r_usb_psignal.o
 .bss           0x00000000        0x0 ./ra/fsp/src/r_usb_basic/src/driver/r_usb_psignal.o
 .text          0x00000000        0x0 ./ra/fsp/src/r_usb_basic/src/driver/r_usb_pstdfunction.o
 .data          0x00000000        0x0 ./ra/fsp/src/r_usb_basic/src/driver/r_usb_pstdfunction.o
 .bss           0x00000000        0x0 ./ra/fsp/src/r_usb_basic/src/driver/r_usb_pstdfunction.o
 .text          0x00000000        0x0 ./ra/fsp/src/r_usb_basic/src/driver/r_usb_pstdrequest.o
 .data          0x00000000        0x0 ./ra/fsp/src/r_usb_basic/src/driver/r_usb_pstdrequest.o
 .bss           0x00000000        0x0 ./ra/fsp/src/r_usb_basic/src/driver/r_usb_pstdrequest.o
 .text.usb_peri_class_request_ioss
                0x00000000        0x4 ./ra/fsp/src/r_usb_basic/src/driver/r_usb_pstdrequest.o
 .text.usb_peri_class_request_rwds
                0x00000000       0x30 ./ra/fsp/src/r_usb_basic/src/driver/r_usb_pstdrequest.o
 .text.usb_peri_other_request
                0x00000000       0x34 ./ra/fsp/src/r_usb_basic/src/driver/r_usb_pstdrequest.o
 .text.usb_peri_class_request_wnss
                0x00000000       0x3c ./ra/fsp/src/r_usb_basic/src/driver/r_usb_pstdrequest.o
 .text          0x00000000        0x0 ./ra/fsp/src/r_usb_basic/r_usb_basic.o
 .data          0x00000000        0x0 ./ra/fsp/src/r_usb_basic/r_usb_basic.o
 .bss           0x00000000        0x0 ./ra/fsp/src/r_usb_basic/r_usb_basic.o
 .text.R_USB_Callback
                0x00000000        0x8 ./ra/fsp/src/r_usb_basic/r_usb_basic.o
 .text.R_USB_Suspend
                0x00000000        0x8 ./ra/fsp/src/r_usb_basic/r_usb_basic.o
 .text.R_USB_VbusSet
                0x00000000        0x8 ./ra/fsp/src/r_usb_basic/r_usb_basic.o
 .text.R_USB_PipeRead
                0x00000000        0x8 ./ra/fsp/src/r_usb_basic/r_usb_basic.o
 .text.R_USB_PipeStop
                0x00000000        0x8 ./ra/fsp/src/r_usb_basic/r_usb_basic.o
 .text.R_USB_ModuleNumberGet
                0x00000000        0xc ./ra/fsp/src/r_usb_basic/r_usb_basic.o
 .text.R_USB_ClassTypeGet
                0x00000000        0xc ./ra/fsp/src/r_usb_basic/r_usb_basic.o
 .text.R_USB_DeviceAddressGet
                0x00000000        0xc ./ra/fsp/src/r_usb_basic/r_usb_basic.o
 .text.R_USB_PipeNumberGet
                0x00000000        0xc ./ra/fsp/src/r_usb_basic/r_usb_basic.o
 .text.R_USB_DataSizeGet
                0x00000000        0xc ./ra/fsp/src/r_usb_basic/r_usb_basic.o
 .text.R_USB_SetupGet
                0x00000000       0x10 ./ra/fsp/src/r_usb_basic/r_usb_basic.o
 .text.R_USB_OtgCallbackSet
                0x00000000       0x14 ./ra/fsp/src/r_usb_basic/r_usb_basic.o
 .text.R_USB_OtgSRP
                0x00000000       0x10 ./ra/fsp/src/r_usb_basic/r_usb_basic.o
 .text.R_USB_DeviceStateGet
                0x00000000       0x70 ./ra/fsp/src/r_usb_basic/r_usb_basic.o
 .text.R_USB_InfoGet
                0x00000000        0xc ./ra/fsp/src/r_usb_basic/r_usb_basic.o
 .text.R_USB_PipeInfoGet
                0x00000000       0xc4 ./ra/fsp/src/r_usb_basic/r_usb_basic.o
 .text.R_USB_UsedPipesGet
                0x00000000       0x88 ./ra/fsp/src/r_usb_basic/r_usb_basic.o
 .text.R_USB_PullUp
                0x00000000       0x34 ./ra/fsp/src/r_usb_basic/r_usb_basic.o
 .text.R_USB_HostControlTransfer
                0x00000000       0x88 ./ra/fsp/src/r_usb_basic/r_usb_basic.o
 .text.R_USB_RemoteWakeup
                0x00000000       0x30 ./ra/fsp/src/r_usb_basic/r_usb_basic.o
 .text.R_USB_PipeWrite
                0x00000000        0x8 ./ra/fsp/src/r_usb_basic/r_usb_basic.o
 .text.R_USB_Resume
                0x00000000        0x8 ./ra/fsp/src/r_usb_basic/r_usb_basic.o
 .rodata.g_usb_on_usb
                0x00000000       0x7c ./ra/fsp/src/r_usb_basic/r_usb_basic.o
 .text          0x00000000        0x0 ./ra/fsp/src/r_rtc/r_rtc.o
 .data          0x00000000        0x0 ./ra/fsp/src/r_rtc/r_rtc.o
 .bss           0x00000000        0x0 ./ra/fsp/src/r_rtc/r_rtc.o
 .text.R_RTC_CallbackSet
                0x00000000       0x34 ./ra/fsp/src/r_rtc/r_rtc.o
 .text.r_rtc_date_validate
                0x00000000       0xb4 ./ra/fsp/src/r_rtc/r_rtc.o
 .text.R_RTC_InfoGet
                0x00000000       0x34 ./ra/fsp/src/r_rtc/r_rtc.o
 .text.R_RTC_Close
                0x00000000       0xec ./ra/fsp/src/r_rtc/r_rtc.o
 .text.R_RTC_CalendarAlarmGet
                0x00000000      0x100 ./ra/fsp/src/r_rtc/r_rtc.o
 .text.R_RTC_ClockSourceSet
                0x00000000       0xb0 ./ra/fsp/src/r_rtc/r_rtc.o
 .text.R_RTC_CalendarTimeGet
                0x00000000      0x1b8 ./ra/fsp/src/r_rtc/r_rtc.o
 .text.r_rtc_error_adjustment_set.isra.0
                0x00000000       0x84 ./ra/fsp/src/r_rtc/r_rtc.o
 .text.R_RTC_CalendarTimeSet
                0x00000000      0x19c ./ra/fsp/src/r_rtc/r_rtc.o
 .text.R_RTC_ErrorAdjustmentSet
                0x00000000       0x44 ./ra/fsp/src/r_rtc/r_rtc.o
 .text.R_RTC_Open
                0x00000000       0xf8 ./ra/fsp/src/r_rtc/r_rtc.o
 .text.R_RTC_PeriodicIrqRateSet
                0x00000000       0x9c ./ra/fsp/src/r_rtc/r_rtc.o
 .text.R_RTC_CalendarAlarmSet
                0x00000000      0x32c ./ra/fsp/src/r_rtc/r_rtc.o
 .text.rtc_alarm_periodic_isr
                0x00000000       0x6c ./ra/fsp/src/r_rtc/r_rtc.o
 .rodata.days_in_months
                0x00000000        0xc ./ra/fsp/src/r_rtc/r_rtc.o
 .rodata.g_rtc_on_rtc
                0x00000000       0x2c ./ra/fsp/src/r_rtc/r_rtc.o
 .text          0x00000000        0x0 ./ra/fsp/src/r_ioport/r_ioport.o
 .data          0x00000000        0x0 ./ra/fsp/src/r_ioport/r_ioport.o
 .bss           0x00000000        0x0 ./ra/fsp/src/r_ioport/r_ioport.o
 .text.R_IOPORT_PinRead
                0x00000000       0x34 ./ra/fsp/src/r_ioport/r_ioport.o
 .text.R_IOPORT_PortRead
                0x00000000       0x2c ./ra/fsp/src/r_ioport/r_ioport.o
 .text.R_IOPORT_PortWrite
                0x00000000       0x48 ./ra/fsp/src/r_ioport/r_ioport.o
 .text.R_IOPORT_PinWrite
                0x00000000       0x40 ./ra/fsp/src/r_ioport/r_ioport.o
 .text.R_IOPORT_PortDirectionSet
                0x00000000       0x4c ./ra/fsp/src/r_ioport/r_ioport.o
 .text.R_IOPORT_PortEventInputRead
                0x00000000       0x40 ./ra/fsp/src/r_ioport/r_ioport.o
 .text.R_IOPORT_PinEventInputRead
                0x00000000       0x58 ./ra/fsp/src/r_ioport/r_ioport.o
 .text.R_IOPORT_PortEventOutputWrite
                0x00000000       0x50 ./ra/fsp/src/r_ioport/r_ioport.o
 .text.R_IOPORT_PinEventOutputWrite
                0x00000000       0x64 ./ra/fsp/src/r_ioport/r_ioport.o
 .text.R_IOPORT_PinCfg
                0x00000000       0xc0 ./ra/fsp/src/r_ioport/r_ioport.o
 .text.R_IOPORT_PinsCfg
                0x00000000       0x2c ./ra/fsp/src/r_ioport/r_ioport.o
 .rodata.g_ioport_on_ioport
                0x00000000       0x34 ./ra/fsp/src/r_ioport/r_ioport.o
 .text          0x00000000        0x0 ./ra/fsp/src/r_flash_hp/r_flash_hp.o
 .data          0x00000000        0x0 ./ra/fsp/src/r_flash_hp/r_flash_hp.o
 .bss           0x00000000        0x0 ./ra/fsp/src/r_flash_hp/r_flash_hp.o
 .text.R_FLASH_HP_IdCodeSet
                0x00000000        0x4 ./ra/fsp/src/r_flash_hp/r_flash_hp.o
 .text.R_FLASH_HP_AccessWindowSet
                0x00000000        0x4 ./ra/fsp/src/r_flash_hp/r_flash_hp.o
 .text.R_FLASH_HP_AccessWindowClear
                0x00000000        0x4 ./ra/fsp/src/r_flash_hp/r_flash_hp.o
 .text.R_FLASH_HP_CallbackSet
                0x00000000       0x34 ./ra/fsp/src/r_flash_hp/r_flash_hp.o
 .text.r_flash_hp_call_callback
                0x00000000       0x38 ./ra/fsp/src/r_flash_hp/r_flash_hp.o
 .text.R_FLASH_HP_StatusGet
                0x00000000       0x30 ./ra/fsp/src/r_flash_hp/r_flash_hp.o
 .text.R_FLASH_HP_InfoGet
                0x00000000       0x48 ./ra/fsp/src/r_flash_hp/r_flash_hp.o
 .text.R_FLASH_HP_BankSwap
                0x00000000        0x4 ./ra/fsp/src/r_flash_hp/r_flash_hp.o
 .text.R_FLASH_HP_UpdateFlashClockFreq
                0x00000000       0x30 ./ra/fsp/src/r_flash_hp/r_flash_hp.o
 .text.R_FLASH_HP_BlankCheck
                0x00000000       0x84 ./ra/fsp/src/r_flash_hp/r_flash_hp.o
 .text.R_FLASH_HP_Reset
                0x00000000       0x1c ./ra/fsp/src/r_flash_hp/r_flash_hp.o
 .text.R_FLASH_HP_StartUpAreaSelect
                0x00000000       0x48 ./ra/fsp/src/r_flash_hp/r_flash_hp.o
 .text.fcu_fiferr_isr
                0x00000000       0x78 ./ra/fsp/src/r_flash_hp/r_flash_hp.o
 .text.fcu_frdyi_isr
                0x00000000       0x94 ./ra/fsp/src/r_flash_hp/r_flash_hp.o
 .rodata.g_code_flash_macro_info
                0x00000000       0x20 ./ra/fsp/src/r_flash_hp/r_flash_hp.o
 .rodata.g_data_flash_macro_info
                0x00000000       0x10 ./ra/fsp/src/r_flash_hp/r_flash_hp.o
 .rodata.g_flash_code_region
                0x00000000        0x8 ./ra/fsp/src/r_flash_hp/r_flash_hp.o
 .rodata.g_flash_data_region
                0x00000000        0x8 ./ra/fsp/src/r_flash_hp/r_flash_hp.o
 .rodata.g_flash_on_flash_hp
                0x00000000       0x3c ./ra/fsp/src/r_flash_hp/r_flash_hp.o
 .text          0x00000000        0x0 ./ra/fsp/src/bsp/mcu/all/bsp_clocks.o
 .data          0x00000000        0x0 ./ra/fsp/src/bsp/mcu/all/bsp_clocks.o
 .bss           0x00000000        0x0 ./ra/fsp/src/bsp/mcu/all/bsp_clocks.o
 .text.bsp_prv_operating_mode_set
                0x00000000       0x60 ./ra/fsp/src/bsp/mcu/all/bsp_clocks.o
 .text.bsp_prv_prepare_pll
                0x00000000        0xc ./ra/fsp/src/bsp/mcu/all/bsp_clocks.o
 .text.prv_clock_dividers_set
                0x00000000        0xc ./ra/fsp/src/bsp/mcu/all/bsp_clocks.o
 .text.bsp_prv_clock_set
                0x00000000       0xb0 ./ra/fsp/src/bsp/mcu/all/bsp_clocks.o
 .text.R_BSP_SubClockStabilizeWait
                0x00000000        0x8 ./ra/fsp/src/bsp/mcu/all/bsp_clocks.o
 .text.R_BSP_OctaclkUpdate
                0x00000000        0x4 ./ra/fsp/src/bsp/mcu/all/bsp_clocks.o
 .text.R_BSP_SourceClockHzGet
                0x00000000        0xc ./ra/fsp/src/bsp/mcu/all/bsp_clocks.o
 .text          0x00000000        0x0 ./ra/fsp/src/bsp/mcu/all/bsp_common.o
 .data          0x00000000        0x0 ./ra/fsp/src/bsp/mcu/all/bsp_common.o
 .bss           0x00000000        0x0 ./ra/fsp/src/bsp/mcu/all/bsp_common.o
 .text.R_FSP_VersionGet
                0x00000000       0x14 ./ra/fsp/src/bsp/mcu/all/bsp_common.o
 .text.__assert_func
                0x00000000        0x4 ./ra/fsp/src/bsp/mcu/all/bsp_common.o
 .text          0x00000000        0x0 ./ra/fsp/src/bsp/mcu/all/bsp_delay.o
 .data          0x00000000        0x0 ./ra/fsp/src/bsp/mcu/all/bsp_delay.o
 .bss           0x00000000        0x0 ./ra/fsp/src/bsp/mcu/all/bsp_delay.o
 .text          0x00000000        0x0 ./ra/fsp/src/bsp/mcu/all/bsp_group_irq.o
 .data          0x00000000        0x0 ./ra/fsp/src/bsp/mcu/all/bsp_group_irq.o
 .bss           0x00000000        0x0 ./ra/fsp/src/bsp/mcu/all/bsp_group_irq.o
 .text.R_BSP_GroupIrqWrite
                0x00000000       0x18 ./ra/fsp/src/bsp/mcu/all/bsp_group_irq.o
 .text          0x00000000        0x0 ./ra/fsp/src/bsp/mcu/all/bsp_guard.o
 .data          0x00000000        0x0 ./ra/fsp/src/bsp/mcu/all/bsp_guard.o
 .bss           0x00000000        0x0 ./ra/fsp/src/bsp/mcu/all/bsp_guard.o
 .debug_info    0x00000000       0x6b ./ra/fsp/src/bsp/mcu/all/bsp_guard.o
 .debug_abbrev  0x00000000       0x26 ./ra/fsp/src/bsp/mcu/all/bsp_guard.o
 .debug_aranges
                0x00000000       0x18 ./ra/fsp/src/bsp/mcu/all/bsp_guard.o
 .debug_line    0x00000000       0x1d ./ra/fsp/src/bsp/mcu/all/bsp_guard.o
 .debug_str     0x00000000      0x1bb ./ra/fsp/src/bsp/mcu/all/bsp_guard.o
 .comment       0x00000000       0x4a ./ra/fsp/src/bsp/mcu/all/bsp_guard.o
 .ARM.attributes
                0x00000000       0x3a ./ra/fsp/src/bsp/mcu/all/bsp_guard.o
 .text          0x00000000        0x0 ./ra/fsp/src/bsp/mcu/all/bsp_io.o
 .data          0x00000000        0x0 ./ra/fsp/src/bsp/mcu/all/bsp_io.o
 .bss           0x00000000        0x0 ./ra/fsp/src/bsp/mcu/all/bsp_io.o
 .text          0x00000000        0x0 ./ra/fsp/src/bsp/mcu/all/bsp_irq.o
 .data          0x00000000        0x0 ./ra/fsp/src/bsp/mcu/all/bsp_irq.o
 .bss           0x00000000        0x0 ./ra/fsp/src/bsp/mcu/all/bsp_irq.o
 .rodata.g_interrupt_event_link_select
                0x00000000       0xc0 ./ra/fsp/src/bsp/mcu/all/bsp_irq.o
 .text          0x00000000        0x0 ./ra/fsp/src/bsp/mcu/all/bsp_register_protection.o
 .data          0x00000000        0x0 ./ra/fsp/src/bsp/mcu/all/bsp_register_protection.o
 .bss           0x00000000        0x0 ./ra/fsp/src/bsp/mcu/all/bsp_register_protection.o
 .text          0x00000000        0x0 ./ra/fsp/src/bsp/mcu/all/bsp_rom_registers.o
 .data          0x00000000        0x0 ./ra/fsp/src/bsp/mcu/all/bsp_rom_registers.o
 .bss           0x00000000        0x0 ./ra/fsp/src/bsp/mcu/all/bsp_rom_registers.o
 .text          0x00000000        0x0 ./ra/fsp/src/bsp/mcu/all/bsp_sbrk.o
 .data          0x00000000        0x0 ./ra/fsp/src/bsp/mcu/all/bsp_sbrk.o
 .bss           0x00000000        0x0 ./ra/fsp/src/bsp/mcu/all/bsp_sbrk.o
 .text._sbrk    0x00000000       0x44 ./ra/fsp/src/bsp/mcu/all/bsp_sbrk.o
 .bss.current_heap_end.0
                0x00000000        0x4 ./ra/fsp/src/bsp/mcu/all/bsp_sbrk.o
 .debug_info    0x00000000      0x13b ./ra/fsp/src/bsp/mcu/all/bsp_sbrk.o
 .debug_abbrev  0x00000000       0xcc ./ra/fsp/src/bsp/mcu/all/bsp_sbrk.o
 .debug_loc     0x00000000      0x11a ./ra/fsp/src/bsp/mcu/all/bsp_sbrk.o
 .debug_aranges
                0x00000000       0x20 ./ra/fsp/src/bsp/mcu/all/bsp_sbrk.o
 .debug_ranges  0x00000000       0x10 ./ra/fsp/src/bsp/mcu/all/bsp_sbrk.o
 .debug_line    0x00000000      0x1f2 ./ra/fsp/src/bsp/mcu/all/bsp_sbrk.o
 .debug_str     0x00000000      0x245 ./ra/fsp/src/bsp/mcu/all/bsp_sbrk.o
 .comment       0x00000000       0x4a ./ra/fsp/src/bsp/mcu/all/bsp_sbrk.o
 .debug_frame   0x00000000       0x28 ./ra/fsp/src/bsp/mcu/all/bsp_sbrk.o
 .ARM.attributes
                0x00000000       0x3a ./ra/fsp/src/bsp/mcu/all/bsp_sbrk.o
 .text          0x00000000        0x0 ./ra/fsp/src/bsp/mcu/all/bsp_security.o
 .data          0x00000000        0x0 ./ra/fsp/src/bsp/mcu/all/bsp_security.o
 .bss           0x00000000        0x0 ./ra/fsp/src/bsp/mcu/all/bsp_security.o
 .rodata.gp_start_of_nonsecure_flash
                0x00000000        0x4 ./ra/fsp/src/bsp/mcu/all/bsp_security.o
 .debug_info    0x00000000       0xb1 ./ra/fsp/src/bsp/mcu/all/bsp_security.o
 .debug_abbrev  0x00000000       0x6b ./ra/fsp/src/bsp/mcu/all/bsp_security.o
 .debug_aranges
                0x00000000       0x18 ./ra/fsp/src/bsp/mcu/all/bsp_security.o
 .debug_line    0x00000000      0x15c ./ra/fsp/src/bsp/mcu/all/bsp_security.o
 .debug_str     0x00000000      0x203 ./ra/fsp/src/bsp/mcu/all/bsp_security.o
 .comment       0x00000000       0x4a ./ra/fsp/src/bsp/mcu/all/bsp_security.o
 .ARM.attributes
                0x00000000       0x3a ./ra/fsp/src/bsp/mcu/all/bsp_security.o
 .text          0x00000000        0x0 ./ra/fsp/src/bsp/cmsis/Device/RENESAS/Source/startup.o
 .data          0x00000000        0x0 ./ra/fsp/src/bsp/cmsis/Device/RENESAS/Source/startup.o
 .bss           0x00000000        0x0 ./ra/fsp/src/bsp/cmsis/Device/RENESAS/Source/startup.o
 .text          0x00000000        0x0 ./ra/fsp/src/bsp/cmsis/Device/RENESAS/Source/system.o
 .data          0x00000000        0x0 ./ra/fsp/src/bsp/cmsis/Device/RENESAS/Source/system.o
 .bss           0x00000000        0x0 ./ra/fsp/src/bsp/cmsis/Device/RENESAS/Source/system.o
 .text          0x00000000      0x254 c:/renesas/ra/e2studio_v2022-10_fsp_v4.2.0/toolchains/gcc_arm/gcc-arm-none-eabi-10.3-2021.10/bin/../lib/gcc/arm-none-eabi/10.3.1/thumb/v8-m.main+fp/hard\libgcc.a(_arm_muldf3.o)
 .data          0x00000000        0x0 c:/renesas/ra/e2studio_v2022-10_fsp_v4.2.0/toolchains/gcc_arm/gcc-arm-none-eabi-10.3-2021.10/bin/../lib/gcc/arm-none-eabi/10.3.1/thumb/v8-m.main+fp/hard\libgcc.a(_arm_muldf3.o)
 .bss           0x00000000        0x0 c:/renesas/ra/e2studio_v2022-10_fsp_v4.2.0/toolchains/gcc_arm/gcc-arm-none-eabi-10.3-2021.10/bin/../lib/gcc/arm-none-eabi/10.3.1/thumb/v8-m.main+fp/hard\libgcc.a(_arm_muldf3.o)
 .debug_frame   0x00000000       0x30 c:/renesas/ra/e2studio_v2022-10_fsp_v4.2.0/toolchains/gcc_arm/gcc-arm-none-eabi-10.3-2021.10/bin/../lib/gcc/arm-none-eabi/10.3.1/thumb/v8-m.main+fp/hard\libgcc.a(_arm_muldf3.o)
 .ARM.attributes
                0x00000000       0x22 c:/renesas/ra/e2studio_v2022-10_fsp_v4.2.0/toolchains/gcc_arm/gcc-arm-none-eabi-10.3-2021.10/bin/../lib/gcc/arm-none-eabi/10.3.1/thumb/v8-m.main+fp/hard\libgcc.a(_arm_muldf3.o)
 .data          0x00000000        0x0 c:/renesas/ra/e2studio_v2022-10_fsp_v4.2.0/toolchains/gcc_arm/gcc-arm-none-eabi-10.3-2021.10/bin/../lib/gcc/arm-none-eabi/10.3.1/thumb/v8-m.main+fp/hard\libgcc.a(_arm_addsubdf3.o)
 .bss           0x00000000        0x0 c:/renesas/ra/e2studio_v2022-10_fsp_v4.2.0/toolchains/gcc_arm/gcc-arm-none-eabi-10.3-2021.10/bin/../lib/gcc/arm-none-eabi/10.3.1/thumb/v8-m.main+fp/hard\libgcc.a(_arm_addsubdf3.o)
 .data          0x00000000        0x0 c:/renesas/ra/e2studio_v2022-10_fsp_v4.2.0/toolchains/gcc_arm/gcc-arm-none-eabi-10.3-2021.10/bin/../lib/gcc/arm-none-eabi/10.3.1/thumb/v8-m.main+fp/hard\libgcc.a(_arm_muldivdf3.o)
 .bss           0x00000000        0x0 c:/renesas/ra/e2studio_v2022-10_fsp_v4.2.0/toolchains/gcc_arm/gcc-arm-none-eabi-10.3-2021.10/bin/../lib/gcc/arm-none-eabi/10.3.1/thumb/v8-m.main+fp/hard\libgcc.a(_arm_muldivdf3.o)
 .data          0x00000000        0x0 c:/renesas/ra/e2studio_v2022-10_fsp_v4.2.0/toolchains/gcc_arm/gcc-arm-none-eabi-10.3-2021.10/bin/../lib/gcc/arm-none-eabi/10.3.1/thumb/v8-m.main+fp/hard\libgcc.a(_arm_cmpdf2.o)
 .bss           0x00000000        0x0 c:/renesas/ra/e2studio_v2022-10_fsp_v4.2.0/toolchains/gcc_arm/gcc-arm-none-eabi-10.3-2021.10/bin/../lib/gcc/arm-none-eabi/10.3.1/thumb/v8-m.main+fp/hard\libgcc.a(_arm_cmpdf2.o)
 .data          0x00000000        0x0 c:/renesas/ra/e2studio_v2022-10_fsp_v4.2.0/toolchains/gcc_arm/gcc-arm-none-eabi-10.3-2021.10/bin/../lib/gcc/arm-none-eabi/10.3.1/thumb/v8-m.main+fp/hard\libgcc.a(_arm_unorddf2.o)
 .bss           0x00000000        0x0 c:/renesas/ra/e2studio_v2022-10_fsp_v4.2.0/toolchains/gcc_arm/gcc-arm-none-eabi-10.3-2021.10/bin/../lib/gcc/arm-none-eabi/10.3.1/thumb/v8-m.main+fp/hard\libgcc.a(_arm_unorddf2.o)
 .data          0x00000000        0x0 c:/renesas/ra/e2studio_v2022-10_fsp_v4.2.0/toolchains/gcc_arm/gcc-arm-none-eabi-10.3-2021.10/bin/../lib/gcc/arm-none-eabi/10.3.1/thumb/v8-m.main+fp/hard\libgcc.a(_arm_fixdfsi.o)
 .bss           0x00000000        0x0 c:/renesas/ra/e2studio_v2022-10_fsp_v4.2.0/toolchains/gcc_arm/gcc-arm-none-eabi-10.3-2021.10/bin/../lib/gcc/arm-none-eabi/10.3.1/thumb/v8-m.main+fp/hard\libgcc.a(_arm_fixdfsi.o)
 .text          0x00000000        0x0 c:/renesas/ra/e2studio_v2022-10_fsp_v4.2.0/toolchains/gcc_arm/gcc-arm-none-eabi-10.3-2021.10/bin/../lib/gcc/arm-none-eabi/10.3.1/../../../../arm-none-eabi/lib/thumb/v8-m.main+fp/hard\libg_nano.a(lib_a-aeabi_memcpy.o)
 .data          0x00000000        0x0 c:/renesas/ra/e2studio_v2022-10_fsp_v4.2.0/toolchains/gcc_arm/gcc-arm-none-eabi-10.3-2021.10/bin/../lib/gcc/arm-none-eabi/10.3.1/../../../../arm-none-eabi/lib/thumb/v8-m.main+fp/hard\libg_nano.a(lib_a-aeabi_memcpy.o)
 .bss           0x00000000        0x0 c:/renesas/ra/e2studio_v2022-10_fsp_v4.2.0/toolchains/gcc_arm/gcc-arm-none-eabi-10.3-2021.10/bin/../lib/gcc/arm-none-eabi/10.3.1/../../../../arm-none-eabi/lib/thumb/v8-m.main+fp/hard\libg_nano.a(lib_a-aeabi_memcpy.o)
 .text          0x00000000        0x0 c:/renesas/ra/e2studio_v2022-10_fsp_v4.2.0/toolchains/gcc_arm/gcc-arm-none-eabi-10.3-2021.10/bin/../lib/gcc/arm-none-eabi/10.3.1/../../../../arm-none-eabi/lib/thumb/v8-m.main+fp/hard\libg_nano.a(lib_a-errno.o)
 .data          0x00000000        0x0 c:/renesas/ra/e2studio_v2022-10_fsp_v4.2.0/toolchains/gcc_arm/gcc-arm-none-eabi-10.3-2021.10/bin/../lib/gcc/arm-none-eabi/10.3.1/../../../../arm-none-eabi/lib/thumb/v8-m.main+fp/hard\libg_nano.a(lib_a-errno.o)
 .bss           0x00000000        0x0 c:/renesas/ra/e2studio_v2022-10_fsp_v4.2.0/toolchains/gcc_arm/gcc-arm-none-eabi-10.3-2021.10/bin/../lib/gcc/arm-none-eabi/10.3.1/../../../../arm-none-eabi/lib/thumb/v8-m.main+fp/hard\libg_nano.a(lib_a-errno.o)
 .text.__errno  0x00000000        0xc c:/renesas/ra/e2studio_v2022-10_fsp_v4.2.0/toolchains/gcc_arm/gcc-arm-none-eabi-10.3-2021.10/bin/../lib/gcc/arm-none-eabi/10.3.1/../../../../arm-none-eabi/lib/thumb/v8-m.main+fp/hard\libg_nano.a(lib_a-errno.o)
 .debug_frame   0x00000000       0x20 c:/renesas/ra/e2studio_v2022-10_fsp_v4.2.0/toolchains/gcc_arm/gcc-arm-none-eabi-10.3-2021.10/bin/../lib/gcc/arm-none-eabi/10.3.1/../../../../arm-none-eabi/lib/thumb/v8-m.main+fp/hard\libg_nano.a(lib_a-errno.o)
 .ARM.attributes
                0x00000000       0x38 c:/renesas/ra/e2studio_v2022-10_fsp_v4.2.0/toolchains/gcc_arm/gcc-arm-none-eabi-10.3-2021.10/bin/../lib/gcc/arm-none-eabi/10.3.1/../../../../arm-none-eabi/lib/thumb/v8-m.main+fp/hard\libg_nano.a(lib_a-errno.o)
 .text          0x00000000        0x0 c:/renesas/ra/e2studio_v2022-10_fsp_v4.2.0/toolchains/gcc_arm/gcc-arm-none-eabi-10.3-2021.10/bin/../lib/gcc/arm-none-eabi/10.3.1/../../../../arm-none-eabi/lib/thumb/v8-m.main+fp/hard\libg_nano.a(lib_a-exit.o)
 .data          0x00000000        0x0 c:/renesas/ra/e2studio_v2022-10_fsp_v4.2.0/toolchains/gcc_arm/gcc-arm-none-eabi-10.3-2021.10/bin/../lib/gcc/arm-none-eabi/10.3.1/../../../../arm-none-eabi/lib/thumb/v8-m.main+fp/hard\libg_nano.a(lib_a-exit.o)
 .bss           0x00000000        0x0 c:/renesas/ra/e2studio_v2022-10_fsp_v4.2.0/toolchains/gcc_arm/gcc-arm-none-eabi-10.3-2021.10/bin/../lib/gcc/arm-none-eabi/10.3.1/../../../../arm-none-eabi/lib/thumb/v8-m.main+fp/hard\libg_nano.a(lib_a-exit.o)
 .text.exit     0x00000000       0x28 c:/renesas/ra/e2studio_v2022-10_fsp_v4.2.0/toolchains/gcc_arm/gcc-arm-none-eabi-10.3-2021.10/bin/../lib/gcc/arm-none-eabi/10.3.1/../../../../arm-none-eabi/lib/thumb/v8-m.main+fp/hard\libg_nano.a(lib_a-exit.o)
 .debug_frame   0x00000000       0x28 c:/renesas/ra/e2studio_v2022-10_fsp_v4.2.0/toolchains/gcc_arm/gcc-arm-none-eabi-10.3-2021.10/bin/../lib/gcc/arm-none-eabi/10.3.1/../../../../arm-none-eabi/lib/thumb/v8-m.main+fp/hard\libg_nano.a(lib_a-exit.o)
 .ARM.attributes
                0x00000000       0x38 c:/renesas/ra/e2studio_v2022-10_fsp_v4.2.0/toolchains/gcc_arm/gcc-arm-none-eabi-10.3-2021.10/bin/../lib/gcc/arm-none-eabi/10.3.1/../../../../arm-none-eabi/lib/thumb/v8-m.main+fp/hard\libg_nano.a(lib_a-exit.o)
 .text          0x00000000        0x0 c:/renesas/ra/e2studio_v2022-10_fsp_v4.2.0/toolchains/gcc_arm/gcc-arm-none-eabi-10.3-2021.10/bin/../lib/gcc/arm-none-eabi/10.3.1/../../../../arm-none-eabi/lib/thumb/v8-m.main+fp/hard\libg_nano.a(lib_a-impure.o)
 .data          0x00000000        0x0 c:/renesas/ra/e2studio_v2022-10_fsp_v4.2.0/toolchains/gcc_arm/gcc-arm-none-eabi-10.3-2021.10/bin/../lib/gcc/arm-none-eabi/10.3.1/../../../../arm-none-eabi/lib/thumb/v8-m.main+fp/hard\libg_nano.a(lib_a-impure.o)
 .bss           0x00000000        0x0 c:/renesas/ra/e2studio_v2022-10_fsp_v4.2.0/toolchains/gcc_arm/gcc-arm-none-eabi-10.3-2021.10/bin/../lib/gcc/arm-none-eabi/10.3.1/../../../../arm-none-eabi/lib/thumb/v8-m.main+fp/hard\libg_nano.a(lib_a-impure.o)
 .data._impure_ptr
                0x00000000        0x4 c:/renesas/ra/e2studio_v2022-10_fsp_v4.2.0/toolchains/gcc_arm/gcc-arm-none-eabi-10.3-2021.10/bin/../lib/gcc/arm-none-eabi/10.3.1/../../../../arm-none-eabi/lib/thumb/v8-m.main+fp/hard\libg_nano.a(lib_a-impure.o)
 .data.impure_data
                0x00000000       0x60 c:/renesas/ra/e2studio_v2022-10_fsp_v4.2.0/toolchains/gcc_arm/gcc-arm-none-eabi-10.3-2021.10/bin/../lib/gcc/arm-none-eabi/10.3.1/../../../../arm-none-eabi/lib/thumb/v8-m.main+fp/hard\libg_nano.a(lib_a-impure.o)
 .rodata._global_impure_ptr
                0x00000000        0x4 c:/renesas/ra/e2studio_v2022-10_fsp_v4.2.0/toolchains/gcc_arm/gcc-arm-none-eabi-10.3-2021.10/bin/../lib/gcc/arm-none-eabi/10.3.1/../../../../arm-none-eabi/lib/thumb/v8-m.main+fp/hard\libg_nano.a(lib_a-impure.o)
 .ARM.attributes
                0x00000000       0x38 c:/renesas/ra/e2studio_v2022-10_fsp_v4.2.0/toolchains/gcc_arm/gcc-arm-none-eabi-10.3-2021.10/bin/../lib/gcc/arm-none-eabi/10.3.1/../../../../arm-none-eabi/lib/thumb/v8-m.main+fp/hard\libg_nano.a(lib_a-impure.o)
 .text          0x00000000        0x0 c:/renesas/ra/e2studio_v2022-10_fsp_v4.2.0/toolchains/gcc_arm/gcc-arm-none-eabi-10.3-2021.10/bin/../lib/gcc/arm-none-eabi/10.3.1/../../../../arm-none-eabi/lib/thumb/v8-m.main+fp/hard\libg_nano.a(lib_a-init.o)
 .data          0x00000000        0x0 c:/renesas/ra/e2studio_v2022-10_fsp_v4.2.0/toolchains/gcc_arm/gcc-arm-none-eabi-10.3-2021.10/bin/../lib/gcc/arm-none-eabi/10.3.1/../../../../arm-none-eabi/lib/thumb/v8-m.main+fp/hard\libg_nano.a(lib_a-init.o)
 .bss           0x00000000        0x0 c:/renesas/ra/e2studio_v2022-10_fsp_v4.2.0/toolchains/gcc_arm/gcc-arm-none-eabi-10.3-2021.10/bin/../lib/gcc/arm-none-eabi/10.3.1/../../../../arm-none-eabi/lib/thumb/v8-m.main+fp/hard\libg_nano.a(lib_a-init.o)
 .text.__libc_init_array
                0x00000000       0x48 c:/renesas/ra/e2studio_v2022-10_fsp_v4.2.0/toolchains/gcc_arm/gcc-arm-none-eabi-10.3-2021.10/bin/../lib/gcc/arm-none-eabi/10.3.1/../../../../arm-none-eabi/lib/thumb/v8-m.main+fp/hard\libg_nano.a(lib_a-init.o)
 .debug_frame   0x00000000       0x2c c:/renesas/ra/e2studio_v2022-10_fsp_v4.2.0/toolchains/gcc_arm/gcc-arm-none-eabi-10.3-2021.10/bin/../lib/gcc/arm-none-eabi/10.3.1/../../../../arm-none-eabi/lib/thumb/v8-m.main+fp/hard\libg_nano.a(lib_a-init.o)
 .ARM.attributes
                0x00000000       0x38 c:/renesas/ra/e2studio_v2022-10_fsp_v4.2.0/toolchains/gcc_arm/gcc-arm-none-eabi-10.3-2021.10/bin/../lib/gcc/arm-none-eabi/10.3.1/../../../../arm-none-eabi/lib/thumb/v8-m.main+fp/hard\libg_nano.a(lib_a-init.o)
 .text          0x00000000        0x0 c:/renesas/ra/e2studio_v2022-10_fsp_v4.2.0/toolchains/gcc_arm/gcc-arm-none-eabi-10.3-2021.10/bin/../lib/gcc/arm-none-eabi/10.3.1/../../../../arm-none-eabi/lib/thumb/v8-m.main+fp/hard\libg_nano.a(lib_a-memcpy-stub.o)
 .data          0x00000000        0x0 c:/renesas/ra/e2studio_v2022-10_fsp_v4.2.0/toolchains/gcc_arm/gcc-arm-none-eabi-10.3-2021.10/bin/../lib/gcc/arm-none-eabi/10.3.1/../../../../arm-none-eabi/lib/thumb/v8-m.main+fp/hard\libg_nano.a(lib_a-memcpy-stub.o)
 .bss           0x00000000        0x0 c:/renesas/ra/e2studio_v2022-10_fsp_v4.2.0/toolchains/gcc_arm/gcc-arm-none-eabi-10.3-2021.10/bin/../lib/gcc/arm-none-eabi/10.3.1/../../../../arm-none-eabi/lib/thumb/v8-m.main+fp/hard\libg_nano.a(lib_a-memcpy-stub.o)
 .text          0x00000000        0x0 c:/renesas/ra/e2studio_v2022-10_fsp_v4.2.0/toolchains/gcc_arm/gcc-arm-none-eabi-10.3-2021.10/bin/../lib/gcc/arm-none-eabi/10.3.1/../../../../arm-none-eabi/lib/thumb/v8-m.main+fp/hard\libg_nano.a(lib_a-memset.o)
 .data          0x00000000        0x0 c:/renesas/ra/e2studio_v2022-10_fsp_v4.2.0/toolchains/gcc_arm/gcc-arm-none-eabi-10.3-2021.10/bin/../lib/gcc/arm-none-eabi/10.3.1/../../../../arm-none-eabi/lib/thumb/v8-m.main+fp/hard\libg_nano.a(lib_a-memset.o)
 .bss           0x00000000        0x0 c:/renesas/ra/e2studio_v2022-10_fsp_v4.2.0/toolchains/gcc_arm/gcc-arm-none-eabi-10.3-2021.10/bin/../lib/gcc/arm-none-eabi/10.3.1/../../../../arm-none-eabi/lib/thumb/v8-m.main+fp/hard\libg_nano.a(lib_a-memset.o)
 .data          0x00000000        0x0 c:/renesas/ra/e2studio_v2022-10_fsp_v4.2.0/toolchains/gcc_arm/gcc-arm-none-eabi-10.3-2021.10/bin/../lib/gcc/arm-none-eabi/10.3.1/../../../../arm-none-eabi/lib/thumb/v8-m.main+fp/hard\libg_nano.a(lib_a-strlen.o)
 .bss           0x00000000        0x0 c:/renesas/ra/e2studio_v2022-10_fsp_v4.2.0/toolchains/gcc_arm/gcc-arm-none-eabi-10.3-2021.10/bin/../lib/gcc/arm-none-eabi/10.3.1/../../../../arm-none-eabi/lib/thumb/v8-m.main+fp/hard\libg_nano.a(lib_a-strlen.o)
 .text          0x00000000        0x0 c:/renesas/ra/e2studio_v2022-10_fsp_v4.2.0/toolchains/gcc_arm/gcc-arm-none-eabi-10.3-2021.10/bin/../lib/gcc/arm-none-eabi/10.3.1/../../../../arm-none-eabi/lib/thumb/v8-m.main+fp/hard\librdimon_nano.a(rdimon-syscalls.o)
 .data          0x00000000        0x0 c:/renesas/ra/e2studio_v2022-10_fsp_v4.2.0/toolchains/gcc_arm/gcc-arm-none-eabi-10.3-2021.10/bin/../lib/gcc/arm-none-eabi/10.3.1/../../../../arm-none-eabi/lib/thumb/v8-m.main+fp/hard\librdimon_nano.a(rdimon-syscalls.o)
 .bss           0x00000000        0x0 c:/renesas/ra/e2studio_v2022-10_fsp_v4.2.0/toolchains/gcc_arm/gcc-arm-none-eabi-10.3-2021.10/bin/../lib/gcc/arm-none-eabi/10.3.1/../../../../arm-none-eabi/lib/thumb/v8-m.main+fp/hard\librdimon_nano.a(rdimon-syscalls.o)
 .text.findslot
                0x00000000       0x34 c:/renesas/ra/e2studio_v2022-10_fsp_v4.2.0/toolchains/gcc_arm/gcc-arm-none-eabi-10.3-2021.10/bin/../lib/gcc/arm-none-eabi/10.3.1/../../../../arm-none-eabi/lib/thumb/v8-m.main+fp/hard\librdimon_nano.a(rdimon-syscalls.o)
 .text.error    0x00000000       0x1c c:/renesas/ra/e2studio_v2022-10_fsp_v4.2.0/toolchains/gcc_arm/gcc-arm-none-eabi-10.3-2021.10/bin/../lib/gcc/arm-none-eabi/10.3.1/../../../../arm-none-eabi/lib/thumb/v8-m.main+fp/hard\librdimon_nano.a(rdimon-syscalls.o)
 .text.checkerror
                0x00000000        0xa c:/renesas/ra/e2studio_v2022-10_fsp_v4.2.0/toolchains/gcc_arm/gcc-arm-none-eabi-10.3-2021.10/bin/../lib/gcc/arm-none-eabi/10.3.1/../../../../arm-none-eabi/lib/thumb/v8-m.main+fp/hard\librdimon_nano.a(rdimon-syscalls.o)
 .text._swiread
                0x00000000       0x20 c:/renesas/ra/e2studio_v2022-10_fsp_v4.2.0/toolchains/gcc_arm/gcc-arm-none-eabi-10.3-2021.10/bin/../lib/gcc/arm-none-eabi/10.3.1/../../../../arm-none-eabi/lib/thumb/v8-m.main+fp/hard\librdimon_nano.a(rdimon-syscalls.o)
 .text._read    0x00000000       0x38 c:/renesas/ra/e2studio_v2022-10_fsp_v4.2.0/toolchains/gcc_arm/gcc-arm-none-eabi-10.3-2021.10/bin/../lib/gcc/arm-none-eabi/10.3.1/../../../../arm-none-eabi/lib/thumb/v8-m.main+fp/hard\librdimon_nano.a(rdimon-syscalls.o)
 .text._swilseek
                0x00000000       0x78 c:/renesas/ra/e2studio_v2022-10_fsp_v4.2.0/toolchains/gcc_arm/gcc-arm-none-eabi-10.3-2021.10/bin/../lib/gcc/arm-none-eabi/10.3.1/../../../../arm-none-eabi/lib/thumb/v8-m.main+fp/hard\librdimon_nano.a(rdimon-syscalls.o)
 .text._lseek   0x00000000        0x4 c:/renesas/ra/e2studio_v2022-10_fsp_v4.2.0/toolchains/gcc_arm/gcc-arm-none-eabi-10.3-2021.10/bin/../lib/gcc/arm-none-eabi/10.3.1/../../../../arm-none-eabi/lib/thumb/v8-m.main+fp/hard\librdimon_nano.a(rdimon-syscalls.o)
 .text._swiwrite
                0x00000000       0x20 c:/renesas/ra/e2studio_v2022-10_fsp_v4.2.0/toolchains/gcc_arm/gcc-arm-none-eabi-10.3-2021.10/bin/../lib/gcc/arm-none-eabi/10.3.1/../../../../arm-none-eabi/lib/thumb/v8-m.main+fp/hard\librdimon_nano.a(rdimon-syscalls.o)
 .text._write   0x00000000       0x48 c:/renesas/ra/e2studio_v2022-10_fsp_v4.2.0/toolchains/gcc_arm/gcc-arm-none-eabi-10.3-2021.10/bin/../lib/gcc/arm-none-eabi/10.3.1/../../../../arm-none-eabi/lib/thumb/v8-m.main+fp/hard\librdimon_nano.a(rdimon-syscalls.o)
 .text._swiclose
                0x00000000       0x1a c:/renesas/ra/e2studio_v2022-10_fsp_v4.2.0/toolchains/gcc_arm/gcc-arm-none-eabi-10.3-2021.10/bin/../lib/gcc/arm-none-eabi/10.3.1/../../../../arm-none-eabi/lib/thumb/v8-m.main+fp/hard\librdimon_nano.a(rdimon-syscalls.o)
 .text._close   0x00000000       0x4c c:/renesas/ra/e2studio_v2022-10_fsp_v4.2.0/toolchains/gcc_arm/gcc-arm-none-eabi-10.3-2021.10/bin/../lib/gcc/arm-none-eabi/10.3.1/../../../../arm-none-eabi/lib/thumb/v8-m.main+fp/hard\librdimon_nano.a(rdimon-syscalls.o)
 .text._getpid  0x00000000        0x4 c:/renesas/ra/e2studio_v2022-10_fsp_v4.2.0/toolchains/gcc_arm/gcc-arm-none-eabi-10.3-2021.10/bin/../lib/gcc/arm-none-eabi/10.3.1/../../../../arm-none-eabi/lib/thumb/v8-m.main+fp/hard\librdimon_nano.a(rdimon-syscalls.o)
 .text._sbrk    0x00000000       0x48 c:/renesas/ra/e2studio_v2022-10_fsp_v4.2.0/toolchains/gcc_arm/gcc-arm-none-eabi-10.3-2021.10/bin/../lib/gcc/arm-none-eabi/10.3.1/../../../../arm-none-eabi/lib/thumb/v8-m.main+fp/hard\librdimon_nano.a(rdimon-syscalls.o)
 .text._swistat
                0x00000000       0x42 c:/renesas/ra/e2studio_v2022-10_fsp_v4.2.0/toolchains/gcc_arm/gcc-arm-none-eabi-10.3-2021.10/bin/../lib/gcc/arm-none-eabi/10.3.1/../../../../arm-none-eabi/lib/thumb/v8-m.main+fp/hard\librdimon_nano.a(rdimon-syscalls.o)
 .text._fstat   0x00000000       0x1c c:/renesas/ra/e2studio_v2022-10_fsp_v4.2.0/toolchains/gcc_arm/gcc-arm-none-eabi-10.3-2021.10/bin/../lib/gcc/arm-none-eabi/10.3.1/../../../../arm-none-eabi/lib/thumb/v8-m.main+fp/hard\librdimon_nano.a(rdimon-syscalls.o)
 .text._stat    0x00000000       0x3a c:/renesas/ra/e2studio_v2022-10_fsp_v4.2.0/toolchains/gcc_arm/gcc-arm-none-eabi-10.3-2021.10/bin/../lib/gcc/arm-none-eabi/10.3.1/../../../../arm-none-eabi/lib/thumb/v8-m.main+fp/hard\librdimon_nano.a(rdimon-syscalls.o)
 .text._swiopen
                0x00000000       0xb4 c:/renesas/ra/e2studio_v2022-10_fsp_v4.2.0/toolchains/gcc_arm/gcc-arm-none-eabi-10.3-2021.10/bin/../lib/gcc/arm-none-eabi/10.3.1/../../../../arm-none-eabi/lib/thumb/v8-m.main+fp/hard\librdimon_nano.a(rdimon-syscalls.o)
 .text._open    0x00000000       0x12 c:/renesas/ra/e2studio_v2022-10_fsp_v4.2.0/toolchains/gcc_arm/gcc-arm-none-eabi-10.3-2021.10/bin/../lib/gcc/arm-none-eabi/10.3.1/../../../../arm-none-eabi/lib/thumb/v8-m.main+fp/hard\librdimon_nano.a(rdimon-syscalls.o)
 .rodata._get_semihosting_exts.str1.1
                0x00000000       0x16 c:/renesas/ra/e2studio_v2022-10_fsp_v4.2.0/toolchains/gcc_arm/gcc-arm-none-eabi-10.3-2021.10/bin/../lib/gcc/arm-none-eabi/10.3.1/../../../../arm-none-eabi/lib/thumb/v8-m.main+fp/hard\librdimon_nano.a(rdimon-syscalls.o)
 .text._get_semihosting_exts
                0x00000000       0xb8 c:/renesas/ra/e2studio_v2022-10_fsp_v4.2.0/toolchains/gcc_arm/gcc-arm-none-eabi-10.3-2021.10/bin/../lib/gcc/arm-none-eabi/10.3.1/../../../../arm-none-eabi/lib/thumb/v8-m.main+fp/hard\librdimon_nano.a(rdimon-syscalls.o)
 .text.initialise_semihosting_exts
                0x00000000       0x34 c:/renesas/ra/e2studio_v2022-10_fsp_v4.2.0/toolchains/gcc_arm/gcc-arm-none-eabi-10.3-2021.10/bin/../lib/gcc/arm-none-eabi/10.3.1/../../../../arm-none-eabi/lib/thumb/v8-m.main+fp/hard\librdimon_nano.a(rdimon-syscalls.o)
 .text._has_ext_exit_extended
                0x00000000       0x18 c:/renesas/ra/e2studio_v2022-10_fsp_v4.2.0/toolchains/gcc_arm/gcc-arm-none-eabi-10.3-2021.10/bin/../lib/gcc/arm-none-eabi/10.3.1/../../../../arm-none-eabi/lib/thumb/v8-m.main+fp/hard\librdimon_nano.a(rdimon-syscalls.o)
 .text._has_ext_stdout_stderr
                0x00000000       0x18 c:/renesas/ra/e2studio_v2022-10_fsp_v4.2.0/toolchains/gcc_arm/gcc-arm-none-eabi-10.3-2021.10/bin/../lib/gcc/arm-none-eabi/10.3.1/../../../../arm-none-eabi/lib/thumb/v8-m.main+fp/hard\librdimon_nano.a(rdimon-syscalls.o)
 .rodata.initialise_monitor_handles.str1.1
                0x00000000        0x4 c:/renesas/ra/e2studio_v2022-10_fsp_v4.2.0/toolchains/gcc_arm/gcc-arm-none-eabi-10.3-2021.10/bin/../lib/gcc/arm-none-eabi/10.3.1/../../../../arm-none-eabi/lib/thumb/v8-m.main+fp/hard\librdimon_nano.a(rdimon-syscalls.o)
 .text.initialise_monitor_handles
                0x00000000       0xc0 c:/renesas/ra/e2studio_v2022-10_fsp_v4.2.0/toolchains/gcc_arm/gcc-arm-none-eabi-10.3-2021.10/bin/../lib/gcc/arm-none-eabi/10.3.1/../../../../arm-none-eabi/lib/thumb/v8-m.main+fp/hard\librdimon_nano.a(rdimon-syscalls.o)
 .text._link    0x00000000       0x10 c:/renesas/ra/e2studio_v2022-10_fsp_v4.2.0/toolchains/gcc_arm/gcc-arm-none-eabi-10.3-2021.10/bin/../lib/gcc/arm-none-eabi/10.3.1/../../../../arm-none-eabi/lib/thumb/v8-m.main+fp/hard\librdimon_nano.a(rdimon-syscalls.o)
 .text._unlink  0x00000000       0x28 c:/renesas/ra/e2studio_v2022-10_fsp_v4.2.0/toolchains/gcc_arm/gcc-arm-none-eabi-10.3-2021.10/bin/../lib/gcc/arm-none-eabi/10.3.1/../../../../arm-none-eabi/lib/thumb/v8-m.main+fp/hard\librdimon_nano.a(rdimon-syscalls.o)
 .text._gettimeofday
                0x00000000       0x28 c:/renesas/ra/e2studio_v2022-10_fsp_v4.2.0/toolchains/gcc_arm/gcc-arm-none-eabi-10.3-2021.10/bin/../lib/gcc/arm-none-eabi/10.3.1/../../../../arm-none-eabi/lib/thumb/v8-m.main+fp/hard\librdimon_nano.a(rdimon-syscalls.o)
 .text._clock   0x00000000       0x12 c:/renesas/ra/e2studio_v2022-10_fsp_v4.2.0/toolchains/gcc_arm/gcc-arm-none-eabi-10.3-2021.10/bin/../lib/gcc/arm-none-eabi/10.3.1/../../../../arm-none-eabi/lib/thumb/v8-m.main+fp/hard\librdimon_nano.a(rdimon-syscalls.o)
 .text._times   0x00000000       0x16 c:/renesas/ra/e2studio_v2022-10_fsp_v4.2.0/toolchains/gcc_arm/gcc-arm-none-eabi-10.3-2021.10/bin/../lib/gcc/arm-none-eabi/10.3.1/../../../../arm-none-eabi/lib/thumb/v8-m.main+fp/hard\librdimon_nano.a(rdimon-syscalls.o)
 .text._isatty  0x00000000       0x38 c:/renesas/ra/e2studio_v2022-10_fsp_v4.2.0/toolchains/gcc_arm/gcc-arm-none-eabi-10.3-2021.10/bin/../lib/gcc/arm-none-eabi/10.3.1/../../../../arm-none-eabi/lib/thumb/v8-m.main+fp/hard\librdimon_nano.a(rdimon-syscalls.o)
 .text._system  0x00000000       0x3c c:/renesas/ra/e2studio_v2022-10_fsp_v4.2.0/toolchains/gcc_arm/gcc-arm-none-eabi-10.3-2021.10/bin/../lib/gcc/arm-none-eabi/10.3.1/../../../../arm-none-eabi/lib/thumb/v8-m.main+fp/hard\librdimon_nano.a(rdimon-syscalls.o)
 .text._rename  0x00000000       0x36 c:/renesas/ra/e2studio_v2022-10_fsp_v4.2.0/toolchains/gcc_arm/gcc-arm-none-eabi-10.3-2021.10/bin/../lib/gcc/arm-none-eabi/10.3.1/../../../../arm-none-eabi/lib/thumb/v8-m.main+fp/hard\librdimon_nano.a(rdimon-syscalls.o)
 .bss.heap_end.0
                0x00000000        0x4 c:/renesas/ra/e2studio_v2022-10_fsp_v4.2.0/toolchains/gcc_arm/gcc-arm-none-eabi-10.3-2021.10/bin/../lib/gcc/arm-none-eabi/10.3.1/../../../../arm-none-eabi/lib/thumb/v8-m.main+fp/hard\librdimon_nano.a(rdimon-syscalls.o)
 .bss.monitor_stderr
                0x00000000        0x4 c:/renesas/ra/e2studio_v2022-10_fsp_v4.2.0/toolchains/gcc_arm/gcc-arm-none-eabi-10.3-2021.10/bin/../lib/gcc/arm-none-eabi/10.3.1/../../../../arm-none-eabi/lib/thumb/v8-m.main+fp/hard\librdimon_nano.a(rdimon-syscalls.o)
 .bss.monitor_stdin
                0x00000000        0x4 c:/renesas/ra/e2studio_v2022-10_fsp_v4.2.0/toolchains/gcc_arm/gcc-arm-none-eabi-10.3-2021.10/bin/../lib/gcc/arm-none-eabi/10.3.1/../../../../arm-none-eabi/lib/thumb/v8-m.main+fp/hard\librdimon_nano.a(rdimon-syscalls.o)
 .bss.monitor_stdout
                0x00000000        0x4 c:/renesas/ra/e2studio_v2022-10_fsp_v4.2.0/toolchains/gcc_arm/gcc-arm-none-eabi-10.3-2021.10/bin/../lib/gcc/arm-none-eabi/10.3.1/../../../../arm-none-eabi/lib/thumb/v8-m.main+fp/hard\librdimon_nano.a(rdimon-syscalls.o)
 .bss.openfiles
                0x00000000       0xa0 c:/renesas/ra/e2studio_v2022-10_fsp_v4.2.0/toolchains/gcc_arm/gcc-arm-none-eabi-10.3-2021.10/bin/../lib/gcc/arm-none-eabi/10.3.1/../../../../arm-none-eabi/lib/thumb/v8-m.main+fp/hard\librdimon_nano.a(rdimon-syscalls.o)
 .data.__heap_limit
                0x00000000        0x4 c:/renesas/ra/e2studio_v2022-10_fsp_v4.2.0/toolchains/gcc_arm/gcc-arm-none-eabi-10.3-2021.10/bin/../lib/gcc/arm-none-eabi/10.3.1/../../../../arm-none-eabi/lib/thumb/v8-m.main+fp/hard\librdimon_nano.a(rdimon-syscalls.o)
 .data.supports_ext_exit_extended
                0x00000000        0x4 c:/renesas/ra/e2studio_v2022-10_fsp_v4.2.0/toolchains/gcc_arm/gcc-arm-none-eabi-10.3-2021.10/bin/../lib/gcc/arm-none-eabi/10.3.1/../../../../arm-none-eabi/lib/thumb/v8-m.main+fp/hard\librdimon_nano.a(rdimon-syscalls.o)
 .data.supports_ext_stdout_stderr
                0x00000000        0x4 c:/renesas/ra/e2studio_v2022-10_fsp_v4.2.0/toolchains/gcc_arm/gcc-arm-none-eabi-10.3-2021.10/bin/../lib/gcc/arm-none-eabi/10.3.1/../../../../arm-none-eabi/lib/thumb/v8-m.main+fp/hard\librdimon_nano.a(rdimon-syscalls.o)
 .debug_frame   0x00000000      0x3a0 c:/renesas/ra/e2studio_v2022-10_fsp_v4.2.0/toolchains/gcc_arm/gcc-arm-none-eabi-10.3-2021.10/bin/../lib/gcc/arm-none-eabi/10.3.1/../../../../arm-none-eabi/lib/thumb/v8-m.main+fp/hard\librdimon_nano.a(rdimon-syscalls.o)
 .ARM.attributes
                0x00000000       0x38 c:/renesas/ra/e2studio_v2022-10_fsp_v4.2.0/toolchains/gcc_arm/gcc-arm-none-eabi-10.3-2021.10/bin/../lib/gcc/arm-none-eabi/10.3.1/../../../../arm-none-eabi/lib/thumb/v8-m.main+fp/hard\librdimon_nano.a(rdimon-syscalls.o)
 .text          0x00000000        0x0 c:/renesas/ra/e2studio_v2022-10_fsp_v4.2.0/toolchains/gcc_arm/gcc-arm-none-eabi-10.3-2021.10/bin/../lib/gcc/arm-none-eabi/10.3.1/../../../../arm-none-eabi/lib/thumb/v8-m.main+fp/hard\librdimon_nano.a(rdimon-_exit.o)
 .data          0x00000000        0x0 c:/renesas/ra/e2studio_v2022-10_fsp_v4.2.0/toolchains/gcc_arm/gcc-arm-none-eabi-10.3-2021.10/bin/../lib/gcc/arm-none-eabi/10.3.1/../../../../arm-none-eabi/lib/thumb/v8-m.main+fp/hard\librdimon_nano.a(rdimon-_exit.o)
 .bss           0x00000000        0x0 c:/renesas/ra/e2studio_v2022-10_fsp_v4.2.0/toolchains/gcc_arm/gcc-arm-none-eabi-10.3-2021.10/bin/../lib/gcc/arm-none-eabi/10.3.1/../../../../arm-none-eabi/lib/thumb/v8-m.main+fp/hard\librdimon_nano.a(rdimon-_exit.o)
 .text._exit    0x00000000       0x14 c:/renesas/ra/e2studio_v2022-10_fsp_v4.2.0/toolchains/gcc_arm/gcc-arm-none-eabi-10.3-2021.10/bin/../lib/gcc/arm-none-eabi/10.3.1/../../../../arm-none-eabi/lib/thumb/v8-m.main+fp/hard\librdimon_nano.a(rdimon-_exit.o)
 .debug_frame   0x00000000       0x28 c:/renesas/ra/e2studio_v2022-10_fsp_v4.2.0/toolchains/gcc_arm/gcc-arm-none-eabi-10.3-2021.10/bin/../lib/gcc/arm-none-eabi/10.3.1/../../../../arm-none-eabi/lib/thumb/v8-m.main+fp/hard\librdimon_nano.a(rdimon-_exit.o)
 .ARM.attributes
                0x00000000       0x38 c:/renesas/ra/e2studio_v2022-10_fsp_v4.2.0/toolchains/gcc_arm/gcc-arm-none-eabi-10.3-2021.10/bin/../lib/gcc/arm-none-eabi/10.3.1/../../../../arm-none-eabi/lib/thumb/v8-m.main+fp/hard\librdimon_nano.a(rdimon-_exit.o)
 .text          0x00000000        0x0 c:/renesas/ra/e2studio_v2022-10_fsp_v4.2.0/toolchains/gcc_arm/gcc-arm-none-eabi-10.3-2021.10/bin/../lib/gcc/arm-none-eabi/10.3.1/../../../../arm-none-eabi/lib/thumb/v8-m.main+fp/hard\librdimon_nano.a(rdimon-_kill.o)
 .data          0x00000000        0x0 c:/renesas/ra/e2studio_v2022-10_fsp_v4.2.0/toolchains/gcc_arm/gcc-arm-none-eabi-10.3-2021.10/bin/../lib/gcc/arm-none-eabi/10.3.1/../../../../arm-none-eabi/lib/thumb/v8-m.main+fp/hard\librdimon_nano.a(rdimon-_kill.o)
 .bss           0x00000000        0x0 c:/renesas/ra/e2studio_v2022-10_fsp_v4.2.0/toolchains/gcc_arm/gcc-arm-none-eabi-10.3-2021.10/bin/../lib/gcc/arm-none-eabi/10.3.1/../../../../arm-none-eabi/lib/thumb/v8-m.main+fp/hard\librdimon_nano.a(rdimon-_kill.o)
 .text._kill_shared
                0x00000000       0x26 c:/renesas/ra/e2studio_v2022-10_fsp_v4.2.0/toolchains/gcc_arm/gcc-arm-none-eabi-10.3-2021.10/bin/../lib/gcc/arm-none-eabi/10.3.1/../../../../arm-none-eabi/lib/thumb/v8-m.main+fp/hard\librdimon_nano.a(rdimon-_kill.o)
 .text._kill    0x00000000       0x18 c:/renesas/ra/e2studio_v2022-10_fsp_v4.2.0/toolchains/gcc_arm/gcc-arm-none-eabi-10.3-2021.10/bin/../lib/gcc/arm-none-eabi/10.3.1/../../../../arm-none-eabi/lib/thumb/v8-m.main+fp/hard\librdimon_nano.a(rdimon-_kill.o)
 .debug_frame   0x00000000       0x40 c:/renesas/ra/e2studio_v2022-10_fsp_v4.2.0/toolchains/gcc_arm/gcc-arm-none-eabi-10.3-2021.10/bin/../lib/gcc/arm-none-eabi/10.3.1/../../../../arm-none-eabi/lib/thumb/v8-m.main+fp/hard\librdimon_nano.a(rdimon-_kill.o)
 .ARM.attributes
                0x00000000       0x38 c:/renesas/ra/e2studio_v2022-10_fsp_v4.2.0/toolchains/gcc_arm/gcc-arm-none-eabi-10.3-2021.10/bin/../lib/gcc/arm-none-eabi/10.3.1/../../../../arm-none-eabi/lib/thumb/v8-m.main+fp/hard\librdimon_nano.a(rdimon-_kill.o)
 .text          0x00000000        0x0 c:/renesas/ra/e2studio_v2022-10_fsp_v4.2.0/toolchains/gcc_arm/gcc-arm-none-eabi-10.3-2021.10/bin/../lib/gcc/arm-none-eabi/10.3.1/../../../../arm-none-eabi/lib/thumb/v8-m.main+fp/hard\libc_nano.a(lib_a-findfp.o)
 .data          0x00000000        0x0 c:/renesas/ra/e2studio_v2022-10_fsp_v4.2.0/toolchains/gcc_arm/gcc-arm-none-eabi-10.3-2021.10/bin/../lib/gcc/arm-none-eabi/10.3.1/../../../../arm-none-eabi/lib/thumb/v8-m.main+fp/hard\libc_nano.a(lib_a-findfp.o)
 .bss           0x00000000        0x0 c:/renesas/ra/e2studio_v2022-10_fsp_v4.2.0/toolchains/gcc_arm/gcc-arm-none-eabi-10.3-2021.10/bin/../lib/gcc/arm-none-eabi/10.3.1/../../../../arm-none-eabi/lib/thumb/v8-m.main+fp/hard\libc_nano.a(lib_a-findfp.o)
 .text.std      0x00000000       0x48 c:/renesas/ra/e2studio_v2022-10_fsp_v4.2.0/toolchains/gcc_arm/gcc-arm-none-eabi-10.3-2021.10/bin/../lib/gcc/arm-none-eabi/10.3.1/../../../../arm-none-eabi/lib/thumb/v8-m.main+fp/hard\libc_nano.a(lib_a-findfp.o)
 .text._cleanup_r
                0x00000000        0xc c:/renesas/ra/e2studio_v2022-10_fsp_v4.2.0/toolchains/gcc_arm/gcc-arm-none-eabi-10.3-2021.10/bin/../lib/gcc/arm-none-eabi/10.3.1/../../../../arm-none-eabi/lib/thumb/v8-m.main+fp/hard\libc_nano.a(lib_a-findfp.o)
 .text.__fp_lock
                0x00000000       0x18 c:/renesas/ra/e2studio_v2022-10_fsp_v4.2.0/toolchains/gcc_arm/gcc-arm-none-eabi-10.3-2021.10/bin/../lib/gcc/arm-none-eabi/10.3.1/../../../../arm-none-eabi/lib/thumb/v8-m.main+fp/hard\libc_nano.a(lib_a-findfp.o)
 .text.__fp_unlock
                0x00000000       0x18 c:/renesas/ra/e2studio_v2022-10_fsp_v4.2.0/toolchains/gcc_arm/gcc-arm-none-eabi-10.3-2021.10/bin/../lib/gcc/arm-none-eabi/10.3.1/../../../../arm-none-eabi/lib/thumb/v8-m.main+fp/hard\libc_nano.a(lib_a-findfp.o)
 .text.__sfmoreglue
                0x00000000       0x2c c:/renesas/ra/e2studio_v2022-10_fsp_v4.2.0/toolchains/gcc_arm/gcc-arm-none-eabi-10.3-2021.10/bin/../lib/gcc/arm-none-eabi/10.3.1/../../../../arm-none-eabi/lib/thumb/v8-m.main+fp/hard\libc_nano.a(lib_a-findfp.o)
 .text._cleanup
                0x00000000        0xc c:/renesas/ra/e2studio_v2022-10_fsp_v4.2.0/toolchains/gcc_arm/gcc-arm-none-eabi-10.3-2021.10/bin/../lib/gcc/arm-none-eabi/10.3.1/../../../../arm-none-eabi/lib/thumb/v8-m.main+fp/hard\libc_nano.a(lib_a-findfp.o)
 .text.__sfp_lock_acquire
                0x00000000        0xc c:/renesas/ra/e2studio_v2022-10_fsp_v4.2.0/toolchains/gcc_arm/gcc-arm-none-eabi-10.3-2021.10/bin/../lib/gcc/arm-none-eabi/10.3.1/../../../../arm-none-eabi/lib/thumb/v8-m.main+fp/hard\libc_nano.a(lib_a-findfp.o)
 .text.__sfp_lock_release
                0x00000000        0xc c:/renesas/ra/e2studio_v2022-10_fsp_v4.2.0/toolchains/gcc_arm/gcc-arm-none-eabi-10.3-2021.10/bin/../lib/gcc/arm-none-eabi/10.3.1/../../../../arm-none-eabi/lib/thumb/v8-m.main+fp/hard\libc_nano.a(lib_a-findfp.o)
 .text.__sinit_lock_acquire
                0x00000000        0xc c:/renesas/ra/e2studio_v2022-10_fsp_v4.2.0/toolchains/gcc_arm/gcc-arm-none-eabi-10.3-2021.10/bin/../lib/gcc/arm-none-eabi/10.3.1/../../../../arm-none-eabi/lib/thumb/v8-m.main+fp/hard\libc_nano.a(lib_a-findfp.o)
 .text.__sinit_lock_release
                0x00000000        0xc c:/renesas/ra/e2studio_v2022-10_fsp_v4.2.0/toolchains/gcc_arm/gcc-arm-none-eabi-10.3-2021.10/bin/../lib/gcc/arm-none-eabi/10.3.1/../../../../arm-none-eabi/lib/thumb/v8-m.main+fp/hard\libc_nano.a(lib_a-findfp.o)
 .text.__sinit  0x00000000       0x70 c:/renesas/ra/e2studio_v2022-10_fsp_v4.2.0/toolchains/gcc_arm/gcc-arm-none-eabi-10.3-2021.10/bin/../lib/gcc/arm-none-eabi/10.3.1/../../../../arm-none-eabi/lib/thumb/v8-m.main+fp/hard\libc_nano.a(lib_a-findfp.o)
 .text.__sfp    0x00000000       0x8c c:/renesas/ra/e2studio_v2022-10_fsp_v4.2.0/toolchains/gcc_arm/gcc-arm-none-eabi-10.3-2021.10/bin/../lib/gcc/arm-none-eabi/10.3.1/../../../../arm-none-eabi/lib/thumb/v8-m.main+fp/hard\libc_nano.a(lib_a-findfp.o)
 .text.__fp_lock_all
                0x00000000       0x1c c:/renesas/ra/e2studio_v2022-10_fsp_v4.2.0/toolchains/gcc_arm/gcc-arm-none-eabi-10.3-2021.10/bin/../lib/gcc/arm-none-eabi/10.3.1/../../../../arm-none-eabi/lib/thumb/v8-m.main+fp/hard\libc_nano.a(lib_a-findfp.o)
 .text.__fp_unlock_all
                0x00000000       0x1c c:/renesas/ra/e2studio_v2022-10_fsp_v4.2.0/toolchains/gcc_arm/gcc-arm-none-eabi-10.3-2021.10/bin/../lib/gcc/arm-none-eabi/10.3.1/../../../../arm-none-eabi/lib/thumb/v8-m.main+fp/hard\libc_nano.a(lib_a-findfp.o)
 .rodata.__sf_fake_stderr
                0x00000000       0x20 c:/renesas/ra/e2studio_v2022-10_fsp_v4.2.0/toolchains/gcc_arm/gcc-arm-none-eabi-10.3-2021.10/bin/../lib/gcc/arm-none-eabi/10.3.1/../../../../arm-none-eabi/lib/thumb/v8-m.main+fp/hard\libc_nano.a(lib_a-findfp.o)
 .rodata.__sf_fake_stdin
                0x00000000       0x20 c:/renesas/ra/e2studio_v2022-10_fsp_v4.2.0/toolchains/gcc_arm/gcc-arm-none-eabi-10.3-2021.10/bin/../lib/gcc/arm-none-eabi/10.3.1/../../../../arm-none-eabi/lib/thumb/v8-m.main+fp/hard\libc_nano.a(lib_a-findfp.o)
 .rodata.__sf_fake_stdout
                0x00000000       0x20 c:/renesas/ra/e2studio_v2022-10_fsp_v4.2.0/toolchains/gcc_arm/gcc-arm-none-eabi-10.3-2021.10/bin/../lib/gcc/arm-none-eabi/10.3.1/../../../../arm-none-eabi/lib/thumb/v8-m.main+fp/hard\libc_nano.a(lib_a-findfp.o)
 .debug_frame   0x00000000      0x14c c:/renesas/ra/e2studio_v2022-10_fsp_v4.2.0/toolchains/gcc_arm/gcc-arm-none-eabi-10.3-2021.10/bin/../lib/gcc/arm-none-eabi/10.3.1/../../../../arm-none-eabi/lib/thumb/v8-m.main+fp/hard\libc_nano.a(lib_a-findfp.o)
 .ARM.attributes
                0x00000000       0x38 c:/renesas/ra/e2studio_v2022-10_fsp_v4.2.0/toolchains/gcc_arm/gcc-arm-none-eabi-10.3-2021.10/bin/../lib/gcc/arm-none-eabi/10.3.1/../../../../arm-none-eabi/lib/thumb/v8-m.main+fp/hard\libc_nano.a(lib_a-findfp.o)
 .text          0x00000000        0x0 c:/renesas/ra/e2studio_v2022-10_fsp_v4.2.0/toolchains/gcc_arm/gcc-arm-none-eabi-10.3-2021.10/bin/../lib/gcc/arm-none-eabi/10.3.1/../../../../arm-none-eabi/lib/thumb/v8-m.main+fp/hard\libc_nano.a(lib_a-fwalk.o)
 .data          0x00000000        0x0 c:/renesas/ra/e2studio_v2022-10_fsp_v4.2.0/toolchains/gcc_arm/gcc-arm-none-eabi-10.3-2021.10/bin/../lib/gcc/arm-none-eabi/10.3.1/../../../../arm-none-eabi/lib/thumb/v8-m.main+fp/hard\libc_nano.a(lib_a-fwalk.o)
 .bss           0x00000000        0x0 c:/renesas/ra/e2studio_v2022-10_fsp_v4.2.0/toolchains/gcc_arm/gcc-arm-none-eabi-10.3-2021.10/bin/../lib/gcc/arm-none-eabi/10.3.1/../../../../arm-none-eabi/lib/thumb/v8-m.main+fp/hard\libc_nano.a(lib_a-fwalk.o)
 .text._fwalk   0x00000000       0x3a c:/renesas/ra/e2studio_v2022-10_fsp_v4.2.0/toolchains/gcc_arm/gcc-arm-none-eabi-10.3-2021.10/bin/../lib/gcc/arm-none-eabi/10.3.1/../../../../arm-none-eabi/lib/thumb/v8-m.main+fp/hard\libc_nano.a(lib_a-fwalk.o)
 .text._fwalk_reent
                0x00000000       0x3e c:/renesas/ra/e2studio_v2022-10_fsp_v4.2.0/toolchains/gcc_arm/gcc-arm-none-eabi-10.3-2021.10/bin/../lib/gcc/arm-none-eabi/10.3.1/../../../../arm-none-eabi/lib/thumb/v8-m.main+fp/hard\libc_nano.a(lib_a-fwalk.o)
 .debug_frame   0x00000000       0x54 c:/renesas/ra/e2studio_v2022-10_fsp_v4.2.0/toolchains/gcc_arm/gcc-arm-none-eabi-10.3-2021.10/bin/../lib/gcc/arm-none-eabi/10.3.1/../../../../arm-none-eabi/lib/thumb/v8-m.main+fp/hard\libc_nano.a(lib_a-fwalk.o)
 .ARM.attributes
                0x00000000       0x38 c:/renesas/ra/e2studio_v2022-10_fsp_v4.2.0/toolchains/gcc_arm/gcc-arm-none-eabi-10.3-2021.10/bin/../lib/gcc/arm-none-eabi/10.3.1/../../../../arm-none-eabi/lib/thumb/v8-m.main+fp/hard\libc_nano.a(lib_a-fwalk.o)
 .text          0x00000000        0x0 c:/renesas/ra/e2studio_v2022-10_fsp_v4.2.0/toolchains/gcc_arm/gcc-arm-none-eabi-10.3-2021.10/bin/../lib/gcc/arm-none-eabi/10.3.1/../../../../arm-none-eabi/lib/thumb/v8-m.main+fp/hard\libc_nano.a(lib_a-lock.o)
 .data          0x00000000        0x0 c:/renesas/ra/e2studio_v2022-10_fsp_v4.2.0/toolchains/gcc_arm/gcc-arm-none-eabi-10.3-2021.10/bin/../lib/gcc/arm-none-eabi/10.3.1/../../../../arm-none-eabi/lib/thumb/v8-m.main+fp/hard\libc_nano.a(lib_a-lock.o)
 .bss           0x00000000        0x0 c:/renesas/ra/e2studio_v2022-10_fsp_v4.2.0/toolchains/gcc_arm/gcc-arm-none-eabi-10.3-2021.10/bin/../lib/gcc/arm-none-eabi/10.3.1/../../../../arm-none-eabi/lib/thumb/v8-m.main+fp/hard\libc_nano.a(lib_a-lock.o)
 .text.__retarget_lock_init
                0x00000000        0x2 c:/renesas/ra/e2studio_v2022-10_fsp_v4.2.0/toolchains/gcc_arm/gcc-arm-none-eabi-10.3-2021.10/bin/../lib/gcc/arm-none-eabi/10.3.1/../../../../arm-none-eabi/lib/thumb/v8-m.main+fp/hard\libc_nano.a(lib_a-lock.o)
 .text.__retarget_lock_init_recursive
                0x00000000        0x2 c:/renesas/ra/e2studio_v2022-10_fsp_v4.2.0/toolchains/gcc_arm/gcc-arm-none-eabi-10.3-2021.10/bin/../lib/gcc/arm-none-eabi/10.3.1/../../../../arm-none-eabi/lib/thumb/v8-m.main+fp/hard\libc_nano.a(lib_a-lock.o)
 .text.__retarget_lock_close
                0x00000000        0x2 c:/renesas/ra/e2studio_v2022-10_fsp_v4.2.0/toolchains/gcc_arm/gcc-arm-none-eabi-10.3-2021.10/bin/../lib/gcc/arm-none-eabi/10.3.1/../../../../arm-none-eabi/lib/thumb/v8-m.main+fp/hard\libc_nano.a(lib_a-lock.o)
 .text.__retarget_lock_close_recursive
                0x00000000        0x2 c:/renesas/ra/e2studio_v2022-10_fsp_v4.2.0/toolchains/gcc_arm/gcc-arm-none-eabi-10.3-2021.10/bin/../lib/gcc/arm-none-eabi/10.3.1/../../../../arm-none-eabi/lib/thumb/v8-m.main+fp/hard\libc_nano.a(lib_a-lock.o)
 .text.__retarget_lock_acquire
                0x00000000        0x2 c:/renesas/ra/e2studio_v2022-10_fsp_v4.2.0/toolchains/gcc_arm/gcc-arm-none-eabi-10.3-2021.10/bin/../lib/gcc/arm-none-eabi/10.3.1/../../../../arm-none-eabi/lib/thumb/v8-m.main+fp/hard\libc_nano.a(lib_a-lock.o)
 .text.__retarget_lock_acquire_recursive
                0x00000000        0x2 c:/renesas/ra/e2studio_v2022-10_fsp_v4.2.0/toolchains/gcc_arm/gcc-arm-none-eabi-10.3-2021.10/bin/../lib/gcc/arm-none-eabi/10.3.1/../../../../arm-none-eabi/lib/thumb/v8-m.main+fp/hard\libc_nano.a(lib_a-lock.o)
 .text.__retarget_lock_try_acquire
                0x00000000        0x4 c:/renesas/ra/e2studio_v2022-10_fsp_v4.2.0/toolchains/gcc_arm/gcc-arm-none-eabi-10.3-2021.10/bin/../lib/gcc/arm-none-eabi/10.3.1/../../../../arm-none-eabi/lib/thumb/v8-m.main+fp/hard\libc_nano.a(lib_a-lock.o)
 .text.__retarget_lock_try_acquire_recursive
                0x00000000        0x4 c:/renesas/ra/e2studio_v2022-10_fsp_v4.2.0/toolchains/gcc_arm/gcc-arm-none-eabi-10.3-2021.10/bin/../lib/gcc/arm-none-eabi/10.3.1/../../../../arm-none-eabi/lib/thumb/v8-m.main+fp/hard\libc_nano.a(lib_a-lock.o)
 .text.__retarget_lock_release
                0x00000000        0x2 c:/renesas/ra/e2studio_v2022-10_fsp_v4.2.0/toolchains/gcc_arm/gcc-arm-none-eabi-10.3-2021.10/bin/../lib/gcc/arm-none-eabi/10.3.1/../../../../arm-none-eabi/lib/thumb/v8-m.main+fp/hard\libc_nano.a(lib_a-lock.o)
 .text.__retarget_lock_release_recursive
                0x00000000        0x2 c:/renesas/ra/e2studio_v2022-10_fsp_v4.2.0/toolchains/gcc_arm/gcc-arm-none-eabi-10.3-2021.10/bin/../lib/gcc/arm-none-eabi/10.3.1/../../../../arm-none-eabi/lib/thumb/v8-m.main+fp/hard\libc_nano.a(lib_a-lock.o)
 .bss.__lock___arc4random_mutex
                0x00000000        0x1 c:/renesas/ra/e2studio_v2022-10_fsp_v4.2.0/toolchains/gcc_arm/gcc-arm-none-eabi-10.3-2021.10/bin/../lib/gcc/arm-none-eabi/10.3.1/../../../../arm-none-eabi/lib/thumb/v8-m.main+fp/hard\libc_nano.a(lib_a-lock.o)
 .bss.__lock___at_quick_exit_mutex
                0x00000000        0x1 c:/renesas/ra/e2studio_v2022-10_fsp_v4.2.0/toolchains/gcc_arm/gcc-arm-none-eabi-10.3-2021.10/bin/../lib/gcc/arm-none-eabi/10.3.1/../../../../arm-none-eabi/lib/thumb/v8-m.main+fp/hard\libc_nano.a(lib_a-lock.o)
 .bss.__lock___atexit_recursive_mutex
                0x00000000        0x1 c:/renesas/ra/e2studio_v2022-10_fsp_v4.2.0/toolchains/gcc_arm/gcc-arm-none-eabi-10.3-2021.10/bin/../lib/gcc/arm-none-eabi/10.3.1/../../../../arm-none-eabi/lib/thumb/v8-m.main+fp/hard\libc_nano.a(lib_a-lock.o)
 .bss.__lock___dd_hash_mutex
                0x00000000        0x1 c:/renesas/ra/e2studio_v2022-10_fsp_v4.2.0/toolchains/gcc_arm/gcc-arm-none-eabi-10.3-2021.10/bin/../lib/gcc/arm-none-eabi/10.3.1/../../../../arm-none-eabi/lib/thumb/v8-m.main+fp/hard\libc_nano.a(lib_a-lock.o)
 .bss.__lock___env_recursive_mutex
                0x00000000        0x1 c:/renesas/ra/e2studio_v2022-10_fsp_v4.2.0/toolchains/gcc_arm/gcc-arm-none-eabi-10.3-2021.10/bin/../lib/gcc/arm-none-eabi/10.3.1/../../../../arm-none-eabi/lib/thumb/v8-m.main+fp/hard\libc_nano.a(lib_a-lock.o)
 .bss.__lock___malloc_recursive_mutex
                0x00000000        0x1 c:/renesas/ra/e2studio_v2022-10_fsp_v4.2.0/toolchains/gcc_arm/gcc-arm-none-eabi-10.3-2021.10/bin/../lib/gcc/arm-none-eabi/10.3.1/../../../../arm-none-eabi/lib/thumb/v8-m.main+fp/hard\libc_nano.a(lib_a-lock.o)
 .bss.__lock___sfp_recursive_mutex
                0x00000000        0x1 c:/renesas/ra/e2studio_v2022-10_fsp_v4.2.0/toolchains/gcc_arm/gcc-arm-none-eabi-10.3-2021.10/bin/../lib/gcc/arm-none-eabi/10.3.1/../../../../arm-none-eabi/lib/thumb/v8-m.main+fp/hard\libc_nano.a(lib_a-lock.o)
 .bss.__lock___sinit_recursive_mutex
                0x00000000        0x1 c:/renesas/ra/e2studio_v2022-10_fsp_v4.2.0/toolchains/gcc_arm/gcc-arm-none-eabi-10.3-2021.10/bin/../lib/gcc/arm-none-eabi/10.3.1/../../../../arm-none-eabi/lib/thumb/v8-m.main+fp/hard\libc_nano.a(lib_a-lock.o)
 .bss.__lock___tz_mutex
                0x00000000        0x1 c:/renesas/ra/e2studio_v2022-10_fsp_v4.2.0/toolchains/gcc_arm/gcc-arm-none-eabi-10.3-2021.10/bin/../lib/gcc/arm-none-eabi/10.3.1/../../../../arm-none-eabi/lib/thumb/v8-m.main+fp/hard\libc_nano.a(lib_a-lock.o)
 .debug_frame   0x00000000       0xb0 c:/renesas/ra/e2studio_v2022-10_fsp_v4.2.0/toolchains/gcc_arm/gcc-arm-none-eabi-10.3-2021.10/bin/../lib/gcc/arm-none-eabi/10.3.1/../../../../arm-none-eabi/lib/thumb/v8-m.main+fp/hard\libc_nano.a(lib_a-lock.o)
 .ARM.attributes
                0x00000000       0x38 c:/renesas/ra/e2studio_v2022-10_fsp_v4.2.0/toolchains/gcc_arm/gcc-arm-none-eabi-10.3-2021.10/bin/../lib/gcc/arm-none-eabi/10.3.1/../../../../arm-none-eabi/lib/thumb/v8-m.main+fp/hard\libc_nano.a(lib_a-lock.o)
 .text          0x00000000        0x0 c:/renesas/ra/e2studio_v2022-10_fsp_v4.2.0/toolchains/gcc_arm/gcc-arm-none-eabi-10.3-2021.10/bin/../lib/gcc/arm-none-eabi/10.3.1/../../../../arm-none-eabi/lib/thumb/v8-m.main+fp/hard\libc_nano.a(lib_a-nano-mallocr.o)
 .data          0x00000000        0x0 c:/renesas/ra/e2studio_v2022-10_fsp_v4.2.0/toolchains/gcc_arm/gcc-arm-none-eabi-10.3-2021.10/bin/../lib/gcc/arm-none-eabi/10.3.1/../../../../arm-none-eabi/lib/thumb/v8-m.main+fp/hard\libc_nano.a(lib_a-nano-mallocr.o)
 .bss           0x00000000        0x0 c:/renesas/ra/e2studio_v2022-10_fsp_v4.2.0/toolchains/gcc_arm/gcc-arm-none-eabi-10.3-2021.10/bin/../lib/gcc/arm-none-eabi/10.3.1/../../../../arm-none-eabi/lib/thumb/v8-m.main+fp/hard\libc_nano.a(lib_a-nano-mallocr.o)
 .text.sbrk_aligned
                0x00000000       0x40 c:/renesas/ra/e2studio_v2022-10_fsp_v4.2.0/toolchains/gcc_arm/gcc-arm-none-eabi-10.3-2021.10/bin/../lib/gcc/arm-none-eabi/10.3.1/../../../../arm-none-eabi/lib/thumb/v8-m.main+fp/hard\libc_nano.a(lib_a-nano-mallocr.o)
 .text._malloc_r
                0x00000000       0xe8 c:/renesas/ra/e2studio_v2022-10_fsp_v4.2.0/toolchains/gcc_arm/gcc-arm-none-eabi-10.3-2021.10/bin/../lib/gcc/arm-none-eabi/10.3.1/../../../../arm-none-eabi/lib/thumb/v8-m.main+fp/hard\libc_nano.a(lib_a-nano-mallocr.o)
 .bss.__malloc_free_list
                0x00000000        0x4 c:/renesas/ra/e2studio_v2022-10_fsp_v4.2.0/toolchains/gcc_arm/gcc-arm-none-eabi-10.3-2021.10/bin/../lib/gcc/arm-none-eabi/10.3.1/../../../../arm-none-eabi/lib/thumb/v8-m.main+fp/hard\libc_nano.a(lib_a-nano-mallocr.o)
 .bss.__malloc_sbrk_start
                0x00000000        0x4 c:/renesas/ra/e2studio_v2022-10_fsp_v4.2.0/toolchains/gcc_arm/gcc-arm-none-eabi-10.3-2021.10/bin/../lib/gcc/arm-none-eabi/10.3.1/../../../../arm-none-eabi/lib/thumb/v8-m.main+fp/hard\libc_nano.a(lib_a-nano-mallocr.o)
 .debug_frame   0x00000000       0x4c c:/renesas/ra/e2studio_v2022-10_fsp_v4.2.0/toolchains/gcc_arm/gcc-arm-none-eabi-10.3-2021.10/bin/../lib/gcc/arm-none-eabi/10.3.1/../../../../arm-none-eabi/lib/thumb/v8-m.main+fp/hard\libc_nano.a(lib_a-nano-mallocr.o)
 .ARM.attributes
                0x00000000       0x38 c:/renesas/ra/e2studio_v2022-10_fsp_v4.2.0/toolchains/gcc_arm/gcc-arm-none-eabi-10.3-2021.10/bin/../lib/gcc/arm-none-eabi/10.3.1/../../../../arm-none-eabi/lib/thumb/v8-m.main+fp/hard\libc_nano.a(lib_a-nano-mallocr.o)
 .text          0x00000000        0x0 c:/renesas/ra/e2studio_v2022-10_fsp_v4.2.0/toolchains/gcc_arm/gcc-arm-none-eabi-10.3-2021.10/bin/../lib/gcc/arm-none-eabi/10.3.1/../../../../arm-none-eabi/lib/thumb/v8-m.main+fp/hard\libc_nano.a(lib_a-sbrkr.o)
 .data          0x00000000        0x0 c:/renesas/ra/e2studio_v2022-10_fsp_v4.2.0/toolchains/gcc_arm/gcc-arm-none-eabi-10.3-2021.10/bin/../lib/gcc/arm-none-eabi/10.3.1/../../../../arm-none-eabi/lib/thumb/v8-m.main+fp/hard\libc_nano.a(lib_a-sbrkr.o)
 .bss           0x00000000        0x0 c:/renesas/ra/e2studio_v2022-10_fsp_v4.2.0/toolchains/gcc_arm/gcc-arm-none-eabi-10.3-2021.10/bin/../lib/gcc/arm-none-eabi/10.3.1/../../../../arm-none-eabi/lib/thumb/v8-m.main+fp/hard\libc_nano.a(lib_a-sbrkr.o)
 .text._sbrk_r  0x00000000       0x20 c:/renesas/ra/e2studio_v2022-10_fsp_v4.2.0/toolchains/gcc_arm/gcc-arm-none-eabi-10.3-2021.10/bin/../lib/gcc/arm-none-eabi/10.3.1/../../../../arm-none-eabi/lib/thumb/v8-m.main+fp/hard\libc_nano.a(lib_a-sbrkr.o)
 .debug_frame   0x00000000       0x2c c:/renesas/ra/e2studio_v2022-10_fsp_v4.2.0/toolchains/gcc_arm/gcc-arm-none-eabi-10.3-2021.10/bin/../lib/gcc/arm-none-eabi/10.3.1/../../../../arm-none-eabi/lib/thumb/v8-m.main+fp/hard\libc_nano.a(lib_a-sbrkr.o)
 .ARM.attributes
                0x00000000       0x38 c:/renesas/ra/e2studio_v2022-10_fsp_v4.2.0/toolchains/gcc_arm/gcc-arm-none-eabi-10.3-2021.10/bin/../lib/gcc/arm-none-eabi/10.3.1/../../../../arm-none-eabi/lib/thumb/v8-m.main+fp/hard\libc_nano.a(lib_a-sbrkr.o)
 .text          0x00000000        0x0 c:/renesas/ra/e2studio_v2022-10_fsp_v4.2.0/toolchains/gcc_arm/gcc-arm-none-eabi-10.3-2021.10/bin/../lib/gcc/arm-none-eabi/10.3.1/../../../../arm-none-eabi/lib/thumb/v8-m.main+fp/hard\libc_nano.a(lib_a-stdio.o)
 .data          0x00000000        0x0 c:/renesas/ra/e2studio_v2022-10_fsp_v4.2.0/toolchains/gcc_arm/gcc-arm-none-eabi-10.3-2021.10/bin/../lib/gcc/arm-none-eabi/10.3.1/../../../../arm-none-eabi/lib/thumb/v8-m.main+fp/hard\libc_nano.a(lib_a-stdio.o)
 .bss           0x00000000        0x0 c:/renesas/ra/e2studio_v2022-10_fsp_v4.2.0/toolchains/gcc_arm/gcc-arm-none-eabi-10.3-2021.10/bin/../lib/gcc/arm-none-eabi/10.3.1/../../../../arm-none-eabi/lib/thumb/v8-m.main+fp/hard\libc_nano.a(lib_a-stdio.o)
 .text.__sread  0x00000000       0x22 c:/renesas/ra/e2studio_v2022-10_fsp_v4.2.0/toolchains/gcc_arm/gcc-arm-none-eabi-10.3-2021.10/bin/../lib/gcc/arm-none-eabi/10.3.1/../../../../arm-none-eabi/lib/thumb/v8-m.main+fp/hard\libc_nano.a(lib_a-stdio.o)
 .text.__seofread
                0x00000000        0x4 c:/renesas/ra/e2studio_v2022-10_fsp_v4.2.0/toolchains/gcc_arm/gcc-arm-none-eabi-10.3-2021.10/bin/../lib/gcc/arm-none-eabi/10.3.1/../../../../arm-none-eabi/lib/thumb/v8-m.main+fp/hard\libc_nano.a(lib_a-stdio.o)
 .text.__swrite
                0x00000000       0x38 c:/renesas/ra/e2studio_v2022-10_fsp_v4.2.0/toolchains/gcc_arm/gcc-arm-none-eabi-10.3-2021.10/bin/../lib/gcc/arm-none-eabi/10.3.1/../../../../arm-none-eabi/lib/thumb/v8-m.main+fp/hard\libc_nano.a(lib_a-stdio.o)
 .text.__sseek  0x00000000       0x24 c:/renesas/ra/e2studio_v2022-10_fsp_v4.2.0/toolchains/gcc_arm/gcc-arm-none-eabi-10.3-2021.10/bin/../lib/gcc/arm-none-eabi/10.3.1/../../../../arm-none-eabi/lib/thumb/v8-m.main+fp/hard\libc_nano.a(lib_a-stdio.o)
 .text.__sclose
                0x00000000        0x8 c:/renesas/ra/e2studio_v2022-10_fsp_v4.2.0/toolchains/gcc_arm/gcc-arm-none-eabi-10.3-2021.10/bin/../lib/gcc/arm-none-eabi/10.3.1/../../../../arm-none-eabi/lib/thumb/v8-m.main+fp/hard\libc_nano.a(lib_a-stdio.o)
 .debug_frame   0x00000000       0x88 c:/renesas/ra/e2studio_v2022-10_fsp_v4.2.0/toolchains/gcc_arm/gcc-arm-none-eabi-10.3-2021.10/bin/../lib/gcc/arm-none-eabi/10.3.1/../../../../arm-none-eabi/lib/thumb/v8-m.main+fp/hard\libc_nano.a(lib_a-stdio.o)
 .ARM.attributes
                0x00000000       0x38 c:/renesas/ra/e2studio_v2022-10_fsp_v4.2.0/toolchains/gcc_arm/gcc-arm-none-eabi-10.3-2021.10/bin/../lib/gcc/arm-none-eabi/10.3.1/../../../../arm-none-eabi/lib/thumb/v8-m.main+fp/hard\libc_nano.a(lib_a-stdio.o)
 .text          0x00000000        0x0 c:/renesas/ra/e2studio_v2022-10_fsp_v4.2.0/toolchains/gcc_arm/gcc-arm-none-eabi-10.3-2021.10/bin/../lib/gcc/arm-none-eabi/10.3.1/../../../../arm-none-eabi/lib/thumb/v8-m.main+fp/hard\libc_nano.a(lib_a-writer.o)
 .data          0x00000000        0x0 c:/renesas/ra/e2studio_v2022-10_fsp_v4.2.0/toolchains/gcc_arm/gcc-arm-none-eabi-10.3-2021.10/bin/../lib/gcc/arm-none-eabi/10.3.1/../../../../arm-none-eabi/lib/thumb/v8-m.main+fp/hard\libc_nano.a(lib_a-writer.o)
 .bss           0x00000000        0x0 c:/renesas/ra/e2studio_v2022-10_fsp_v4.2.0/toolchains/gcc_arm/gcc-arm-none-eabi-10.3-2021.10/bin/../lib/gcc/arm-none-eabi/10.3.1/../../../../arm-none-eabi/lib/thumb/v8-m.main+fp/hard\libc_nano.a(lib_a-writer.o)
 .text._write_r
                0x00000000       0x24 c:/renesas/ra/e2studio_v2022-10_fsp_v4.2.0/toolchains/gcc_arm/gcc-arm-none-eabi-10.3-2021.10/bin/../lib/gcc/arm-none-eabi/10.3.1/../../../../arm-none-eabi/lib/thumb/v8-m.main+fp/hard\libc_nano.a(lib_a-writer.o)
 .debug_frame   0x00000000       0x2c c:/renesas/ra/e2studio_v2022-10_fsp_v4.2.0/toolchains/gcc_arm/gcc-arm-none-eabi-10.3-2021.10/bin/../lib/gcc/arm-none-eabi/10.3.1/../../../../arm-none-eabi/lib/thumb/v8-m.main+fp/hard\libc_nano.a(lib_a-writer.o)
 .ARM.attributes
                0x00000000       0x38 c:/renesas/ra/e2studio_v2022-10_fsp_v4.2.0/toolchains/gcc_arm/gcc-arm-none-eabi-10.3-2021.10/bin/../lib/gcc/arm-none-eabi/10.3.1/../../../../arm-none-eabi/lib/thumb/v8-m.main+fp/hard\libc_nano.a(lib_a-writer.o)
 .text          0x00000000        0x0 c:/renesas/ra/e2studio_v2022-10_fsp_v4.2.0/toolchains/gcc_arm/gcc-arm-none-eabi-10.3-2021.10/bin/../lib/gcc/arm-none-eabi/10.3.1/../../../../arm-none-eabi/lib/thumb/v8-m.main+fp/hard\libc_nano.a(lib_a-closer.o)
 .data          0x00000000        0x0 c:/renesas/ra/e2studio_v2022-10_fsp_v4.2.0/toolchains/gcc_arm/gcc-arm-none-eabi-10.3-2021.10/bin/../lib/gcc/arm-none-eabi/10.3.1/../../../../arm-none-eabi/lib/thumb/v8-m.main+fp/hard\libc_nano.a(lib_a-closer.o)
 .bss           0x00000000        0x0 c:/renesas/ra/e2studio_v2022-10_fsp_v4.2.0/toolchains/gcc_arm/gcc-arm-none-eabi-10.3-2021.10/bin/../lib/gcc/arm-none-eabi/10.3.1/../../../../arm-none-eabi/lib/thumb/v8-m.main+fp/hard\libc_nano.a(lib_a-closer.o)
 .text._close_r
                0x00000000       0x20 c:/renesas/ra/e2studio_v2022-10_fsp_v4.2.0/toolchains/gcc_arm/gcc-arm-none-eabi-10.3-2021.10/bin/../lib/gcc/arm-none-eabi/10.3.1/../../../../arm-none-eabi/lib/thumb/v8-m.main+fp/hard\libc_nano.a(lib_a-closer.o)
 .debug_frame   0x00000000       0x2c c:/renesas/ra/e2studio_v2022-10_fsp_v4.2.0/toolchains/gcc_arm/gcc-arm-none-eabi-10.3-2021.10/bin/../lib/gcc/arm-none-eabi/10.3.1/../../../../arm-none-eabi/lib/thumb/v8-m.main+fp/hard\libc_nano.a(lib_a-closer.o)
 .ARM.attributes
                0x00000000       0x38 c:/renesas/ra/e2studio_v2022-10_fsp_v4.2.0/toolchains/gcc_arm/gcc-arm-none-eabi-10.3-2021.10/bin/../lib/gcc/arm-none-eabi/10.3.1/../../../../arm-none-eabi/lib/thumb/v8-m.main+fp/hard\libc_nano.a(lib_a-closer.o)
 .text          0x00000000        0x0 c:/renesas/ra/e2studio_v2022-10_fsp_v4.2.0/toolchains/gcc_arm/gcc-arm-none-eabi-10.3-2021.10/bin/../lib/gcc/arm-none-eabi/10.3.1/../../../../arm-none-eabi/lib/thumb/v8-m.main+fp/hard\libc_nano.a(lib_a-fflush.o)
 .data          0x00000000        0x0 c:/renesas/ra/e2studio_v2022-10_fsp_v4.2.0/toolchains/gcc_arm/gcc-arm-none-eabi-10.3-2021.10/bin/../lib/gcc/arm-none-eabi/10.3.1/../../../../arm-none-eabi/lib/thumb/v8-m.main+fp/hard\libc_nano.a(lib_a-fflush.o)
 .bss           0x00000000        0x0 c:/renesas/ra/e2studio_v2022-10_fsp_v4.2.0/toolchains/gcc_arm/gcc-arm-none-eabi-10.3-2021.10/bin/../lib/gcc/arm-none-eabi/10.3.1/../../../../arm-none-eabi/lib/thumb/v8-m.main+fp/hard\libc_nano.a(lib_a-fflush.o)
 .text.__sflush_r
                0x00000000      0x108 c:/renesas/ra/e2studio_v2022-10_fsp_v4.2.0/toolchains/gcc_arm/gcc-arm-none-eabi-10.3-2021.10/bin/../lib/gcc/arm-none-eabi/10.3.1/../../../../arm-none-eabi/lib/thumb/v8-m.main+fp/hard\libc_nano.a(lib_a-fflush.o)
 .text._fflush_r
                0x00000000       0x78 c:/renesas/ra/e2studio_v2022-10_fsp_v4.2.0/toolchains/gcc_arm/gcc-arm-none-eabi-10.3-2021.10/bin/../lib/gcc/arm-none-eabi/10.3.1/../../../../arm-none-eabi/lib/thumb/v8-m.main+fp/hard\libc_nano.a(lib_a-fflush.o)
 .text.fflush   0x00000000       0x24 c:/renesas/ra/e2studio_v2022-10_fsp_v4.2.0/toolchains/gcc_arm/gcc-arm-none-eabi-10.3-2021.10/bin/../lib/gcc/arm-none-eabi/10.3.1/../../../../arm-none-eabi/lib/thumb/v8-m.main+fp/hard\libc_nano.a(lib_a-fflush.o)
 .debug_frame   0x00000000       0x5c c:/renesas/ra/e2studio_v2022-10_fsp_v4.2.0/toolchains/gcc_arm/gcc-arm-none-eabi-10.3-2021.10/bin/../lib/gcc/arm-none-eabi/10.3.1/../../../../arm-none-eabi/lib/thumb/v8-m.main+fp/hard\libc_nano.a(lib_a-fflush.o)
 .ARM.attributes
                0x00000000       0x38 c:/renesas/ra/e2studio_v2022-10_fsp_v4.2.0/toolchains/gcc_arm/gcc-arm-none-eabi-10.3-2021.10/bin/../lib/gcc/arm-none-eabi/10.3.1/../../../../arm-none-eabi/lib/thumb/v8-m.main+fp/hard\libc_nano.a(lib_a-fflush.o)
 .text          0x00000000        0x0 c:/renesas/ra/e2studio_v2022-10_fsp_v4.2.0/toolchains/gcc_arm/gcc-arm-none-eabi-10.3-2021.10/bin/../lib/gcc/arm-none-eabi/10.3.1/../../../../arm-none-eabi/lib/thumb/v8-m.main+fp/hard\libc_nano.a(lib_a-lseekr.o)
 .data          0x00000000        0x0 c:/renesas/ra/e2studio_v2022-10_fsp_v4.2.0/toolchains/gcc_arm/gcc-arm-none-eabi-10.3-2021.10/bin/../lib/gcc/arm-none-eabi/10.3.1/../../../../arm-none-eabi/lib/thumb/v8-m.main+fp/hard\libc_nano.a(lib_a-lseekr.o)
 .bss           0x00000000        0x0 c:/renesas/ra/e2studio_v2022-10_fsp_v4.2.0/toolchains/gcc_arm/gcc-arm-none-eabi-10.3-2021.10/bin/../lib/gcc/arm-none-eabi/10.3.1/../../../../arm-none-eabi/lib/thumb/v8-m.main+fp/hard\libc_nano.a(lib_a-lseekr.o)
 .text._lseek_r
                0x00000000       0x24 c:/renesas/ra/e2studio_v2022-10_fsp_v4.2.0/toolchains/gcc_arm/gcc-arm-none-eabi-10.3-2021.10/bin/../lib/gcc/arm-none-eabi/10.3.1/../../../../arm-none-eabi/lib/thumb/v8-m.main+fp/hard\libc_nano.a(lib_a-lseekr.o)
 .debug_frame   0x00000000       0x2c c:/renesas/ra/e2studio_v2022-10_fsp_v4.2.0/toolchains/gcc_arm/gcc-arm-none-eabi-10.3-2021.10/bin/../lib/gcc/arm-none-eabi/10.3.1/../../../../arm-none-eabi/lib/thumb/v8-m.main+fp/hard\libc_nano.a(lib_a-lseekr.o)
 .ARM.attributes
                0x00000000       0x38 c:/renesas/ra/e2studio_v2022-10_fsp_v4.2.0/toolchains/gcc_arm/gcc-arm-none-eabi-10.3-2021.10/bin/../lib/gcc/arm-none-eabi/10.3.1/../../../../arm-none-eabi/lib/thumb/v8-m.main+fp/hard\libc_nano.a(lib_a-lseekr.o)
 .text          0x00000000        0x0 c:/renesas/ra/e2studio_v2022-10_fsp_v4.2.0/toolchains/gcc_arm/gcc-arm-none-eabi-10.3-2021.10/bin/../lib/gcc/arm-none-eabi/10.3.1/../../../../arm-none-eabi/lib/thumb/v8-m.main+fp/hard\libc_nano.a(lib_a-mlock.o)
 .data          0x00000000        0x0 c:/renesas/ra/e2studio_v2022-10_fsp_v4.2.0/toolchains/gcc_arm/gcc-arm-none-eabi-10.3-2021.10/bin/../lib/gcc/arm-none-eabi/10.3.1/../../../../arm-none-eabi/lib/thumb/v8-m.main+fp/hard\libc_nano.a(lib_a-mlock.o)
 .bss           0x00000000        0x0 c:/renesas/ra/e2studio_v2022-10_fsp_v4.2.0/toolchains/gcc_arm/gcc-arm-none-eabi-10.3-2021.10/bin/../lib/gcc/arm-none-eabi/10.3.1/../../../../arm-none-eabi/lib/thumb/v8-m.main+fp/hard\libc_nano.a(lib_a-mlock.o)
 .text.__malloc_lock
                0x00000000        0xc c:/renesas/ra/e2studio_v2022-10_fsp_v4.2.0/toolchains/gcc_arm/gcc-arm-none-eabi-10.3-2021.10/bin/../lib/gcc/arm-none-eabi/10.3.1/../../../../arm-none-eabi/lib/thumb/v8-m.main+fp/hard\libc_nano.a(lib_a-mlock.o)
 .text.__malloc_unlock
                0x00000000        0xc c:/renesas/ra/e2studio_v2022-10_fsp_v4.2.0/toolchains/gcc_arm/gcc-arm-none-eabi-10.3-2021.10/bin/../lib/gcc/arm-none-eabi/10.3.1/../../../../arm-none-eabi/lib/thumb/v8-m.main+fp/hard\libc_nano.a(lib_a-mlock.o)
 .debug_frame   0x00000000       0x30 c:/renesas/ra/e2studio_v2022-10_fsp_v4.2.0/toolchains/gcc_arm/gcc-arm-none-eabi-10.3-2021.10/bin/../lib/gcc/arm-none-eabi/10.3.1/../../../../arm-none-eabi/lib/thumb/v8-m.main+fp/hard\libc_nano.a(lib_a-mlock.o)
 .ARM.attributes
                0x00000000       0x38 c:/renesas/ra/e2studio_v2022-10_fsp_v4.2.0/toolchains/gcc_arm/gcc-arm-none-eabi-10.3-2021.10/bin/../lib/gcc/arm-none-eabi/10.3.1/../../../../arm-none-eabi/lib/thumb/v8-m.main+fp/hard\libc_nano.a(lib_a-mlock.o)
 .text          0x00000000        0x0 c:/renesas/ra/e2studio_v2022-10_fsp_v4.2.0/toolchains/gcc_arm/gcc-arm-none-eabi-10.3-2021.10/bin/../lib/gcc/arm-none-eabi/10.3.1/../../../../arm-none-eabi/lib/thumb/v8-m.main+fp/hard\libc_nano.a(lib_a-nano-freer.o)
 .data          0x00000000        0x0 c:/renesas/ra/e2studio_v2022-10_fsp_v4.2.0/toolchains/gcc_arm/gcc-arm-none-eabi-10.3-2021.10/bin/../lib/gcc/arm-none-eabi/10.3.1/../../../../arm-none-eabi/lib/thumb/v8-m.main+fp/hard\libc_nano.a(lib_a-nano-freer.o)
 .bss           0x00000000        0x0 c:/renesas/ra/e2studio_v2022-10_fsp_v4.2.0/toolchains/gcc_arm/gcc-arm-none-eabi-10.3-2021.10/bin/../lib/gcc/arm-none-eabi/10.3.1/../../../../arm-none-eabi/lib/thumb/v8-m.main+fp/hard\libc_nano.a(lib_a-nano-freer.o)
 .text._free_r  0x00000000       0x98 c:/renesas/ra/e2studio_v2022-10_fsp_v4.2.0/toolchains/gcc_arm/gcc-arm-none-eabi-10.3-2021.10/bin/../lib/gcc/arm-none-eabi/10.3.1/../../../../arm-none-eabi/lib/thumb/v8-m.main+fp/hard\libc_nano.a(lib_a-nano-freer.o)
 .debug_frame   0x00000000       0x38 c:/renesas/ra/e2studio_v2022-10_fsp_v4.2.0/toolchains/gcc_arm/gcc-arm-none-eabi-10.3-2021.10/bin/../lib/gcc/arm-none-eabi/10.3.1/../../../../arm-none-eabi/lib/thumb/v8-m.main+fp/hard\libc_nano.a(lib_a-nano-freer.o)
 .ARM.attributes
                0x00000000       0x38 c:/renesas/ra/e2studio_v2022-10_fsp_v4.2.0/toolchains/gcc_arm/gcc-arm-none-eabi-10.3-2021.10/bin/../lib/gcc/arm-none-eabi/10.3.1/../../../../arm-none-eabi/lib/thumb/v8-m.main+fp/hard\libc_nano.a(lib_a-nano-freer.o)
 .text          0x00000000        0x0 c:/renesas/ra/e2studio_v2022-10_fsp_v4.2.0/toolchains/gcc_arm/gcc-arm-none-eabi-10.3-2021.10/bin/../lib/gcc/arm-none-eabi/10.3.1/../../../../arm-none-eabi/lib/thumb/v8-m.main+fp/hard\libc_nano.a(lib_a-readr.o)
 .data          0x00000000        0x0 c:/renesas/ra/e2studio_v2022-10_fsp_v4.2.0/toolchains/gcc_arm/gcc-arm-none-eabi-10.3-2021.10/bin/../lib/gcc/arm-none-eabi/10.3.1/../../../../arm-none-eabi/lib/thumb/v8-m.main+fp/hard\libc_nano.a(lib_a-readr.o)
 .bss           0x00000000        0x0 c:/renesas/ra/e2studio_v2022-10_fsp_v4.2.0/toolchains/gcc_arm/gcc-arm-none-eabi-10.3-2021.10/bin/../lib/gcc/arm-none-eabi/10.3.1/../../../../arm-none-eabi/lib/thumb/v8-m.main+fp/hard\libc_nano.a(lib_a-readr.o)
 .text._read_r  0x00000000       0x24 c:/renesas/ra/e2studio_v2022-10_fsp_v4.2.0/toolchains/gcc_arm/gcc-arm-none-eabi-10.3-2021.10/bin/../lib/gcc/arm-none-eabi/10.3.1/../../../../arm-none-eabi/lib/thumb/v8-m.main+fp/hard\libc_nano.a(lib_a-readr.o)
 .debug_frame   0x00000000       0x2c c:/renesas/ra/e2studio_v2022-10_fsp_v4.2.0/toolchains/gcc_arm/gcc-arm-none-eabi-10.3-2021.10/bin/../lib/gcc/arm-none-eabi/10.3.1/../../../../arm-none-eabi/lib/thumb/v8-m.main+fp/hard\libc_nano.a(lib_a-readr.o)
 .ARM.attributes
                0x00000000       0x38 c:/renesas/ra/e2studio_v2022-10_fsp_v4.2.0/toolchains/gcc_arm/gcc-arm-none-eabi-10.3-2021.10/bin/../lib/gcc/arm-none-eabi/10.3.1/../../../../arm-none-eabi/lib/thumb/v8-m.main+fp/hard\libc_nano.a(lib_a-readr.o)
 .text          0x00000000        0x0 c:/renesas/ra/e2studio_v2022-10_fsp_v4.2.0/toolchains/gcc_arm/gcc-arm-none-eabi-10.3-2021.10/bin/../lib/gcc/arm-none-eabi/10.3.1/../../../../arm-none-eabi/lib/thumb/v8-m.main+fp/hard\libc_nano.a(lib_a-reent.o)
 .data          0x00000000        0x0 c:/renesas/ra/e2studio_v2022-10_fsp_v4.2.0/toolchains/gcc_arm/gcc-arm-none-eabi-10.3-2021.10/bin/../lib/gcc/arm-none-eabi/10.3.1/../../../../arm-none-eabi/lib/thumb/v8-m.main+fp/hard\libc_nano.a(lib_a-reent.o)
 .bss           0x00000000        0x0 c:/renesas/ra/e2studio_v2022-10_fsp_v4.2.0/toolchains/gcc_arm/gcc-arm-none-eabi-10.3-2021.10/bin/../lib/gcc/arm-none-eabi/10.3.1/../../../../arm-none-eabi/lib/thumb/v8-m.main+fp/hard\libc_nano.a(lib_a-reent.o)
 .text.cleanup_glue
                0x00000000       0x1a c:/renesas/ra/e2studio_v2022-10_fsp_v4.2.0/toolchains/gcc_arm/gcc-arm-none-eabi-10.3-2021.10/bin/../lib/gcc/arm-none-eabi/10.3.1/../../../../arm-none-eabi/lib/thumb/v8-m.main+fp/hard\libc_nano.a(lib_a-reent.o)
 .text._reclaim_reent
                0x00000000       0xb8 c:/renesas/ra/e2studio_v2022-10_fsp_v4.2.0/toolchains/gcc_arm/gcc-arm-none-eabi-10.3-2021.10/bin/../lib/gcc/arm-none-eabi/10.3.1/../../../../arm-none-eabi/lib/thumb/v8-m.main+fp/hard\libc_nano.a(lib_a-reent.o)
 .bss.errno     0x00000000        0x4 c:/renesas/ra/e2studio_v2022-10_fsp_v4.2.0/toolchains/gcc_arm/gcc-arm-none-eabi-10.3-2021.10/bin/../lib/gcc/arm-none-eabi/10.3.1/../../../../arm-none-eabi/lib/thumb/v8-m.main+fp/hard\libc_nano.a(lib_a-reent.o)
 .debug_frame   0x00000000       0x5c c:/renesas/ra/e2studio_v2022-10_fsp_v4.2.0/toolchains/gcc_arm/gcc-arm-none-eabi-10.3-2021.10/bin/../lib/gcc/arm-none-eabi/10.3.1/../../../../arm-none-eabi/lib/thumb/v8-m.main+fp/hard\libc_nano.a(lib_a-reent.o)
 .ARM.attributes
                0x00000000       0x38 c:/renesas/ra/e2studio_v2022-10_fsp_v4.2.0/toolchains/gcc_arm/gcc-arm-none-eabi-10.3-2021.10/bin/../lib/gcc/arm-none-eabi/10.3.1/../../../../arm-none-eabi/lib/thumb/v8-m.main+fp/hard\libc_nano.a(lib_a-reent.o)
 .text          0x00000000        0x0 c:/renesas/ra/e2studio_v2022-10_fsp_v4.2.0/toolchains/gcc_arm/gcc-arm-none-eabi-10.3-2021.10/bin/../lib/gcc/arm-none-eabi/10.3.1/thumb/v8-m.main+fp/hard/crtend.o
 .data          0x00000000        0x0 c:/renesas/ra/e2studio_v2022-10_fsp_v4.2.0/toolchains/gcc_arm/gcc-arm-none-eabi-10.3-2021.10/bin/../lib/gcc/arm-none-eabi/10.3.1/thumb/v8-m.main+fp/hard/crtend.o
 .bss           0x00000000        0x0 c:/renesas/ra/e2studio_v2022-10_fsp_v4.2.0/toolchains/gcc_arm/gcc-arm-none-eabi-10.3-2021.10/bin/../lib/gcc/arm-none-eabi/10.3.1/thumb/v8-m.main+fp/hard/crtend.o
 .rodata        0x00000000       0x24 c:/renesas/ra/e2studio_v2022-10_fsp_v4.2.0/toolchains/gcc_arm/gcc-arm-none-eabi-10.3-2021.10/bin/../lib/gcc/arm-none-eabi/10.3.1/thumb/v8-m.main+fp/hard/crtend.o
 .text          0x00000000        0x0 c:/renesas/ra/e2studio_v2022-10_fsp_v4.2.0/toolchains/gcc_arm/gcc-arm-none-eabi-10.3-2021.10/bin/../lib/gcc/arm-none-eabi/10.3.1/thumb/v8-m.main+fp/hard/crtn.o
 .data          0x00000000        0x0 c:/renesas/ra/e2studio_v2022-10_fsp_v4.2.0/toolchains/gcc_arm/gcc-arm-none-eabi-10.3-2021.10/bin/../lib/gcc/arm-none-eabi/10.3.1/thumb/v8-m.main+fp/hard/crtn.o
 .bss           0x00000000        0x0 c:/renesas/ra/e2studio_v2022-10_fsp_v4.2.0/toolchains/gcc_arm/gcc-arm-none-eabi-10.3-2021.10/bin/../lib/gcc/arm-none-eabi/10.3.1/thumb/v8-m.main+fp/hard/crtn.o

Memory Configuration

Name             Origin             Length             Attributes
ITCM             0x00000000         0x00000000         xr
DTCM             0x00000000         0x00000000         xrw
FLASH            0x00000000         0x00080000         xr
RAM              0x20000000         0x00020000         xrw
DATA_FLASH       0x08000000         0x00002000         xr
QSPI_FLASH       0x60000000         0x04000000         xr
OSPI_DEVICE_0    0x80020000         0x00000000         xr
OSPI_DEVICE_1    0x80030000         0x00000000         xr
OSPI_DEVICE_0_RAM 0x80020000         0x00000000         xrw
OSPI_DEVICE_1_RAM 0x80030000         0x00000000         xrw
SDRAM            0x80010000         0x00000000         xrw
OPTION_SETTING   0x0100a100         0x00000100         r
OPTION_SETTING_S 0x0100a200         0x00000100         r
ID_CODE          0x00000000         0x00000000         xr
*default*        0x00000000         0xffffffff

Linker script and memory map

LOAD c:/renesas/ra/e2studio_v2022-10_fsp_v4.2.0/toolchains/gcc_arm/gcc-arm-none-eabi-10.3-2021.10/bin/../lib/gcc/arm-none-eabi/10.3.1/thumb/v8-m.main+fp/hard/crti.o
LOAD c:/renesas/ra/e2studio_v2022-10_fsp_v4.2.0/toolchains/gcc_arm/gcc-arm-none-eabi-10.3-2021.10/bin/../lib/gcc/arm-none-eabi/10.3.1/thumb/v8-m.main+fp/hard/crtbegin.o
LOAD c:/renesas/ra/e2studio_v2022-10_fsp_v4.2.0/toolchains/gcc_arm/gcc-arm-none-eabi-10.3-2021.10/bin/../lib/gcc/arm-none-eabi/10.3.1/../../../../arm-none-eabi/lib/thumb/v8-m.main+fp/hard/rdimon-crt0.o
START GROUP
LOAD ./src/hal_entry.o
LOAD ./src/udp_cdc.o
LOAD ./src/udp_printf.o
LOAD ./src/usb_desc.o
LOAD ./ra_gen/common_data.o
LOAD ./ra_gen/hal_data.o
LOAD ./ra_gen/main.o
LOAD ./ra_gen/pin_data.o
LOAD ./ra_gen/vector_data.o
LOAD ./ra/fsp/src/r_usb_pcdc/src/r_usb_pcdc_driver.o
LOAD ./ra/fsp/src/r_usb_basic/src/hw/r_usb_creg_abs.o
LOAD ./ra/fsp/src/r_usb_basic/src/hw/r_usb_creg_access.o
LOAD ./ra/fsp/src/r_usb_basic/src/hw/r_usb_dma.o
LOAD ./ra/fsp/src/r_usb_basic/src/hw/r_usb_hostelectrical.o
LOAD ./ra/fsp/src/r_usb_basic/src/hw/r_usb_hreg_abs.o
LOAD ./ra/fsp/src/r_usb_basic/src/hw/r_usb_hreg_access.o
LOAD ./ra/fsp/src/r_usb_basic/src/hw/r_usb_mcu.o
LOAD ./ra/fsp/src/r_usb_basic/src/hw/r_usb_preg_abs.o
LOAD ./ra/fsp/src/r_usb_basic/src/hw/r_usb_preg_access.o
LOAD ./ra/fsp/src/r_usb_basic/src/driver/r_usb_cdataio.o
LOAD ./ra/fsp/src/r_usb_basic/src/driver/r_usb_clibusbip.o
LOAD ./ra/fsp/src/r_usb_basic/src/driver/r_usb_cstd_rtos.o
LOAD ./ra/fsp/src/r_usb_basic/src/driver/r_usb_hbc.o
LOAD ./ra/fsp/src/r_usb_basic/src/driver/r_usb_hcontrolrw.o
LOAD ./ra/fsp/src/r_usb_basic/src/driver/r_usb_hdriver.o
LOAD ./ra/fsp/src/r_usb_basic/src/driver/r_usb_hhubsys.o
LOAD ./ra/fsp/src/r_usb_basic/src/driver/r_usb_hintfifo.o
LOAD ./ra/fsp/src/r_usb_basic/src/driver/r_usb_hinthandler_usbip0.o
LOAD ./ra/fsp/src/r_usb_basic/src/driver/r_usb_hinthandler_usbip1.o
LOAD ./ra/fsp/src/r_usb_basic/src/driver/r_usb_hlibusbip.o
LOAD ./ra/fsp/src/r_usb_basic/src/driver/r_usb_hmanager.o
LOAD ./ra/fsp/src/r_usb_basic/src/driver/r_usb_hscheduler.o
LOAD ./ra/fsp/src/r_usb_basic/src/driver/r_usb_hsignal.o
LOAD ./ra/fsp/src/r_usb_basic/src/driver/r_usb_hstdfunction.o
LOAD ./ra/fsp/src/r_usb_basic/src/driver/r_usb_pbc.o
LOAD ./ra/fsp/src/r_usb_basic/src/driver/r_usb_pcontrolrw.o
LOAD ./ra/fsp/src/r_usb_basic/src/driver/r_usb_pdriver.o
LOAD ./ra/fsp/src/r_usb_basic/src/driver/r_usb_pintfifo.o
LOAD ./ra/fsp/src/r_usb_basic/src/driver/r_usb_pinthandler_usbip0.o
LOAD ./ra/fsp/src/r_usb_basic/src/driver/r_usb_plibusbip.o
LOAD ./ra/fsp/src/r_usb_basic/src/driver/r_usb_psignal.o
LOAD ./ra/fsp/src/r_usb_basic/src/driver/r_usb_pstdfunction.o
LOAD ./ra/fsp/src/r_usb_basic/src/driver/r_usb_pstdrequest.o
LOAD ./ra/fsp/src/r_usb_basic/r_usb_basic.o
LOAD ./ra/fsp/src/r_rtc/r_rtc.o
LOAD ./ra/fsp/src/r_ioport/r_ioport.o
LOAD ./ra/fsp/src/r_flash_hp/r_flash_hp.o
LOAD ./ra/fsp/src/bsp/mcu/all/bsp_clocks.o
LOAD ./ra/fsp/src/bsp/mcu/all/bsp_common.o
LOAD ./ra/fsp/src/bsp/mcu/all/bsp_delay.o
LOAD ./ra/fsp/src/bsp/mcu/all/bsp_group_irq.o
LOAD ./ra/fsp/src/bsp/mcu/all/bsp_guard.o
LOAD ./ra/fsp/src/bsp/mcu/all/bsp_io.o
LOAD ./ra/fsp/src/bsp/mcu/all/bsp_irq.o
LOAD ./ra/fsp/src/bsp/mcu/all/bsp_register_protection.o
LOAD ./ra/fsp/src/bsp/mcu/all/bsp_rom_registers.o
LOAD ./ra/fsp/src/bsp/mcu/all/bsp_sbrk.o
LOAD ./ra/fsp/src/bsp/mcu/all/bsp_security.o
LOAD ./ra/fsp/src/bsp/cmsis/Device/RENESAS/Source/startup.o
LOAD ./ra/fsp/src/bsp/cmsis/Device/RENESAS/Source/system.o
END GROUP
START GROUP
LOAD c:/renesas/ra/e2studio_v2022-10_fsp_v4.2.0/toolchains/gcc_arm/gcc-arm-none-eabi-10.3-2021.10/bin/../lib/gcc/arm-none-eabi/10.3.1/thumb/v8-m.main+fp/hard\libgcc.a
LOAD c:/renesas/ra/e2studio_v2022-10_fsp_v4.2.0/toolchains/gcc_arm/gcc-arm-none-eabi-10.3-2021.10/bin/../lib/gcc/arm-none-eabi/10.3.1/../../../../arm-none-eabi/lib/thumb/v8-m.main+fp/hard\libg_nano.a
LOAD c:/renesas/ra/e2studio_v2022-10_fsp_v4.2.0/toolchains/gcc_arm/gcc-arm-none-eabi-10.3-2021.10/bin/../lib/gcc/arm-none-eabi/10.3.1/../../../../arm-none-eabi/lib/thumb/v8-m.main+fp/hard\libc_nano.a
END GROUP
START GROUP
LOAD c:/renesas/ra/e2studio_v2022-10_fsp_v4.2.0/toolchains/gcc_arm/gcc-arm-none-eabi-10.3-2021.10/bin/../lib/gcc/arm-none-eabi/10.3.1/thumb/v8-m.main+fp/hard\libgcc.a
LOAD c:/renesas/ra/e2studio_v2022-10_fsp_v4.2.0/toolchains/gcc_arm/gcc-arm-none-eabi-10.3-2021.10/bin/../lib/gcc/arm-none-eabi/10.3.1/../../../../arm-none-eabi/lib/thumb/v8-m.main+fp/hard\libc_nano.a
LOAD c:/renesas/ra/e2studio_v2022-10_fsp_v4.2.0/toolchains/gcc_arm/gcc-arm-none-eabi-10.3-2021.10/bin/../lib/gcc/arm-none-eabi/10.3.1/../../../../arm-none-eabi/lib/thumb/v8-m.main+fp/hard\librdimon_nano.a
END GROUP
START GROUP
LOAD c:/renesas/ra/e2studio_v2022-10_fsp_v4.2.0/toolchains/gcc_arm/gcc-arm-none-eabi-10.3-2021.10/bin/../lib/gcc/arm-none-eabi/10.3.1/thumb/v8-m.main+fp/hard\libgcc.a
LOAD c:/renesas/ra/e2studio_v2022-10_fsp_v4.2.0/toolchains/gcc_arm/gcc-arm-none-eabi-10.3-2021.10/bin/../lib/gcc/arm-none-eabi/10.3.1/../../../../arm-none-eabi/lib/thumb/v8-m.main+fp/hard\libc_nano.a
LOAD c:/renesas/ra/e2studio_v2022-10_fsp_v4.2.0/toolchains/gcc_arm/gcc-arm-none-eabi-10.3-2021.10/bin/../lib/gcc/arm-none-eabi/10.3.1/../../../../arm-none-eabi/lib/thumb/v8-m.main+fp/hard\librdimon_nano.a
END GROUP
LOAD c:/renesas/ra/e2studio_v2022-10_fsp_v4.2.0/toolchains/gcc_arm/gcc-arm-none-eabi-10.3-2021.10/bin/../lib/gcc/arm-none-eabi/10.3.1/thumb/v8-m.main+fp/hard/crtend.o
LOAD c:/renesas/ra/e2studio_v2022-10_fsp_v4.2.0/toolchains/gcc_arm/gcc-arm-none-eabi-10.3-2021.10/bin/../lib/gcc/arm-none-eabi/10.3.1/thumb/v8-m.main+fp/hard/crtn.o
                0x20000000                RAM_START = 0x20000000
                0x00020000                RAM_LENGTH = 0x20000
                0x00000000                FLASH_START = 0x0
                0x00080000                FLASH_LENGTH = 0x80000
                0x08000000                DATA_FLASH_START = 0x8000000
                0x00002000                DATA_FLASH_LENGTH = 0x2000
                0x0100a100                OPTION_SETTING_START = 0x100a100
                0x00000100                OPTION_SETTING_LENGTH = 0x100
                0x0100a200                OPTION_SETTING_S_START = 0x100a200
                0x00000100                OPTION_SETTING_S_LENGTH = 0x100
                0x00000000                ID_CODE_START = 0x0
                0x00000000                ID_CODE_LENGTH = 0x0
                0x80010000                SDRAM_START = 0x80010000
                0x00000000                SDRAM_LENGTH = 0x0
                0x60000000                QSPI_FLASH_START = 0x60000000
                0x04000000                QSPI_FLASH_LENGTH = 0x4000000
                0x80020000                OSPI_DEVICE_0_START = 0x80020000
                0x00000000                OSPI_DEVICE_0_LENGTH = 0x0
                0x80030000                OSPI_DEVICE_1_START = 0x80030000
                0x00000000                OSPI_DEVICE_1_LENGTH = 0x0
                0x04000000                QSPI_FLASH_PRV_LENGTH = DEFINED (QSPI_FLASH_SIZE)?ABSOLUTE (QSPI_FLASH_SIZE):ABSOLUTE (QSPI_FLASH_LENGTH)
                0x00000000                OSPI_DEVICE_0_PRV_LENGTH = DEFINED (OSPI_DEVICE_0_SIZE)?ABSOLUTE (OSPI_DEVICE_0_SIZE):ABSOLUTE (OSPI_DEVICE_0_LENGTH)
                0x00000000                OSPI_DEVICE_1_PRV_LENGTH = DEFINED (OSPI_DEVICE_1_SIZE)?ABSOLUTE (OSPI_DEVICE_1_SIZE):ABSOLUTE (OSPI_DEVICE_1_LENGTH)
                0x00000000                __RESERVE_NS_RAM = ((! (DEFINED (PROJECT_NONSECURE)) && DEFINED (RAM_NS_BUFFER_LENGTH)) && (OPTION_SETTING_S_LENGTH != 0x0))
                0x00000000                ITCM_START = DEFINED (ITCM_START)?ITCM_START:0x0
                0x00000000                ITCM_LENGTH = DEFINED (ITCM_LENGTH)?ITCM_LENGTH:0x0
                0x00000000                DTCM_START = DEFINED (DTCM_START)?DTCM_START:0x0
                0x00000000                DTCM_LENGTH = DEFINED (DTCM_LENGTH)?DTCM_LENGTH:0x0
                0x00000000                NS_OFFSET_START = DEFINED (NS_OFFSET_START)?NS_OFFSET_START:0x0
                0x00000000                NS_IMAGE_OFFSET = DEFINED (PROJECT_NONSECURE)?NS_OFFSET_START:0x0
                0x00000000                RAM_NS_BUFFER_BLOCK_LENGTH = DEFINED (RAM_NS_BUFFER_LENGTH)?ALIGN (RAM_NS_BUFFER_LENGTH, 0x2000):0x0
                0x00000000                RAM_NS_BUFFER_LENGTH = DEFINED (RAM_NS_BUFFER_LENGTH)?RAM_NS_BUFFER_LENGTH:0x0
                0x20020000                RAM_NS_BUFFER_START = ((RAM_START + RAM_LENGTH) - RAM_NS_BUFFER_LENGTH)
                0x20020000                RAM_NS_BUFFER_BLOCK_START = ((RAM_START + RAM_LENGTH) - RAM_NS_BUFFER_BLOCK_LENGTH)
                0x0100a180                OPTION_SETTING_START_NS = DEFINED (PROJECT_NONSECURE)?OPTION_SETTING_START:(OPTION_SETTING_START + 0x80)
                0x00000001                __bl_FSP_BOOTABLE_IMAGE = 0x1
                0x00000001                __bln_FSP_BOOTABLE_IMAGE = 0x1
                0x00000001                PROJECT_SECURE_OR_FLAT = (((! (DEFINED (PROJECT_NONSECURE)) || DEFINED (PROJECT_SECURE)) && OPTION_SETTING_LENGTH) && ! (DEFINED (FSP_BOOTABLE_IMAGE)))
                0x00000000                USE_OPTION_SETTING_NS = (DEFINED (PROJECT_NONSECURE) && ! (DEFINED (FSP_BOOTABLE_IMAGE)))
                0x00000000                __bl_FLASH_IMAGE_START = ! (DEFINED (FLASH_BOOTLOADER_LENGTH))?0x0:(FLASH_APPLICATION_IMAGE_NUMBER == 0x1)?(FLASH_BOOTLOADER_LENGTH + FLASH_BOOTLOADER_HEADER_LENGTH):(((FLASH_BOOTLOADER_LENGTH + FLASH_BOOTLOADER_SCRATCH_LENGTH) + FLASH_APPLICATION_S_LENGTH) + FLASH_BOOTLOADER_HEADER_LENGTH)
                0x00000000                __bl_FLASH_IMAGE_LENGTH = ! (DEFINED (FLASH_BOOTLOADER_LENGTH))?0x0:(FLASH_APPLICATION_S_LENGTH - FLASH_BOOTLOADER_HEADER_LENGTH)
                0x00000000                __bl_FLASH_IMAGE_END = (__bl_FLASH_IMAGE_START + __bl_FLASH_IMAGE_LENGTH)
                0x00000000                __bl_XIP_SECONDARY_FLASH_IMAGE_START = ! (DEFINED (FLASH_BOOTLOADER_LENGTH))?0x0:((FLASH_BOOTLOADER_LENGTH + FLASH_APPLICATION_S_LENGTH) + FLASH_BOOTLOADER_HEADER_LENGTH)
                0x00000000                __bl_XIP_SECONDARY_FLASH_IMAGE_END = (__bl_XIP_SECONDARY_FLASH_IMAGE_START + __bl_FLASH_IMAGE_LENGTH)
                0x00000000                __bl_FLASH_NS_START = ! (DEFINED (FLASH_BOOTLOADER_LENGTH))?0x0:(FLASH_APPLICATION_NS_LENGTH == 0x0)?__bl_FLASH_IMAGE_END:((__bl_FLASH_IMAGE_START - FLASH_BOOTLOADER_HEADER_LENGTH) + FLASH_APPLICATION_S_LENGTH)
                0x00000000                __bl_FLASH_NSC_START = ! (DEFINED (FLASH_BOOTLOADER_LENGTH))?0x0:(FLASH_APPLICATION_NS_LENGTH == 0x0)?__bl_FLASH_IMAGE_END:(__bl_FLASH_NS_START - FLASH_APPLICATION_NSC_LENGTH)
                0x00000000                __bl_RAM_NS_START = ! (DEFINED (FLASH_BOOTLOADER_LENGTH))?0x0:(FLASH_APPLICATION_NS_LENGTH == 0x0)?(RAM_START + RAM_LENGTH):((RAM_START + RAM_LENGTH) - RAM_APPLICATION_NS_LENGTH)
                0x00000000                __bl_RAM_NSC_START = ! (DEFINED (FLASH_BOOTLOADER_LENGTH))?0x0:(FLASH_APPLICATION_NS_LENGTH == 0x0)?(RAM_START + RAM_LENGTH):(__bl_RAM_NS_START - RAM_APPLICATION_NSC_LENGTH)
                0x00000000                __bl_FLASH_NS_IMAGE_START = ! (DEFINED (FLASH_BOOTLOADER_LENGTH))?0x0:(FLASH_APPLICATION_NS_LENGTH == 0x0)?__bl_FLASH_IMAGE_END:(__bl_FLASH_NS_START + FLASH_BOOTLOADER_HEADER_LENGTH_2)
                0x00000000                __bln_FLASH_IMAGE_START = __bl_FLASH_NS_IMAGE_START
                0x00000000                __bln_FLASH_IMAGE_LENGTH = ! (DEFINED (FLASH_BOOTLOADER_LENGTH))?0x0:(FLASH_APPLICATION_NS_LENGTH == 0x0)?__bl_FLASH_IMAGE_END:(FLASH_APPLICATION_NS_LENGTH - FLASH_BOOTLOADER_HEADER_LENGTH_2)
                0x00000000                XIP_SECONDARY_SLOT_IMAGE = DEFINED (XIP_SECONDARY_SLOT_IMAGE)?XIP_SECONDARY_SLOT_IMAGE:0x0
                0x00000000                FLASH_ORIGIN = ! (DEFINED (FLASH_IMAGE_START))?FLASH_START:(XIP_SECONDARY_SLOT_IMAGE == 0x1)?XIP_SECONDARY_FLASH_IMAGE_START:FLASH_IMAGE_START
                0x00080000                LIMITED_FLASH_LENGTH = DEFINED (FLASH_IMAGE_LENGTH)?FLASH_IMAGE_LENGTH:DEFINED (FLASH_BOOTLOADER_LENGTH)?FLASH_BOOTLOADER_LENGTH:FLASH_LENGTH
START GROUP
LOAD c:/renesas/ra/e2studio_v2022-10_fsp_v4.2.0/toolchains/gcc_arm/gcc-arm-none-eabi-10.3-2021.10/bin/../lib/gcc/arm-none-eabi/10.3.1/thumb/v8-m.main+fp/hard\libgcc.a
LOAD c:/renesas/ra/e2studio_v2022-10_fsp_v4.2.0/toolchains/gcc_arm/gcc-arm-none-eabi-10.3-2021.10/bin/../lib/gcc/arm-none-eabi/10.3.1/../../../../arm-none-eabi/lib/thumb/v8-m.main+fp/hard\libc.a
LOAD c:/renesas/ra/e2studio_v2022-10_fsp_v4.2.0/toolchains/gcc_arm/gcc-arm-none-eabi-10.3-2021.10/bin/../lib/gcc/arm-none-eabi/10.3.1/../../../../arm-none-eabi/lib/thumb/v8-m.main+fp/hard\libm.a
LOAD c:/renesas/ra/e2studio_v2022-10_fsp_v4.2.0/toolchains/gcc_arm/gcc-arm-none-eabi-10.3-2021.10/bin/../lib/gcc/arm-none-eabi/10.3.1/../../../../arm-none-eabi/lib/thumb/v8-m.main+fp/hard\libnosys.a
END GROUP

.itcm_data      0x00000000        0x0
                0x00000000                __tz_ITCM_S = ABSOLUTE (ITCM_START)
                0x00000000                __itcm_data_start__ = .
 *(.itcm_data*)
                0x00000000                __itcm_data_end__ = .
                0x00000000                __tz_ITCM_N = DEFINED (ITCM_NS_START)?ABSOLUTE (ITCM_NS_START):ALIGN (__itcm_data_end__, 0x2000)

.text           0x00000000     0x7228
                0x00000000                __tz_FLASH_S = ABSOLUTE (FLASH_START)
                0x00000000                __ROM_Start = .
 *(.fixed_vectors*)
 .fixed_vectors
                0x00000000       0x40 ./ra/fsp/src/bsp/cmsis/Device/RENESAS/Source/startup.o
                0x00000000                __Vectors
 *(.application_vectors*)
 .application_vectors
                0x00000040      0x180 ./ra_gen/vector_data.o
                0x00000040                g_vector_table
                0x000001c0                __Vectors_End = .
                0x000001c0                . = (OPTION_SETTING_LENGTH > 0x0)?.:(__ROM_Start + 0x400)
 *(.rom_registers*)
                0x000001c0                . = (OPTION_SETTING_LENGTH > 0x0)?.:(__ROM_Start + 0x500)
                0x00000200                . = ALIGN (0x80)
 *fill*         0x000001c0       0x40 ff
 *(.mcuboot_sce9_key*)
 *(.text*)
 .text          0x00000200       0x40 c:/renesas/ra/e2studio_v2022-10_fsp_v4.2.0/toolchains/gcc_arm/gcc-arm-none-eabi-10.3-2021.10/bin/../lib/gcc/arm-none-eabi/10.3.1/thumb/v8-m.main+fp/hard/crtbegin.o
 .text.wait     0x00000240       0x3c ./src/hal_entry.o
 .text.H2I.part.0
                0x0000027c       0x90 ./src/hal_entry.o
 .text.getstr.constprop.0
                0x0000030c       0x68 ./src/hal_entry.o
 .text.my_get_char.0
                0x00000374       0xbc ./src/hal_entry.o
 .text.hal_entry
                0x00000430      0x9b4 ./src/hal_entry.o
                0x00000430                hal_entry
 .text.udp_event_poll
                0x00000de4      0x168 ./src/udp_cdc.o
 .text.udp_rx_buff
                0x00000f4c       0x20 ./src/udp_cdc.o
                0x00000f4c                udp_rx_buff
 .text.udp_rx_purge
                0x00000f6c       0x10 ./src/udp_cdc.o
                0x00000f6c                udp_rx_purge
 .text.udp_putc
                0x00000f7c       0x40 ./src/udp_cdc.o
                0x00000f7c                udp_putc
 .text.udp_puts
                0x00000fbc       0x90 ./src/udp_cdc.o
                0x00000fbc                udp_puts
 .text.udp_putsb
                0x0000104c       0xc8 ./src/udp_cdc.o
                0x0000104c                udp_putsb
 .text.udp_getc
                0x00001114       0x44 ./src/udp_cdc.o
                0x00001114                udp_getc
 .text.udp_init
                0x00001158       0x3c ./src/udp_cdc.o
                0x00001158                udp_init
 .text.udp_deinit
                0x00001194       0x28 ./src/udp_cdc.o
                0x00001194                udp_deinit
 *fill*         0x000011bc        0x4 ff
 .text.udp_printf
                0x000011c0      0xad4 ./src/udp_printf.o
                0x000011c0                udp_printf
 .text.startup.main
                0x00001c94        0xc ./ra_gen/main.o
                0x00001c94                main
 .text.usb_pcdc_read_complete
                0x00001ca0       0x74 ./ra/fsp/src/r_usb_pcdc/src/r_usb_pcdc_driver.o
                0x00001ca0                usb_pcdc_read_complete
 .text.usb_pcdc_write_complete
                0x00001d14       0x5c ./ra/fsp/src/r_usb_pcdc/src/r_usb_pcdc_driver.o
                0x00001d14                usb_pcdc_write_complete
 .text.usb_cstd_get_buf_size
                0x00001d70       0x30 ./ra/fsp/src/r_usb_basic/src/hw/r_usb_creg_abs.o
                0x00001d70                usb_cstd_get_buf_size
 .text.usb_cstd_pipe_init
                0x00001da0      0x140 ./ra/fsp/src/r_usb_basic/src/hw/r_usb_creg_abs.o
                0x00001da0                usb_cstd_pipe_init
 .text.usb_cstd_clr_pipe_cnfg
                0x00001ee0       0xd0 ./ra/fsp/src/r_usb_basic/src/hw/r_usb_creg_abs.o
                0x00001ee0                usb_cstd_clr_pipe_cnfg
 .text.usb_cstd_set_nak
                0x00001fb0       0x28 ./ra/fsp/src/r_usb_basic/src/hw/r_usb_creg_abs.o
                0x00001fb0                usb_cstd_set_nak
 .text.usb_cstd_is_set_frdy
                0x00001fd8       0x5c ./ra/fsp/src/r_usb_basic/src/hw/r_usb_creg_abs.o
                0x00001fd8                usb_cstd_is_set_frdy
 .text.usb_cstd_chg_curpipe
                0x00002034       0x2c ./ra/fsp/src/r_usb_basic/src/hw/r_usb_creg_abs.o
                0x00002034                usb_cstd_chg_curpipe
 .text.usb_cstd_set_transaction_counter
                0x00002060       0x28 ./ra/fsp/src/r_usb_basic/src/hw/r_usb_creg_abs.o
                0x00002060                usb_cstd_set_transaction_counter
 .text.usb_cstd_clr_transaction_counter
                0x00002088       0x18 ./ra/fsp/src/r_usb_basic/src/hw/r_usb_creg_abs.o
                0x00002088                usb_cstd_clr_transaction_counter
 .text.hw_usb_read_syscfg
                0x000020a0       0x34 ./ra/fsp/src/r_usb_basic/src/hw/r_usb_creg_access.o
                0x000020a0                hw_usb_read_syscfg
 .text.hw_usb_read_syssts
                0x000020d4       0x34 ./ra/fsp/src/r_usb_basic/src/hw/r_usb_creg_access.o
                0x000020d4                hw_usb_read_syssts
 .text.hw_usb_read_dvstctr
                0x00002108       0x34 ./ra/fsp/src/r_usb_basic/src/hw/r_usb_creg_access.o
                0x00002108                hw_usb_read_dvstctr
 .text.hw_usb_read_fifo16
                0x0000213c       0x34 ./ra/fsp/src/r_usb_basic/src/hw/r_usb_creg_access.o
                0x0000213c                hw_usb_read_fifo16
 .text.hw_usb_write_fifo16
                0x00002170       0x5c ./ra/fsp/src/r_usb_basic/src/hw/r_usb_creg_access.o
                0x00002170                hw_usb_write_fifo16
 .text.hw_usb_write_fifo8
                0x000021cc       0x5c ./ra/fsp/src/r_usb_basic/src/hw/r_usb_creg_access.o
                0x000021cc                hw_usb_write_fifo8
 .text.hw_usb_read_fifosel
                0x00002228       0x6c ./ra/fsp/src/r_usb_basic/src/hw/r_usb_creg_access.o
                0x00002228                hw_usb_read_fifosel
 .text.hw_usb_rmw_fifosel
                0x00002294       0x84 ./ra/fsp/src/r_usb_basic/src/hw/r_usb_creg_access.o
                0x00002294                hw_usb_rmw_fifosel
 .text.hw_usb_set_mbw
                0x00002318       0x8c ./ra/fsp/src/r_usb_basic/src/hw/r_usb_creg_access.o
                0x00002318                hw_usb_set_mbw
 .text.hw_usb_read_fifoctr
                0x000023a4       0x6c ./ra/fsp/src/r_usb_basic/src/hw/r_usb_creg_access.o
                0x000023a4                hw_usb_read_fifoctr
 .text.hw_usb_set_bval
                0x00002410       0x70 ./ra/fsp/src/r_usb_basic/src/hw/r_usb_creg_access.o
                0x00002410                hw_usb_set_bval
 .text.hw_usb_set_bclr
                0x00002480       0x74 ./ra/fsp/src/r_usb_basic/src/hw/r_usb_creg_access.o
                0x00002480                hw_usb_set_bclr
 .text.hw_usb_set_brdyenb
                0x000024f4       0x38 ./ra/fsp/src/r_usb_basic/src/hw/r_usb_creg_access.o
                0x000024f4                hw_usb_set_brdyenb
 .text.hw_usb_clear_brdyenb
                0x0000252c       0x3c ./ra/fsp/src/r_usb_basic/src/hw/r_usb_creg_access.o
                0x0000252c                hw_usb_clear_brdyenb
 .text.hw_usb_set_nrdyenb
                0x00002568       0x38 ./ra/fsp/src/r_usb_basic/src/hw/r_usb_creg_access.o
                0x00002568                hw_usb_set_nrdyenb
 .text.hw_usb_clear_nrdyenb
                0x000025a0       0x3c ./ra/fsp/src/r_usb_basic/src/hw/r_usb_creg_access.o
                0x000025a0                hw_usb_clear_nrdyenb
 .text.hw_usb_set_bempenb
                0x000025dc       0x60 ./ra/fsp/src/r_usb_basic/src/hw/r_usb_creg_access.o
                0x000025dc                hw_usb_set_bempenb
 .text.hw_usb_clear_bempenb
                0x0000263c       0x3c ./ra/fsp/src/r_usb_basic/src/hw/r_usb_creg_access.o
                0x0000263c                hw_usb_clear_bempenb
 .text.hw_usb_read_intsts
                0x00002678       0x20 ./ra/fsp/src/r_usb_basic/src/hw/r_usb_creg_access.o
                0x00002678                hw_usb_read_intsts
 .text.hw_usb_clear_sts_brdy
                0x00002698       0x48 ./ra/fsp/src/r_usb_basic/src/hw/r_usb_creg_access.o
                0x00002698                hw_usb_clear_sts_brdy
 .text.hw_usb_clear_status_nrdy
                0x000026e0       0x48 ./ra/fsp/src/r_usb_basic/src/hw/r_usb_creg_access.o
                0x000026e0                hw_usb_clear_status_nrdy
 .text.hw_usb_clear_status_bemp
                0x00002728       0x48 ./ra/fsp/src/r_usb_basic/src/hw/r_usb_creg_access.o
                0x00002728                hw_usb_clear_status_bemp
 .text.hw_usb_read_frmnum
                0x00002770       0x38 ./ra/fsp/src/r_usb_basic/src/hw/r_usb_creg_access.o
                0x00002770                hw_usb_read_frmnum
 .text.hw_usb_read_usbreq
                0x000027a8       0x20 ./ra/fsp/src/r_usb_basic/src/hw/r_usb_creg_access.o
                0x000027a8                hw_usb_read_usbreq
 .text.hw_usb_read_usbval
                0x000027c8       0x20 ./ra/fsp/src/r_usb_basic/src/hw/r_usb_creg_access.o
                0x000027c8                hw_usb_read_usbval
 .text.hw_usb_read_usbindx
                0x000027e8       0x20 ./ra/fsp/src/r_usb_basic/src/hw/r_usb_creg_access.o
                0x000027e8                hw_usb_read_usbindx
 .text.hw_usb_read_usbleng
                0x00002808       0x20 ./ra/fsp/src/r_usb_basic/src/hw/r_usb_creg_access.o
                0x00002808                hw_usb_read_usbleng
 .text.hw_usb_read_dcpcfg
                0x00002828       0x38 ./ra/fsp/src/r_usb_basic/src/hw/r_usb_creg_access.o
                0x00002828                hw_usb_read_dcpcfg
 .text.hw_usb_write_dcpcfg
                0x00002860       0x30 ./ra/fsp/src/r_usb_basic/src/hw/r_usb_creg_access.o
                0x00002860                hw_usb_write_dcpcfg
 .text.hw_usb_read_dcpmaxp
                0x00002890       0x38 ./ra/fsp/src/r_usb_basic/src/hw/r_usb_creg_access.o
                0x00002890                hw_usb_read_dcpmaxp
 .text.hw_usb_write_dcpmxps
                0x000028c8       0x30 ./ra/fsp/src/r_usb_basic/src/hw/r_usb_creg_access.o
                0x000028c8                hw_usb_write_dcpmxps
 .text.hw_usb_read_dcpctr
                0x000028f8       0x20 ./ra/fsp/src/r_usb_basic/src/hw/r_usb_creg_access.o
                0x000028f8                hw_usb_read_dcpctr
 .text.hw_usb_write_pipesel
                0x00002918       0x30 ./ra/fsp/src/r_usb_basic/src/hw/r_usb_creg_access.o
                0x00002918                hw_usb_write_pipesel
 .text.hw_usb_read_pipecfg
                0x00002948       0x38 ./ra/fsp/src/r_usb_basic/src/hw/r_usb_creg_access.o
                0x00002948                hw_usb_read_pipecfg
 .text.hw_usb_write_pipecfg
                0x00002980       0x30 ./ra/fsp/src/r_usb_basic/src/hw/r_usb_creg_access.o
                0x00002980                hw_usb_write_pipecfg
 .text.hw_usb_read_pipemaxp
                0x000029b0       0x38 ./ra/fsp/src/r_usb_basic/src/hw/r_usb_creg_access.o
                0x000029b0                hw_usb_read_pipemaxp
 .text.hw_usb_write_pipemaxp
                0x000029e8       0x30 ./ra/fsp/src/r_usb_basic/src/hw/r_usb_creg_access.o
                0x000029e8                hw_usb_write_pipemaxp
 .text.hw_usb_write_pipeperi
                0x00002a18       0x30 ./ra/fsp/src/r_usb_basic/src/hw/r_usb_creg_access.o
                0x00002a18                hw_usb_write_pipeperi
 .text.hw_usb_read_pipectr
                0x00002a48       0x68 ./ra/fsp/src/r_usb_basic/src/hw/r_usb_creg_access.o
                0x00002a48                hw_usb_read_pipectr
 .text.hw_usb_set_csclr
                0x00002ab0       0x3c ./ra/fsp/src/r_usb_basic/src/hw/r_usb_creg_access.o
                0x00002ab0                hw_usb_set_csclr
 .text.hw_usb_set_aclrm
                0x00002aec       0x44 ./ra/fsp/src/r_usb_basic/src/hw/r_usb_creg_access.o
                0x00002aec                hw_usb_set_aclrm
 .text.hw_usb_clear_aclrm
                0x00002b30       0x3c ./ra/fsp/src/r_usb_basic/src/hw/r_usb_creg_access.o
                0x00002b30                hw_usb_clear_aclrm
 .text.hw_usb_set_sqclr
                0x00002b6c       0x74 ./ra/fsp/src/r_usb_basic/src/hw/r_usb_creg_access.o
                0x00002b6c                hw_usb_set_sqclr
 .text.hw_usb_set_pid
                0x00002be0       0x58 ./ra/fsp/src/r_usb_basic/src/hw/r_usb_creg_access.o
                0x00002be0                hw_usb_set_pid
 .text.hw_usb_clear_pid
                0x00002c38       0x50 ./ra/fsp/src/r_usb_basic/src/hw/r_usb_creg_access.o
                0x00002c38                hw_usb_clear_pid
 .text.hw_usb_set_trenb
                0x00002c88       0x3c ./ra/fsp/src/r_usb_basic/src/hw/r_usb_creg_access.o
                0x00002c88                hw_usb_set_trenb
 .text.hw_usb_clear_trenb
                0x00002cc4       0x3c ./ra/fsp/src/r_usb_basic/src/hw/r_usb_creg_access.o
                0x00002cc4                hw_usb_clear_trenb
 .text.hw_usb_set_trclr
                0x00002d00       0x3c ./ra/fsp/src/r_usb_basic/src/hw/r_usb_creg_access.o
                0x00002d00                hw_usb_set_trclr
 .text.hw_usb_write_pipetrn
                0x00002d3c       0x34 ./ra/fsp/src/r_usb_basic/src/hw/r_usb_creg_access.o
                0x00002d3c                hw_usb_write_pipetrn
 .text.hw_usb_set_suspendm
                0x00002d70        0x4 ./ra/fsp/src/r_usb_basic/src/hw/r_usb_creg_access.o
                0x00002d70                hw_usb_set_suspendm
 .text.hw_usb_clear_suspm
                0x00002d74        0x4 ./ra/fsp/src/r_usb_basic/src/hw/r_usb_creg_access.o
                0x00002d74                hw_usb_clear_suspm
 .text.usb_module_start
                0x00002d78       0x50 ./ra/fsp/src/r_usb_basic/src/hw/r_usb_mcu.o
                0x00002d78                usb_module_start
 .text.usb_module_register_clear
                0x00002dc8      0x100 ./ra/fsp/src/r_usb_basic/src/hw/r_usb_mcu.o
                0x00002dc8                usb_module_register_clear
 .text.usb_module_stop
                0x00002ec8       0x54 ./ra/fsp/src/r_usb_basic/src/hw/r_usb_mcu.o
                0x00002ec8                usb_module_stop
 .text.usb_cpu_usbint_init
                0x00002f1c       0xc0 ./ra/fsp/src/r_usb_basic/src/hw/r_usb_mcu.o
                0x00002f1c                usb_cpu_usbint_init
 .text.usb_cpu_delay_1us
                0x00002fdc        0x8 ./ra/fsp/src/r_usb_basic/src/hw/r_usb_mcu.o
                0x00002fdc                usb_cpu_delay_1us
 .text.usb_cpu_delay_xms
                0x00002fe4        0x8 ./ra/fsp/src/r_usb_basic/src/hw/r_usb_mcu.o
                0x00002fe4                usb_cpu_delay_xms
 .text.usbfs_interrupt_handler
                0x00002fec       0x34 ./ra/fsp/src/r_usb_basic/src/hw/r_usb_mcu.o
                0x00002fec                usbfs_interrupt_handler
 .text.usbfs_resume_handler
                0x00003020       0x34 ./ra/fsp/src/r_usb_basic/src/hw/r_usb_mcu.o
                0x00003020                usbfs_resume_handler
 .text.usbfs_d0fifo_handler
                0x00003054       0x24 ./ra/fsp/src/r_usb_basic/src/hw/r_usb_mcu.o
                0x00003054                usbfs_d0fifo_handler
 .text.usbfs_d1fifo_handler
                0x00003078       0x24 ./ra/fsp/src/r_usb_basic/src/hw/r_usb_mcu.o
                0x00003078                usbfs_d1fifo_handler
 .text.usb_pstd_interrupt_handler
                0x0000309c      0x1f4 ./ra/fsp/src/r_usb_basic/src/hw/r_usb_preg_abs.o
                0x0000309c                usb_pstd_interrupt_handler
 .text.usb_pstd_save_request
                0x00003290       0x48 ./ra/fsp/src/r_usb_basic/src/hw/r_usb_preg_abs.o
                0x00003290                usb_pstd_save_request
 .text.usb_pstd_chk_configured
                0x000032d8       0x1c ./ra/fsp/src/r_usb_basic/src/hw/r_usb_preg_abs.o
                0x000032d8                usb_pstd_chk_configured
 .text.usb_pstd_test_mode
                0x000032f4        0x4 ./ra/fsp/src/r_usb_basic/src/hw/r_usb_preg_abs.o
                0x000032f4                usb_pstd_test_mode
 .text.usb_pstd_resume_process
                0x000032f8       0x18 ./ra/fsp/src/r_usb_basic/src/hw/r_usb_preg_abs.o
                0x000032f8                usb_pstd_resume_process
 .text.usb_pstd_set_stall
                0x00003310        0xc ./ra/fsp/src/r_usb_basic/src/hw/r_usb_preg_abs.o
                0x00003310                usb_pstd_set_stall
 .text.usb_pstd_set_stall_pipe0
                0x0000331c        0x8 ./ra/fsp/src/r_usb_basic/src/hw/r_usb_preg_abs.o
                0x0000331c                usb_pstd_set_stall_pipe0
 .text.usb_pstd_write_fifo
                0x00003324       0x5c ./ra/fsp/src/r_usb_basic/src/hw/r_usb_preg_abs.o
                0x00003324                usb_pstd_write_fifo
 .text.usb_pstd_read_fifo
                0x00003380       0x44 ./ra/fsp/src/r_usb_basic/src/hw/r_usb_preg_abs.o
                0x00003380                usb_pstd_read_fifo
 .text.usb_pstd_forced_termination
                0x000033c4       0xa0 ./ra/fsp/src/r_usb_basic/src/hw/r_usb_preg_abs.o
                0x000033c4                usb_pstd_forced_termination
 .text.usb_pstd_interrupt_clock
                0x00003464       0x20 ./ra/fsp/src/r_usb_basic/src/hw/r_usb_preg_abs.o
                0x00003464                usb_pstd_interrupt_clock
 .text.usb_pstd_stop_clock
                0x00003484       0x10 ./ra/fsp/src/r_usb_basic/src/hw/r_usb_preg_abs.o
                0x00003484                usb_pstd_stop_clock
 .text.hw_usb_pset_dprpu
                0x00003494       0x28 ./ra/fsp/src/r_usb_basic/src/hw/r_usb_preg_access.o
                0x00003494                hw_usb_pset_dprpu
 .text.hw_usb_pclear_dprpu
                0x000034bc       0x20 ./ra/fsp/src/r_usb_basic/src/hw/r_usb_preg_access.o
                0x000034bc                hw_usb_pclear_dprpu
 .text.hw_usb_pset_enb_rsme
                0x000034dc       0x28 ./ra/fsp/src/r_usb_basic/src/hw/r_usb_preg_access.o
                0x000034dc                hw_usb_pset_enb_rsme
 .text.hw_usb_pclear_enb_rsme
                0x00003504       0x20 ./ra/fsp/src/r_usb_basic/src/hw/r_usb_preg_access.o
                0x00003504                hw_usb_pclear_enb_rsme
 .text.hw_usb_pclear_sts_resm
                0x00003524       0x20 ./ra/fsp/src/r_usb_basic/src/hw/r_usb_preg_access.o
                0x00003524                hw_usb_pclear_sts_resm
 .text.hw_usb_pclear_sts_valid
                0x00003544       0x20 ./ra/fsp/src/r_usb_basic/src/hw/r_usb_preg_access.o
                0x00003544                hw_usb_pclear_sts_valid
 .text.hw_usb_pset_ccpl
                0x00003564       0x30 ./ra/fsp/src/r_usb_basic/src/hw/r_usb_preg_access.o
                0x00003564                hw_usb_pset_ccpl
 .text.hw_usb_pmodule_init
                0x00003594       0x40 ./ra/fsp/src/r_usb_basic/src/hw/r_usb_preg_access.o
                0x00003594                hw_usb_pmodule_init
 .text.hw_usb_pcontrol_dcpctr_pid
                0x000035d4       0x3c ./ra/fsp/src/r_usb_basic/src/hw/r_usb_preg_access.o
                0x000035d4                hw_usb_pcontrol_dcpctr_pid
 .text.usb_ctrl_read
                0x00003610       0x50 ./ra/fsp/src/r_usb_basic/src/driver/r_usb_cdataio.o
                0x00003610                usb_ctrl_read
 .text.usb_ctrl_write
                0x00003660       0x90 ./ra/fsp/src/r_usb_basic/src/driver/r_usb_cdataio.o
                0x00003660                usb_ctrl_write
 .text.usb_data_read
                0x000036f0       0x54 ./ra/fsp/src/r_usb_basic/src/driver/r_usb_cdataio.o
                0x000036f0                usb_data_read
 .text.usb_data_write
                0x00003744       0x98 ./ra/fsp/src/r_usb_basic/src/driver/r_usb_cdataio.o
                0x00003744                usb_data_write
 .text.usb_data_stop
                0x000037dc       0x30 ./ra/fsp/src/r_usb_basic/src/driver/r_usb_cdataio.o
                0x000037dc                usb_data_stop
 .text.usb_cstd_nrdy_enable
                0x0000380c        0xc ./ra/fsp/src/r_usb_basic/src/driver/r_usb_clibusbip.o
                0x0000380c                usb_cstd_nrdy_enable
 .text.usb_cstd_get_pid
                0x00003818       0x14 ./ra/fsp/src/r_usb_basic/src/driver/r_usb_clibusbip.o
                0x00003818                usb_cstd_get_pid
 .text.usb_cstd_get_maxpacket_size
                0x0000382c       0x28 ./ra/fsp/src/r_usb_basic/src/driver/r_usb_clibusbip.o
                0x0000382c                usb_cstd_get_maxpacket_size
 .text.usb_cstd_get_pipe_dir
                0x00003854       0x1c ./ra/fsp/src/r_usb_basic/src/driver/r_usb_clibusbip.o
                0x00003854                usb_cstd_get_pipe_dir
 .text.usb_cstd_get_pipe_type
                0x00003870       0x1c ./ra/fsp/src/r_usb_basic/src/driver/r_usb_clibusbip.o
                0x00003870                usb_cstd_get_pipe_type
 .text.usb_cstd_do_aclrm
                0x0000388c       0x1c ./ra/fsp/src/r_usb_basic/src/driver/r_usb_clibusbip.o
                0x0000388c                usb_cstd_do_aclrm
 .text.usb_cstd_set_buf
                0x000038a8        0xc ./ra/fsp/src/r_usb_basic/src/driver/r_usb_clibusbip.o
                0x000038a8                usb_cstd_set_buf
 .text.usb_cstd_clr_stall
                0x000038b4       0x20 ./ra/fsp/src/r_usb_basic/src/driver/r_usb_clibusbip.o
                0x000038b4                usb_cstd_clr_stall
 .text.usb_cstd_port_speed
                0x000038d4       0x20 ./ra/fsp/src/r_usb_basic/src/driver/r_usb_clibusbip.o
                0x000038d4                usb_cstd_port_speed
 .text.usb_set_event
                0x000038f4       0x44 ./ra/fsp/src/r_usb_basic/src/driver/r_usb_clibusbip.o
                0x000038f4                usb_set_event
 .text.usb_cstd_usb_task
                0x00003938        0x4 ./ra/fsp/src/r_usb_basic/src/driver/r_usb_clibusbip.o
                0x00003938                usb_cstd_usb_task
 .text.usb_pstd_ctrl_read
                0x0000393c       0x88 ./ra/fsp/src/r_usb_basic/src/driver/r_usb_pcontrolrw.o
                0x0000393c                usb_pstd_ctrl_read
 .text.usb_pstd_ctrl_write
                0x000039c4       0x50 ./ra/fsp/src/r_usb_basic/src/driver/r_usb_pcontrolrw.o
                0x000039c4                usb_pstd_ctrl_write
 .text.usb_pstd_ctrl_end
                0x00003a14       0x74 ./ra/fsp/src/r_usb_basic/src/driver/r_usb_pcontrolrw.o
                0x00003a14                usb_pstd_ctrl_end
 .text.usb_pstd_dummy_function
                0x00003a88        0x4 ./ra/fsp/src/r_usb_basic/src/driver/r_usb_pdriver.o
                0x00003a88                usb_pstd_dummy_function
 .text.usb_pstd_dummy_trn
                0x00003a8c        0x4 ./ra/fsp/src/r_usb_basic/src/driver/r_usb_pdriver.o
                0x00003a8c                usb_pstd_dummy_trn
 .text.usb_peri_configured
                0x00003a90       0x2c ./ra/fsp/src/r_usb_basic/src/driver/r_usb_pdriver.o
                0x00003a90                usb_peri_configured
 .text.usb_peri_suspended
                0x00003abc       0x1c ./ra/fsp/src/r_usb_basic/src/driver/r_usb_pdriver.o
                0x00003abc                usb_peri_suspended
 .text.usb_peri_resume
                0x00003ad8       0x1c ./ra/fsp/src/r_usb_basic/src/driver/r_usb_pdriver.o
                0x00003ad8                usb_peri_resume
 .text.usb_peri_interface
                0x00003af4        0x4 ./ra/fsp/src/r_usb_basic/src/driver/r_usb_pdriver.o
                0x00003af4                usb_peri_interface
 .text.usb_peri_detach
                0x00003af8       0x2c ./ra/fsp/src/r_usb_basic/src/driver/r_usb_pdriver.o
                0x00003af8                usb_peri_detach
 .text.usb_pstd_pcd_task
                0x00003b24      0x200 ./ra/fsp/src/r_usb_basic/src/driver/r_usb_pdriver.o
                0x00003b24                usb_pstd_pcd_task
 .text.usb_pstd_set_submitutr
                0x00003d24       0x44 ./ra/fsp/src/r_usb_basic/src/driver/r_usb_pdriver.o
                0x00003d24                usb_pstd_set_submitutr
 .text.usb_pstd_clr_mem
                0x00003d68       0x28 ./ra/fsp/src/r_usb_basic/src/driver/r_usb_pdriver.o
                0x00003d68                usb_pstd_clr_mem
 .text.usb_pstd_set_config_num
                0x00003d90       0x1c ./ra/fsp/src/r_usb_basic/src/driver/r_usb_pdriver.o
                0x00003d90                usb_pstd_set_config_num
 .text.usb_pstd_clr_eptbl_index
                0x00003dac       0x18 ./ra/fsp/src/r_usb_basic/src/driver/r_usb_pdriver.o
                0x00003dac                usb_pstd_clr_eptbl_index
 .text.usb_pstd_get_interface_num
                0x00003dc4        0xc ./ra/fsp/src/r_usb_basic/src/driver/r_usb_pdriver.o
                0x00003dc4                usb_pstd_get_interface_num
 .text.usb_pstd_get_alternate_num
                0x00003dd0       0x54 ./ra/fsp/src/r_usb_basic/src/driver/r_usb_pdriver.o
                0x00003dd0                usb_pstd_get_alternate_num
 .text.usb_pstd_set_eptbl_index
                0x00003e24       0xa0 ./ra/fsp/src/r_usb_basic/src/driver/r_usb_pdriver.o
                0x00003e24                usb_pstd_set_eptbl_index
 .text.usb_pstd_chk_remote
                0x00003ec4       0x1c ./ra/fsp/src/r_usb_basic/src/driver/r_usb_pdriver.o
                0x00003ec4                usb_pstd_chk_remote
 .text.usb_pstd_get_current_power
                0x00003ee0       0x10 ./ra/fsp/src/r_usb_basic/src/driver/r_usb_pdriver.o
                0x00003ee0                usb_pstd_get_current_power
 .text.usb_pstd_fifo_to_buf
                0x00003ef0       0x70 ./ra/fsp/src/r_usb_basic/src/driver/r_usb_pdriver.o
                0x00003ef0                usb_pstd_fifo_to_buf
 .text.usb_pstd_buf_to_fifo
                0x00003f60       0x70 ./ra/fsp/src/r_usb_basic/src/driver/r_usb_pdriver.o
                0x00003f60                usb_pstd_buf_to_fifo
 .text.usb_pstd_transfer_start
                0x00003fd0       0x40 ./ra/fsp/src/r_usb_basic/src/driver/r_usb_pdriver.o
                0x00003fd0                usb_pstd_transfer_start
 .text.usb_pstd_transfer_end
                0x00004010       0x2c ./ra/fsp/src/r_usb_basic/src/driver/r_usb_pdriver.o
                0x00004010                usb_pstd_transfer_end
 .text.usb_pstd_driver_release
                0x0000403c       0x30 ./ra/fsp/src/r_usb_basic/src/driver/r_usb_pdriver.o
                0x0000403c                usb_pstd_driver_release
 .text.usb_peri_registration
                0x0000406c       0x68 ./ra/fsp/src/r_usb_basic/src/driver/r_usb_pdriver.o
                0x0000406c                usb_peri_registration
 .text.usb_peri_pipe_info
                0x000040d4       0x6c ./ra/fsp/src/r_usb_basic/src/driver/r_usb_pdriver.o
                0x000040d4                usb_peri_pipe_info
 .text.usb_peri_devdefault
                0x00004140       0xa8 ./ra/fsp/src/r_usb_basic/src/driver/r_usb_pdriver.o
                0x00004140                usb_peri_devdefault
 .text.usb_pstd_brdy_pipe
                0x000041e8       0x60 ./ra/fsp/src/r_usb_basic/src/driver/r_usb_pintfifo.o
                0x000041e8                usb_pstd_brdy_pipe
 .text.usb_pstd_nrdy_pipe
                0x00004248        0xc ./ra/fsp/src/r_usb_basic/src/driver/r_usb_pintfifo.o
                0x00004248                usb_pstd_nrdy_pipe
 .text.usb_pstd_bemp_pipe
                0x00004254       0x48 ./ra/fsp/src/r_usb_basic/src/driver/r_usb_pintfifo.o
                0x00004254                usb_pstd_bemp_pipe
 .text.usb_pstd_usb_handler
                0x0000429c       0x5c ./ra/fsp/src/r_usb_basic/src/driver/r_usb_pinthandler_usbip0.o
                0x0000429c                usb_pstd_usb_handler
 .text.usb_pstd_data_end.part.0
                0x000042f8       0x74 ./ra/fsp/src/r_usb_basic/src/driver/r_usb_plibusbip.o
 .text.usb_pstd_epadr2pipe
                0x0000436c       0x50 ./ra/fsp/src/r_usb_basic/src/driver/r_usb_plibusbip.o
                0x0000436c                usb_pstd_epadr2pipe
 .text.usb_pstd_pipe2fport
                0x000043bc        0x4 ./ra/fsp/src/r_usb_basic/src/driver/r_usb_plibusbip.o
                0x000043bc                usb_pstd_pipe2fport
 .text.usb_pstd_hi_speed_enable
                0x000043c0        0xc ./ra/fsp/src/r_usb_basic/src/driver/r_usb_plibusbip.o
                0x000043c0                usb_pstd_hi_speed_enable
 .text.usb_pstd_send_start
                0x000043cc       0x5c ./ra/fsp/src/r_usb_basic/src/driver/r_usb_plibusbip.o
                0x000043cc                usb_pstd_send_start
 .text.usb_pstd_write_data
                0x00004428      0x118 ./ra/fsp/src/r_usb_basic/src/driver/r_usb_plibusbip.o
                0x00004428                usb_pstd_write_data
 .text.usb_pstd_receive_start
                0x00004540       0x80 ./ra/fsp/src/r_usb_basic/src/driver/r_usb_plibusbip.o
                0x00004540                usb_pstd_receive_start
 .text.usb_pstd_read_data
                0x000045c0       0xf0 ./ra/fsp/src/r_usb_basic/src/driver/r_usb_plibusbip.o
                0x000045c0                usb_pstd_read_data
 .text.usb_pstd_data_end
                0x000046b0        0xc ./ra/fsp/src/r_usb_basic/src/driver/r_usb_plibusbip.o
                0x000046b0                usb_pstd_data_end
 .text.usb_pstd_brdy_pipe_process
                0x000046bc       0x64 ./ra/fsp/src/r_usb_basic/src/driver/r_usb_plibusbip.o
                0x000046bc                usb_pstd_brdy_pipe_process
 .text.usb_pstd_nrdy_pipe_process
                0x00004720       0x58 ./ra/fsp/src/r_usb_basic/src/driver/r_usb_plibusbip.o
                0x00004720                usb_pstd_nrdy_pipe_process
 .text.usb_pstd_bemp_pipe_process
                0x00004778       0xe0 ./ra/fsp/src/r_usb_basic/src/driver/r_usb_plibusbip.o
                0x00004778                usb_pstd_bemp_pipe_process
 .text.usb_pstd_set_pipe_table
                0x00004858       0xd0 ./ra/fsp/src/r_usb_basic/src/driver/r_usb_plibusbip.o
                0x00004858                usb_pstd_set_pipe_table
 .text.usb_pstd_clr_pipe_table
                0x00004928       0x34 ./ra/fsp/src/r_usb_basic/src/driver/r_usb_plibusbip.o
                0x00004928                usb_pstd_clr_pipe_table
 .text.usb_pstd_set_pipe_reg
                0x0000495c       0xa0 ./ra/fsp/src/r_usb_basic/src/driver/r_usb_plibusbip.o
                0x0000495c                usb_pstd_set_pipe_reg
 .text.usb_pstd_clr_pipe_reg
                0x000049fc       0x3c ./ra/fsp/src/r_usb_basic/src/driver/r_usb_plibusbip.o
                0x000049fc                usb_pstd_clr_pipe_reg
 .text.usb_pstd_bus_reset
                0x00004a38       0x3c ./ra/fsp/src/r_usb_basic/src/driver/r_usb_psignal.o
                0x00004a38                usb_pstd_bus_reset
 .text.usb_pstd_attach_process
                0x00004a74       0x18 ./ra/fsp/src/r_usb_basic/src/driver/r_usb_psignal.o
                0x00004a74                usb_pstd_attach_process
 .text.usb_pstd_detach_process
                0x00004a8c       0x84 ./ra/fsp/src/r_usb_basic/src/driver/r_usb_psignal.o
                0x00004a8c                usb_pstd_detach_process
 .text.usb_pstd_suspend_process
                0x00004b10       0x68 ./ra/fsp/src/r_usb_basic/src/driver/r_usb_psignal.o
                0x00004b10                usb_pstd_suspend_process
 .text.usb_pstd_set_feature_function
                0x00004b78        0x4 ./ra/fsp/src/r_usb_basic/src/driver/r_usb_pstdfunction.o
                0x00004b78                usb_pstd_set_feature_function
 .text.usb_pstd_chk_vbsts
                0x00004b7c       0x40 ./ra/fsp/src/r_usb_basic/src/driver/r_usb_pstdfunction.o
                0x00004b7c                usb_pstd_chk_vbsts
 .text.usb_pstd_busreset_function
                0x00004bbc        0x4 ./ra/fsp/src/r_usb_basic/src/driver/r_usb_pstdfunction.o
                0x00004bbc                usb_pstd_busreset_function
 .text.usb_pstd_suspend_function
                0x00004bc0        0x4 ./ra/fsp/src/r_usb_basic/src/driver/r_usb_pstdfunction.o
                0x00004bc0                usb_pstd_suspend_function
 .text.usb_pdriver_init
                0x00004bc4       0xf8 ./ra/fsp/src/r_usb_basic/src/driver/r_usb_pstdfunction.o
                0x00004bc4                usb_pdriver_init
 .text.usb_pstd_stand_req0
                0x00004cbc       0x80 ./ra/fsp/src/r_usb_basic/src/driver/r_usb_pstdrequest.o
                0x00004cbc                usb_pstd_stand_req0
 .text.usb_pstd_stand_req1
                0x00004d3c      0x29c ./ra/fsp/src/r_usb_basic/src/driver/r_usb_pstdrequest.o
                0x00004d3c                usb_pstd_stand_req1
 .text.usb_pstd_stand_req2
                0x00004fd8        0x4 ./ra/fsp/src/r_usb_basic/src/driver/r_usb_pstdrequest.o
                0x00004fd8                usb_pstd_stand_req2
 .text.usb_pstd_stand_req3
                0x00004fdc      0x330 ./ra/fsp/src/r_usb_basic/src/driver/r_usb_pstdrequest.o
                0x00004fdc                usb_pstd_stand_req3
 .text.usb_pstd_stand_req4
                0x0000530c       0xb4 ./ra/fsp/src/r_usb_basic/src/driver/r_usb_pstdrequest.o
                0x0000530c                usb_pstd_stand_req4
 .text.usb_pstd_stand_req5
                0x000053c0       0x98 ./ra/fsp/src/r_usb_basic/src/driver/r_usb_pstdrequest.o
                0x000053c0                usb_pstd_stand_req5
 .text.usb_peri_class_request_rss
                0x00005458       0x4c ./ra/fsp/src/r_usb_basic/src/driver/r_usb_pstdrequest.o
                0x00005458                usb_peri_class_request_rss
 .text.usb_peri_class_request_wss
                0x000054a4       0x58 ./ra/fsp/src/r_usb_basic/src/driver/r_usb_pstdrequest.o
                0x000054a4                usb_peri_class_request_wss
 .text.usb_peri_class_request
                0x000054fc       0xf0 ./ra/fsp/src/r_usb_basic/src/driver/r_usb_pstdrequest.o
                0x000054fc                usb_peri_class_request
 .text.R_USB_EventGet
                0x000055ec       0x58 ./ra/fsp/src/r_usb_basic/r_usb_basic.o
                0x000055ec                R_USB_EventGet
 .text.R_USB_Open
                0x00005644      0x180 ./ra/fsp/src/r_usb_basic/r_usb_basic.o
                0x00005644                R_USB_Open
 .text.R_USB_Close
                0x000057c4       0x78 ./ra/fsp/src/r_usb_basic/r_usb_basic.o
                0x000057c4                R_USB_Close
 .text.R_USB_InfoGet.part.0
                0x0000583c       0xd0 ./ra/fsp/src/r_usb_basic/r_usb_basic.o
 .text.R_USB_Read
                0x0000590c       0xa4 ./ra/fsp/src/r_usb_basic/r_usb_basic.o
                0x0000590c                R_USB_Read
 .text.R_USB_Write
                0x000059b0       0xac ./ra/fsp/src/r_usb_basic/r_usb_basic.o
                0x000059b0                R_USB_Write
 .text.R_USB_Stop
                0x00005a5c       0x9c ./ra/fsp/src/r_usb_basic/r_usb_basic.o
                0x00005a5c                R_USB_Stop
 .text.R_USB_PeriControlDataGet
                0x00005af8       0x4c ./ra/fsp/src/r_usb_basic/r_usb_basic.o
                0x00005af8                R_USB_PeriControlDataGet
 .text.R_USB_PeriControlDataSet
                0x00005b44       0x4c ./ra/fsp/src/r_usb_basic/r_usb_basic.o
                0x00005b44                R_USB_PeriControlDataSet
 .text.R_USB_PeriControlStatusSet
                0x00005b90       0x40 ./ra/fsp/src/r_usb_basic/r_usb_basic.o
                0x00005b90                R_USB_PeriControlStatusSet
 .text.rtc_carry_isr
                0x00005bd0       0x30 ./ra/fsp/src/r_rtc/r_rtc.o
                0x00005bd0                rtc_carry_isr
 .text.R_IOPORT_Close
                0x00005c00       0x20 ./ra/fsp/src/r_ioport/r_ioport.o
                0x00005c00                R_IOPORT_Close
 .text.bsp_vbatt_init
                0x00005c20       0xac ./ra/fsp/src/r_ioport/r_ioport.o
 .text.r_ioport_pins_config
                0x00005ccc       0xc0 ./ra/fsp/src/r_ioport/r_ioport.o
 .text.R_IOPORT_Open
                0x00005d8c       0x2c ./ra/fsp/src/r_ioport/r_ioport.o
                0x00005d8c                R_IOPORT_Open
 .text.flash_hp_init
                0x00005db8      0x114 ./ra/fsp/src/r_flash_hp/r_flash_hp.o
 .text.R_FLASH_HP_Close
                0x00005ecc       0x88 ./ra/fsp/src/r_flash_hp/r_flash_hp.o
                0x00005ecc                R_FLASH_HP_Close
 .text.R_FLASH_HP_Open
                0x00005f54      0x11c ./ra/fsp/src/r_flash_hp/r_flash_hp.o
                0x00005f54                R_FLASH_HP_Open
 .text.R_FLASH_HP_Write
                0x00006070       0x80 ./ra/fsp/src/r_flash_hp/r_flash_hp.o
                0x00006070                R_FLASH_HP_Write
 .text.R_FLASH_HP_Erase
                0x000060f0       0x98 ./ra/fsp/src/r_flash_hp/r_flash_hp.o
                0x000060f0                R_FLASH_HP_Erase
 .text.SystemCoreClockUpdate
                0x00006188       0x28 ./ra/fsp/src/bsp/mcu/all/bsp_clocks.o
                0x00006188                SystemCoreClockUpdate
 .text.bsp_clock_init
                0x000061b0      0x150 ./ra/fsp/src/bsp/mcu/all/bsp_clocks.o
                0x000061b0                bsp_clock_init
 .text.bsp_init_internal
                0x00006300        0x4 ./ra/fsp/src/bsp/mcu/all/bsp_common.o
                0x00006300                bsp_init_internal
                0x00006300                bsp_init
 .text.bsp_prv_software_delay_loop
                0x00006304        0xc ./ra/fsp/src/bsp/mcu/all/bsp_delay.o
                0x00006304                bsp_prv_software_delay_loop
 .text.R_BSP_SoftwareDelay
                0x00006310       0x68 ./ra/fsp/src/bsp/mcu/all/bsp_delay.o
                0x00006310                R_BSP_SoftwareDelay
 .text.NMI_Handler
                0x00006378       0x38 ./ra/fsp/src/bsp/mcu/all/bsp_group_irq.o
                0x00006378                NMI_Handler
 .text.bsp_irq_cfg
                0x000063b0       0xa0 ./ra/fsp/src/bsp/mcu/all/bsp_irq.o
                0x000063b0                bsp_irq_cfg
 .text.R_BSP_RegisterProtectEnable
                0x00006450       0x60 ./ra/fsp/src/bsp/mcu/all/bsp_register_protection.o
                0x00006450                R_BSP_RegisterProtectEnable
 .text.R_BSP_RegisterProtectDisable
                0x000064b0       0x54 ./ra/fsp/src/bsp/mcu/all/bsp_register_protection.o
                0x000064b0                R_BSP_RegisterProtectDisable
 .text.Default_Handler
                0x00006504        0x4 ./ra/fsp/src/bsp/cmsis/Device/RENESAS/Source/startup.o
                0x00006504                DebugMon_Handler
                0x00006504                HardFault_Handler
                0x00006504                SysTick_Handler
                0x00006504                PendSV_Handler
                0x00006504                UsageFault_Handler
                0x00006504                SecureFault_Handler
                0x00006504                Default_Handler
                0x00006504                MemManage_Handler
                0x00006504                SVC_Handler
                0x00006504                BusFault_Handler
 .text.Reset_Handler
                0x00006508        0xc ./ra/fsp/src/bsp/cmsis/Device/RENESAS/Source/startup.o
                0x00006508                Reset_Handler
 .text.R_BSP_WarmStart
                0x00006514        0x4 ./ra/fsp/src/bsp/cmsis/Device/RENESAS/Source/system.o
                0x00006514                R_BSP_WarmStart
 .text.SystemInit
                0x00006518       0xc0 ./ra/fsp/src/bsp/cmsis/Device/RENESAS/Source/system.o
                0x00006518                SystemInit
 .text          0x000065d8      0x378 c:/renesas/ra/e2studio_v2022-10_fsp_v4.2.0/toolchains/gcc_arm/gcc-arm-none-eabi-10.3-2021.10/bin/../lib/gcc/arm-none-eabi/10.3.1/thumb/v8-m.main+fp/hard\libgcc.a(_arm_addsubdf3.o)
                0x000065d8                __aeabi_drsub
                0x000065e0                __aeabi_dsub
                0x000065e0                __subdf3
                0x000065e4                __aeabi_dadd
                0x000065e4                __adddf3
                0x0000685c                __floatunsidf
                0x0000685c                __aeabi_ui2d
                0x0000687c                __floatsidf
                0x0000687c                __aeabi_i2d
                0x000068a0                __aeabi_f2d
                0x000068a0                __extendsfdf2
                0x000068e4                __floatundidf
                0x000068e4                __aeabi_ul2d
                0x000068f4                __floatdidf
                0x000068f4                __aeabi_l2d
 .text          0x00006950      0x424 c:/renesas/ra/e2studio_v2022-10_fsp_v4.2.0/toolchains/gcc_arm/gcc-arm-none-eabi-10.3-2021.10/bin/../lib/gcc/arm-none-eabi/10.3.1/thumb/v8-m.main+fp/hard\libgcc.a(_arm_muldivdf3.o)
                0x00006950                __aeabi_dmul
                0x00006950                __muldf3
                0x00006ba4                __divdf3
                0x00006ba4                __aeabi_ddiv
 .text          0x00006d74      0x110 c:/renesas/ra/e2studio_v2022-10_fsp_v4.2.0/toolchains/gcc_arm/gcc-arm-none-eabi-10.3-2021.10/bin/../lib/gcc/arm-none-eabi/10.3.1/thumb/v8-m.main+fp/hard\libgcc.a(_arm_cmpdf2.o)
                0x00006d74                __gtdf2
                0x00006d74                __gedf2
                0x00006d7c                __ltdf2
                0x00006d7c                __ledf2
                0x00006d84                __nedf2
                0x00006d84                __eqdf2
                0x00006d84                __cmpdf2
                0x00006e00                __aeabi_cdrcmple
                0x00006e10                __aeabi_cdcmpeq
                0x00006e10                __aeabi_cdcmple
                0x00006e20                __aeabi_dcmpeq
                0x00006e34                __aeabi_dcmplt
                0x00006e48                __aeabi_dcmple
                0x00006e5c                __aeabi_dcmpge
                0x00006e70                __aeabi_dcmpgt
 .text          0x00006e84       0x2c c:/renesas/ra/e2studio_v2022-10_fsp_v4.2.0/toolchains/gcc_arm/gcc-arm-none-eabi-10.3-2021.10/bin/../lib/gcc/arm-none-eabi/10.3.1/thumb/v8-m.main+fp/hard\libgcc.a(_arm_unorddf2.o)
                0x00006e84                __unorddf2
                0x00006e84                __aeabi_dcmpun
 .text          0x00006eb0       0x50 c:/renesas/ra/e2studio_v2022-10_fsp_v4.2.0/toolchains/gcc_arm/gcc-arm-none-eabi-10.3-2021.10/bin/../lib/gcc/arm-none-eabi/10.3.1/thumb/v8-m.main+fp/hard\libgcc.a(_arm_fixdfsi.o)
                0x00006eb0                __aeabi_d2iz
                0x00006eb0                __fixdfsi
 .text.__aeabi_memcpy
                0x00006f00        0x4 c:/renesas/ra/e2studio_v2022-10_fsp_v4.2.0/toolchains/gcc_arm/gcc-arm-none-eabi-10.3-2021.10/bin/../lib/gcc/arm-none-eabi/10.3.1/../../../../arm-none-eabi/lib/thumb/v8-m.main+fp/hard\libg_nano.a(lib_a-aeabi_memcpy.o)
                0x00006f00                __aeabi_memcpy4
                0x00006f00                __aeabi_memcpy8
                0x00006f00                __aeabi_memcpy
 .text.memcpy   0x00006f04       0x1a c:/renesas/ra/e2studio_v2022-10_fsp_v4.2.0/toolchains/gcc_arm/gcc-arm-none-eabi-10.3-2021.10/bin/../lib/gcc/arm-none-eabi/10.3.1/../../../../arm-none-eabi/lib/thumb/v8-m.main+fp/hard\libg_nano.a(lib_a-memcpy-stub.o)
                0x00006f04                memcpy
 .text.memset   0x00006f1e       0x10 c:/renesas/ra/e2studio_v2022-10_fsp_v4.2.0/toolchains/gcc_arm/gcc-arm-none-eabi-10.3-2021.10/bin/../lib/gcc/arm-none-eabi/10.3.1/../../../../arm-none-eabi/lib/thumb/v8-m.main+fp/hard\libg_nano.a(lib_a-memset.o)
                0x00006f1e                memset
 .text          0x00006f2e       0x10 c:/renesas/ra/e2studio_v2022-10_fsp_v4.2.0/toolchains/gcc_arm/gcc-arm-none-eabi-10.3-2021.10/bin/../lib/gcc/arm-none-eabi/10.3.1/../../../../arm-none-eabi/lib/thumb/v8-m.main+fp/hard\libg_nano.a(lib_a-strlen.o)
                0x00006f2e                strlen
 *(.version)
 *fill*         0x00006f3e        0x2 ff
 .version       0x00006f40       0x50 ./ra/fsp/src/bsp/mcu/all/bsp_common.o
 *(.init)
 .init          0x00006f90        0x4 c:/renesas/ra/e2studio_v2022-10_fsp_v4.2.0/toolchains/gcc_arm/gcc-arm-none-eabi-10.3-2021.10/bin/../lib/gcc/arm-none-eabi/10.3.1/thumb/v8-m.main+fp/hard/crti.o
                0x00006f90                _init
 .init          0x00006f94        0x8 c:/renesas/ra/e2studio_v2022-10_fsp_v4.2.0/toolchains/gcc_arm/gcc-arm-none-eabi-10.3-2021.10/bin/../lib/gcc/arm-none-eabi/10.3.1/thumb/v8-m.main+fp/hard/crtn.o
 *(.fini)
 .fini          0x00006f9c        0x4 c:/renesas/ra/e2studio_v2022-10_fsp_v4.2.0/toolchains/gcc_arm/gcc-arm-none-eabi-10.3-2021.10/bin/../lib/gcc/arm-none-eabi/10.3.1/thumb/v8-m.main+fp/hard/crti.o
                0x00006f9c                _fini
 .fini          0x00006fa0        0x8 c:/renesas/ra/e2studio_v2022-10_fsp_v4.2.0/toolchains/gcc_arm/gcc-arm-none-eabi-10.3-2021.10/bin/../lib/gcc/arm-none-eabi/10.3.1/thumb/v8-m.main+fp/hard/crtn.o
 .fini.__stub   0x00006fa8       0x20 linker stubs
 *crtbegin.o(.ctors)
 *crtbegin?.o(.ctors)
 *(EXCLUDE_FILE(*crtend.o *crtend?.o) .ctors)
 *(SORT_BY_NAME(.ctors.*))
 *(.ctors)
 *crtbegin.o(.dtors)
 *crtbegin?.o(.dtors)
 *(EXCLUDE_FILE(*crtend.o *crtend?.o) .dtors)
 *(SORT_BY_NAME(.dtors.*))
 *(.dtors)
 *(.rodata*)
 .rodata.str1.4
                0x00006fc8       0x44 ./src/hal_entry.o
 .rodata.getstr.constprop.0.str1.4
                0x0000700c        0x4 ./src/hal_entry.o
 .rodata.hal_entry.str1.4
                0x00007010       0xae ./src/hal_entry.o
 *fill*         0x000070be        0x2 ff
 .rodata.udp_printf.str1.4
                0x000070c0        0xb ./src/udp_printf.o
                                  0xf (size before relaxing)
 *fill*         0x000070cb        0x1 ff
 .rodata.usb_descriptor
                0x000070cc       0x18 ./src/usb_desc.o
                0x000070cc                usb_descriptor
 .rodata.g_basic0_cfg
                0x000070e4       0x2c ./ra_gen/hal_data.o
                0x000070e4                g_basic0_cfg
 .rodata.g_flash0_cfg
                0x00007110       0x14 ./ra_gen/hal_data.o
                0x00007110                g_flash0_cfg
 .rodata.g_bsp_pin_cfg
                0x00007124        0x8 ./ra_gen/pin_data.o
                0x00007124                g_bsp_pin_cfg
 .rodata.g_bsp_pin_cfg_data
                0x0000712c       0x18 ./ra_gen/pin_data.o
                0x0000712c                g_bsp_pin_cfg_data
 .rodata.g_interrupt_event_link_select
                0x00007144       0xc0 ./ra_gen/vector_data.o
                0x00007144                g_interrupt_event_link_select
 .rodata.g_usb_pipe_peri
                0x00007204       0x10 ./ra/fsp/src/r_usb_basic/src/driver/r_usb_cdataio.o
 .rodata.CSWTCH.10
                0x00007214        0x8 ./ra/fsp/src/r_usb_basic/src/driver/r_usb_clibusbip.o
 .rodata.g_prcr_masks
                0x0000721c        0x8 ./ra/fsp/src/bsp/mcu/all/bsp_register_protection.o
                0x00007224                __usb_dev_descriptor_start_fs = .
 *(.usb_device_desc_fs*)
                0x00007224                __usb_cfg_descriptor_start_fs = .
 *(.usb_config_desc_fs*)
                0x00007224                __usb_interface_descriptor_start_fs = .
 *(.usb_interface_desc_fs*)
                0x00007224                __usb_descriptor_end_fs = .
                0x00007224                __usb_dev_descriptor_start_hs = .
 *(.usb_device_desc_hs*)
                0x00007224                __usb_cfg_descriptor_start_hs = .
 *(.usb_config_desc_hs*)
                0x00007224                __usb_interface_descriptor_start_hs = .
 *(.usb_interface_desc_hs*)
                0x00007224                __usb_descriptor_end_hs = .
 *(.eh_frame*)
 .eh_frame      0x00007224        0x0 c:/renesas/ra/e2studio_v2022-10_fsp_v4.2.0/toolchains/gcc_arm/gcc-arm-none-eabi-10.3-2021.10/bin/../lib/gcc/arm-none-eabi/10.3.1/thumb/v8-m.main+fp/hard/crtbegin.o
 .eh_frame      0x00007224        0x4 c:/renesas/ra/e2studio_v2022-10_fsp_v4.2.0/toolchains/gcc_arm/gcc-arm-none-eabi-10.3-2021.10/bin/../lib/gcc/arm-none-eabi/10.3.1/thumb/v8-m.main+fp/hard/crtend.o
                0x00007228                __ROM_End = .
                0x000001c0                __Vectors_Size = (__Vectors_End - __Vectors)

.glue_7         0x00007228        0x0
 .glue_7        0x00007228        0x0 linker stubs

.glue_7t        0x00007228        0x0
 .glue_7t       0x00007228        0x0 linker stubs

.vfp11_veneer   0x00007228        0x0
 .vfp11_veneer  0x00007228        0x0 linker stubs

.v4_bx          0x00007228        0x0
 .v4_bx         0x00007228        0x0 linker stubs

.iplt           0x00007228        0x0
 .iplt          0x00007228        0x0 c:/renesas/ra/e2studio_v2022-10_fsp_v4.2.0/toolchains/gcc_arm/gcc-arm-none-eabi-10.3-2021.10/bin/../lib/gcc/arm-none-eabi/10.3.1/thumb/v8-m.main+fp/hard/crtbegin.o

.ARM.extab
 *(.ARM.extab* .gnu.linkonce.armextab.*)
                0x00007228                __exidx_start = .

.ARM.exidx
 *(.ARM.exidx* .gnu.linkonce.armexidx.*)
                0x00007228                __exidx_end = .
                0x00007228                __etext = .
                0x20000000                __tz_RAM_S = ORIGIN (RAM)

.fsp_dtc_vector_table
                0x20000000        0x0
                0x20000000                . = ORIGIN (RAM)
 *(.fsp_dtc_vector_table)

.data           0x20000000      0x934 load address 0x00007228
                0x20000000                __data_start__ = .
                0x20000000                . = ALIGN (0x4)
                0x20000000                __Code_In_RAM_Start = .
 *(.code_in_ram*)
 .code_in_ram   0x20000000      0x708 ./ra/fsp/src/r_flash_hp/r_flash_hp.o
                0x20000708                __Code_In_RAM_End = .
 *(vtable)
 *(.data.*)
 .data.packetno.2
                0x20000708        0x1 ./src/hal_entry.o
 .data.txcomplete
                0x20000709        0x1 ./src/udp_cdc.o
 *fill*         0x2000070a        0x2 
 .data.g_apl_configuration
                0x2000070c       0x44 ./src/usb_desc.o
                0x2000070c                g_apl_configuration
 .data.g_apl_device
                0x20000750       0x12 ./src/usb_desc.o
                0x20000750                g_apl_device
 *fill*         0x20000762        0x2 
 .data.g_apl_hs_configuration
                0x20000764       0x44 ./src/usb_desc.o
                0x20000764                g_apl_hs_configuration
 .data.g_apl_qualifier_descriptor
                0x200007a8        0xa ./src/usb_desc.o
                0x200007a8                g_apl_qualifier_descriptor
 *fill*         0x200007b2        0x2 
 .data.g_apl_string_table
                0x200007b4       0x1c ./src/usb_desc.o
                0x200007b4                g_apl_string_table
 .data.g_cdc_string_descriptor0
                0x200007d0        0x4 ./src/usb_desc.o
                0x200007d0                g_cdc_string_descriptor0
 .data.g_cdc_string_descriptor1
                0x200007d4       0x10 ./src/usb_desc.o
                0x200007d4                g_cdc_string_descriptor1
 .data.g_cdc_string_descriptor2
                0x200007e4       0x2c ./src/usb_desc.o
                0x200007e4                g_cdc_string_descriptor2
 .data.g_cdc_string_descriptor3
                0x20000810       0x2e ./src/usb_desc.o
                0x20000810                g_cdc_string_descriptor3
 *fill*         0x2000083e        0x2 
 .data.g_cdc_string_descriptor4
                0x20000840       0x16 ./src/usb_desc.o
                0x20000840                g_cdc_string_descriptor4
 *fill*         0x20000856        0x2 
 .data.g_cdc_string_descriptor5
                0x20000858       0x12 ./src/usb_desc.o
                0x20000858                g_cdc_string_descriptor5
 *fill*         0x2000086a        0x2 
 .data.g_cdc_string_descriptor6
                0x2000086c       0x1c ./src/usb_desc.o
                0x2000086c                g_cdc_string_descriptor6
 .data.g_usb_callback
                0x20000888       0x88 ./ra/fsp/src/r_usb_basic/src/driver/r_usb_cdataio.o
                0x20000888                g_usb_callback
 .data.g_usb_pcdc_serialstate_table
                0x20000910        0xa ./ra/fsp/src/r_usb_basic/src/driver/r_usb_cdataio.o
                0x20000910                g_usb_pcdc_serialstate_table
 *fill*         0x2000091a        0x2 
 .data.g_configuration_area_data
                0x2000091c       0x10 ./ra/fsp/src/r_flash_hp/r_flash_hp.o
 *(.data)
                0x2000092c                . = ALIGN (0x4)
                0x2000092c                PROVIDE (__preinit_array_start = .)
 *(.preinit_array)
                0x2000092c                PROVIDE (__preinit_array_end = .)
                0x2000092c                . = ALIGN (0x4)
                0x2000092c                PROVIDE (__init_array_start = .)
 *(SORT_BY_NAME(.init_array.*))
 *(.init_array)
 .init_array    0x2000092c        0x4 c:/renesas/ra/e2studio_v2022-10_fsp_v4.2.0/toolchains/gcc_arm/gcc-arm-none-eabi-10.3-2021.10/bin/../lib/gcc/arm-none-eabi/10.3.1/thumb/v8-m.main+fp/hard/crtbegin.o
                0x20000930                PROVIDE (__init_array_end = .)
                0x20000930                . = ALIGN (0x4)
                [!provide]                PROVIDE (__fini_array_start = .)
 *(SORT_BY_NAME(.fini_array.*))
 *(.fini_array)
 .fini_array    0x20000930        0x4 c:/renesas/ra/e2studio_v2022-10_fsp_v4.2.0/toolchains/gcc_arm/gcc-arm-none-eabi-10.3-2021.10/bin/../lib/gcc/arm-none-eabi/10.3.1/thumb/v8-m.main+fp/hard/crtbegin.o
                [!provide]                PROVIDE (__fini_array_end = .)
 *(.jcr*)
                0x20000934                . = ALIGN (0x4)
                0x20000934                __data_end__ = .
                0x00007b5c                __dtcm_data_init_start = ((__etext + __data_end__) - __data_start__)

.igot.plt       0x20000934        0x0 load address 0x00007b5c
 .igot.plt      0x20000934        0x0 c:/renesas/ra/e2studio_v2022-10_fsp_v4.2.0/toolchains/gcc_arm/gcc-arm-none-eabi-10.3-2021.10/bin/../lib/gcc/arm-none-eabi/10.3.1/thumb/v8-m.main+fp/hard/crtbegin.o

.dtcm_data      0x00000000        0x0 load address 0x00007b5c
                0x00000000                __tz_DTCM_S = ABSOLUTE (DTCM_START)
                0x00000000                __dtcm_data_start__ = .
 *(.dtcm_data*)
                0x00000000                __dtcm_data_end__ = .

.dtcm_noinit    0x00000000        0x0 load address 0x00007b5c
                0x00000000                __dtcm_noinit_start = .
 *(.dtcm_noinit*)
                0x00000000                __dtcm_noinit_end = .
                0x00000000                __tz_DTCM_N = DEFINED (DTCM_NS_START)?ABSOLUTE (DTCM_NS_START):ALIGN (__dtcm_noinit_end, 0x2000)
                0x00007b5c                DATA_END = (LOADADDR (.data) + SIZEOF (.data))
                0x00007c00                SGSTUBS_LOC = (DEFINED (PROJECT_SECURE) && DEFINED (FLASH_NSC_START))?ABSOLUTE (FLASH_NSC_START):ALIGN (DATA_END, 0x400)

.gnu.sgstubs    0x00007c00        0x0
                0x00007c00                __tz_FLASH_C = DEFINED (FLASH_NSC_START)?ABSOLUTE (FLASH_NSC_START):__RESERVE_NS_RAM?ABSOLUTE ((FLASH_START + FLASH_LENGTH)):ALIGN (0x400)
                0x00007c00                _start_sg = .
 *(.gnu.sgstubs*)
                0x00007c00                . = ALIGN (0x20)
                0x00007c00                _end_sg = .
                0x00008000                __tz_FLASH_N = DEFINED (FLASH_NS_START)?ABSOLUTE (FLASH_NS_START):__RESERVE_NS_RAM?ABSOLUTE ((FLASH_START + FLASH_LENGTH)):(FLASH_LENGTH < 0x8000)?FLASH_LENGTH:ALIGN (0x8000)
                0x00008000                FLASH_NS_IMAGE_START = DEFINED (FLASH_NS_IMAGE_START)?FLASH_NS_IMAGE_START:__tz_FLASH_N
                0x60000000                __tz_QSPI_FLASH_S = ORIGIN (QSPI_FLASH)

.qspi_flash     0x60000000        0x0
                0x60000000                __qspi_flash_start__ = .
 *(.qspi_flash*)
 *(.code_in_qspi*)
                0x60000000                __qspi_flash_end__ = .
                0x00000000                __qspi_flash_code_size__ = (__qspi_flash_end__ - __qspi_flash_start__)
                0x00007b5c                __qspi_flash_code_addr__ = (__etext + (__data_end__ - __data_start__))

.qspi_non_retentive
                0x60000000        0x0 load address 0x00007b5c
                0x60000000                __qspi_non_retentive_start__ = .
 *(.qspi_non_retentive*)
                0x60000000                __qspi_non_retentive_end__ = .
                0x00000000                __qspi_non_retentive_size__ = (__qspi_non_retentive_end__ - __qspi_non_retentive_start__)
                0x04000000                __qspi_region_max_size__ = 0x4000000
                0x60000000                __qspi_region_start_address__ = __qspi_flash_start__
                0x64000000                __qspi_region_end_address__ = (__qspi_flash_start__ + __qspi_region_max_size__)
                0x60000000                __tz_QSPI_FLASH_N = __qspi_non_retentive_end__

.OSPI_DEVICE_0_NO_LOAD
                0x80020000        0x0
                0x80020000                . = ALIGN (0x4)
                0x80020000                __ospi_device_0_start__ = .
 *(.ospi_device_0_no_load*)
                0x80020000                . = ALIGN (0x4)
                0x80020000                __ospi_device_0_end__ = .

.OSPI_DEVICE_1_NO_LOAD
                0x80030000        0x0
                0x80030000                . = ALIGN (0x4)
                0x80030000                __ospi_device_1_start__ = .
 *(.ospi_device_1_no_load*)
                0x80030000                . = ALIGN (0x4)
                0x80030000                __ospi_device_1_end__ = .
                0x80020000                __tz_OSPI_DEVICE_0_S = ORIGIN (OSPI_DEVICE_0)

.OSPI_DEVICE_0  0x80020000        0x0
                0x80020000                __ospi_device_0_start__ = .
 *(.ospi_device_0*)
 *(.code_in_ospi_device_0*)
                0x80020000                __ospi_device_0_end__ = .
                0x00000000                __ospi_device_0_code_size__ = (__ospi_device_0_end__ - __ospi_device_0_start__)
                0x00007b5c                __ospi_device_0_code_addr__ = (__etext + (__data_end__ - __data_start__))

.ospi_device_0_non_retentive
                0x80020000        0x0 load address 0x00007b5c
                0x80020000                __ospi_device_0_non_retentive_start__ = .
 *(.ospi_device_0_non_retentive*)
                0x80020000                __ospi_device_0_non_retentive_end__ = .
                0x00000000                __ospi_device_0_non_retentive_size__ = (__ospi_device_0_non_retentive_end__ - __ospi_device_0_non_retentive_start__)
                0x08000000                __ospi_device_0_region_max_size__ = 0x8000000
                0x80020000                __ospi_device_0_region_start_address__ = __ospi_device_0_start__
                0x88020000                __ospi_device_0_region_end_address__ = (__ospi_device_0_start__ + __ospi_device_0_region_max_size__)
                0x80020000                __tz_OSPI_DEVICE_0_N = __ospi_device_0_non_retentive_end__
                0x80030000                __tz_OSPI_DEVICE_1_S = ORIGIN (OSPI_DEVICE_1)

.OSPI_DEVICE_1  0x80030000        0x0
                0x80030000                __ospi_device_1_start__ = .
 *(.ospi_device_1*)
 *(.code_in_ospi_device_1*)
                0x80030000                __ospi_device_1_end__ = .
                0x00000000                __ospi_device_1_code_size__ = (__ospi_device_1_end__ - __ospi_device_1_start__)
                0x00007b5c                __ospi_device_1_code_addr__ = (__etext + (__data_end__ - __data_start__))

.ospi_device_1_non_retentive
                0x80030000        0x0 load address 0x00007b5c
                0x80030000                __ospi_device_1_non_retentive_start__ = .
 *(.ospi_device_1_non_retentive*)
                0x80030000                __ospi_device_1_non_retentive_end__ = .
                0x00000000                __ospi_device_1_non_retentive_size__ = (__ospi_device_1_non_retentive_end__ - __ospi_device_1_non_retentive_start__)
                0x10000000                __ospi_device_1_region_max_size__ = 0x10000000
                0x80030000                __ospi_device_1_region_start_address__ = __ospi_device_1_start__
                0x90030000                __ospi_device_1_region_end_address__ = (__ospi_device_1_start__ + __ospi_device_1_region_max_size__)
                0x80030000                __tz_OSPI_DEVICE_1_N = __ospi_device_1_non_retentive_end__

.noinit         0x20000934       0x1c
                0x20000934                . = ALIGN (0x4)
                0x20000934                __noinit_start = .
 *(.noinit*)
 .noinit        0x20000934       0x1c ./ra/fsp/src/bsp/mcu/all/bsp_clocks.o
                0x20000950                . = ALIGN (0x8)
 *(.heap.*)
                0x20000950                __noinit_end = .

.bss            0x20000950     0x2704
                0x20000950                . = ALIGN (0x4)
                0x20000950                __bss_start__ = .
 *(.bss*)
 .bss           0x20000950       0x1c c:/renesas/ra/e2studio_v2022-10_fsp_v4.2.0/toolchains/gcc_arm/gcc-arm-none-eabi-10.3-2021.10/bin/../lib/gcc/arm-none-eabi/10.3.1/thumb/v8-m.main+fp/hard/crtbegin.o
 .bss.rxb       0x2000096c      0x7d0 ./src/hal_entry.o
                0x2000096c                rxb
 .bss.txb       0x2000113c       0x64 ./src/hal_entry.o
                0x2000113c                txb
 .bss.xbuff.3   0x200011a0      0x41e ./src/hal_entry.o
 *fill*         0x200015be        0x2 
 .bss.xbuff.4   0x200015c0      0x400 ./src/hal_entry.o
 .bss.FIFO      0x200019c0       0x18 ./src/udp_cdc.o
 .bss.b_usb_attach
                0x200019d8        0x1 ./src/udp_cdc.o
 *fill*         0x200019d9        0x3 
 .bss.g_buf     0x200019dc      0x800 ./src/udp_cdc.o
 .bss.g_line_coding
                0x200021dc        0x8 ./src/udp_cdc.o
 .bss.buf.0     0x200021e4      0x400 ./src/udp_printf.o
 .bss.g_ioport_ctrl
                0x200025e4        0x8 ./ra_gen/common_data.o
                0x200025e4                g_ioport_ctrl
 .bss.g_basic0_ctrl
                0x200025ec       0x24 ./ra_gen/hal_data.o
                0x200025ec                g_basic0_ctrl
 .bss.g_flash0_ctrl
                0x20002610       0x44 ./ra_gen/hal_data.o
                0x20002610                g_flash0_ctrl
 .bss.g_usb_cstd_suspend_mode
                0x20002654        0x2 ./ra/fsp/src/r_usb_basic/src/hw/r_usb_preg_abs.o
                0x20002654                g_usb_cstd_suspend_mode
 *fill*         0x20002656        0x2 
 .bss.g_p_usb_pstd_pipe
                0x20002658       0x28 ./ra/fsp/src/r_usb_basic/src/driver/r_usb_cdataio.o
                0x20002658                g_p_usb_pstd_pipe
 .bss.g_usb_cstd_bemp_skip
                0x20002680       0x28 ./ra/fsp/src/r_usb_basic/src/driver/r_usb_cdataio.o
                0x20002680                g_usb_cstd_bemp_skip
 .bss.g_usb_pipe_table
                0x200026a8       0xc8 ./ra/fsp/src/r_usb_basic/src/driver/r_usb_cdataio.o
                0x200026a8                g_usb_pipe_table
 .bss.g_usb_pstd_data_cnt
                0x20002770       0x28 ./ra/fsp/src/r_usb_basic/src/driver/r_usb_cdataio.o
                0x20002770                g_usb_pstd_data_cnt
 .bss.gp_usb_pstd_data
                0x20002798       0x28 ./ra/fsp/src/r_usb_basic/src/driver/r_usb_cdataio.o
                0x20002798                gp_usb_pstd_data
 .bss.g_usb_peri_connected
                0x200027c0        0x2 ./ra/fsp/src/r_usb_basic/src/driver/r_usb_pdriver.o
                0x200027c0                g_usb_peri_connected
 *fill*         0x200027c2        0x2 
 .bss.g_usb_pstd_alt_num
                0x200027c4      0x1fe ./ra/fsp/src/r_usb_basic/src/driver/r_usb_pdriver.o
                0x200027c4                g_usb_pstd_alt_num
 .bss.g_usb_pstd_config_num
                0x200029c2        0x2 ./ra/fsp/src/r_usb_basic/src/driver/r_usb_pdriver.o
                0x200029c2                g_usb_pstd_config_num
 .bss.g_usb_pstd_driver
                0x200029c4       0x34 ./ra/fsp/src/r_usb_basic/src/driver/r_usb_pdriver.o
                0x200029c4                g_usb_pstd_driver
 .bss.g_usb_pstd_eptbl_index
                0x200029f8       0x40 ./ra/fsp/src/r_usb_basic/src/driver/r_usb_pdriver.o
                0x200029f8                g_usb_pstd_eptbl_index
 .bss.g_usb_pstd_pipe0_request
                0x20002a38        0x2 ./ra/fsp/src/r_usb_basic/src/driver/r_usb_pdriver.o
                0x20002a38                g_usb_pstd_pipe0_request
 .bss.g_usb_pstd_remote_wakeup
                0x20002a3a        0x2 ./ra/fsp/src/r_usb_basic/src/driver/r_usb_pdriver.o
                0x20002a3a                g_usb_pstd_remote_wakeup
 .bss.g_usb_pstd_req_index
                0x20002a3c        0x2 ./ra/fsp/src/r_usb_basic/src/driver/r_usb_pdriver.o
                0x20002a3c                g_usb_pstd_req_index
 .bss.g_usb_pstd_req_length
                0x20002a3e        0x2 ./ra/fsp/src/r_usb_basic/src/driver/r_usb_pdriver.o
                0x20002a3e                g_usb_pstd_req_length
 .bss.g_usb_pstd_req_reg
                0x20002a40        0x8 ./ra/fsp/src/r_usb_basic/src/driver/r_usb_pdriver.o
                0x20002a40                g_usb_pstd_req_reg
 .bss.g_usb_pstd_req_type
                0x20002a48        0x2 ./ra/fsp/src/r_usb_basic/src/driver/r_usb_pdriver.o
                0x20002a48                g_usb_pstd_req_type
 .bss.g_usb_pstd_req_value
                0x20002a4a        0x2 ./ra/fsp/src/r_usb_basic/src/driver/r_usb_pdriver.o
                0x20002a4a                g_usb_pstd_req_value
 .bss.g_usb_pstd_stall_cb
                0x20002a4c        0x4 ./ra/fsp/src/r_usb_basic/src/driver/r_usb_pdriver.o
                0x20002a4c                g_usb_pstd_stall_cb
 .bss.g_usb_pstd_stall_pipe
                0x20002a50       0x14 ./ra/fsp/src/r_usb_basic/src/driver/r_usb_pdriver.o
                0x20002a50                g_usb_pstd_stall_pipe
 .bss.g_usb_pstd_std_request
                0x20002a64        0x2 ./ra/fsp/src/r_usb_basic/src/driver/r_usb_pdriver.o
                0x20002a64                g_usb_pstd_std_request
 .bss.g_usb_pstd_test_mode_flag
                0x20002a66        0x2 ./ra/fsp/src/r_usb_basic/src/driver/r_usb_pdriver.o
                0x20002a66                g_usb_pstd_test_mode_flag
 .bss.g_usb_pstd_test_mode_select
                0x20002a68        0x2 ./ra/fsp/src/r_usb_basic/src/driver/r_usb_pdriver.o
                0x20002a68                g_usb_pstd_test_mode_select
 *fill*         0x20002a6a        0x2 
 .bss.g_usb_pstd_usb_int
                0x20002a6c       0x54 ./ra/fsp/src/r_usb_basic/src/driver/r_usb_pinthandler_usbip0.o
                0x20002a6c                g_usb_pstd_usb_int
 .bss.tbl.0     0x20002ac0        0x2 ./ra/fsp/src/r_usb_basic/src/driver/r_usb_pstdrequest.o
 *fill*         0x20002ac2        0x2 
 .bss.tbl.1     0x20002ac4        0x2 ./ra/fsp/src/r_usb_basic/src/driver/r_usb_pstdrequest.o
 *fill*         0x20002ac6        0x2 
 .bss.tbl.2     0x20002ac8        0x2 ./ra/fsp/src/r_usb_basic/src/driver/r_usb_pstdrequest.o
 *fill*         0x20002aca        0x2 
 .bss.g_usb_change_device_state
                0x20002acc        0x4 ./ra/fsp/src/r_usb_basic/r_usb_basic.o
                0x20002acc                g_usb_change_device_state
 .bss.g_usb_cstd_event
                0x20002ad0      0x174 ./ra/fsp/src/r_usb_basic/r_usb_basic.o
                0x20002ad0                g_usb_cstd_event
 .bss.g_usb_open_class
                0x20002c44        0x8 ./ra/fsp/src/r_usb_basic/r_usb_basic.o
                0x20002c44                g_usb_open_class
 .bss.g_usb_pdata
                0x20002c4c      0x230 ./ra/fsp/src/r_usb_basic/r_usb_basic.o
                0x20002c4c                g_usb_pdata
 .bss.g_usb_usbmode
                0x20002e7c        0x4 ./ra/fsp/src/r_usb_basic/r_usb_basic.o
                0x20002e7c                g_usb_usbmode
 .bss.is_init   0x20002e80        0x2 ./ra/fsp/src/r_usb_basic/r_usb_basic.o
 *fill*         0x20002e82        0x2 
 .bss.g_bsp_group_irq_sources
                0x20002e84       0x40 ./ra/fsp/src/bsp/mcu/all/bsp_group_irq.o
                0x20002e84                g_bsp_group_irq_sources
 .bss.g_protect_pfswe_counter
                0x20002ec4        0x4 ./ra/fsp/src/bsp/mcu/all/bsp_io.o
                0x20002ec4                g_protect_pfswe_counter
 .bss.gp_renesas_isr_context
                0x20002ec8      0x180 ./ra/fsp/src/bsp/mcu/all/bsp_irq.o
                0x20002ec8                gp_renesas_isr_context
 .bss.g_protect_counters
                0x20003048        0x8 ./ra/fsp/src/bsp/mcu/all/bsp_register_protection.o
                0x20003048                g_protect_counters
 .bss.SystemCoreClock
                0x20003050        0x4 ./ra/fsp/src/bsp/cmsis/Device/RENESAS/Source/system.o
                0x20003050                SystemCoreClock
 *(COMMON)
                0x20003054                . = ALIGN (0x4)
                0x20003054                __bss_end__ = .

.heap           0x20003058      0x400
                0x20003058                . = ALIGN (0x8)
                0x20003058                __HeapBase = .
 *(.heap)
 .heap          0x20003058      0x400 ./ra/fsp/src/bsp/cmsis/Device/RENESAS/Source/startup.o
                0x20003458                __HeapLimit = .

.stack_dummy    0x20003458      0x400
                0x20003458                . = ALIGN (0x8)
                0x20003458                __StackLimit = .
 *(.stack)
 .stack         0x20003458      0x400 ./ra/fsp/src/bsp/cmsis/Device/RENESAS/Source/startup.o
                0x20003858                __StackTop = .
 *(.stack*)
                0x20003858                __StackTopAll = .
                0x20003858                PROVIDE (__stack = __StackTopAll)
                0x20003858                __RAM_segment_used_end__ = ALIGN (__StackTopAll, 0x4)
                0x20003c00                __tz_RAM_C = DEFINED (RAM_NSC_START)?ABSOLUTE (RAM_NSC_START):__RESERVE_NS_RAM?ABSOLUTE (RAM_NS_BUFFER_BLOCK_START):ALIGN (__RAM_segment_used_end__, 0x400)
                0x20004000                __tz_RAM_N = DEFINED (RAM_NS_START)?ABSOLUTE (RAM_NS_START):__RESERVE_NS_RAM?ABSOLUTE (RAM_NS_BUFFER_BLOCK_START):ALIGN (__tz_RAM_C, 0x2000)

.ns_buffer      0x20003858        0x0
                0x20003858                . = __RESERVE_NS_RAM?ABSOLUTE ((RAM_NS_BUFFER_START & 0xffffffe0)):.
 *(.ns_buffer*)

.data_flash     0x08000000        0x0
                0x08000000                . = ORIGIN (DATA_FLASH)
                0x08000000                __tz_DATA_FLASH_S = .
                0x08000000                __Data_Flash_Start = .
 *(.data_flash*)
                0x08000000                __Data_Flash_End = .
                0x08000000                __tz_DATA_FLASH_N = DEFINED (DATA_FLASH_NS_START)?ABSOLUTE (DATA_FLASH_NS_START):__RESERVE_NS_RAM?ABSOLUTE ((DATA_FLASH_START + DATA_FLASH_LENGTH)):ALIGN (0x400)
                0x80010000                __tz_SDRAM_S = ORIGIN (SDRAM)

.sdram          0x80010000        0x0
                0x80010000                __SDRAM_Start = .
 *(.sdram*)
 *(.frame*)
                0x80010000                __SDRAM_End = .
                0x80010000                __tz_SDRAM_N = __SDRAM_End
                0x00000000                __tz_ID_CODE_S = ORIGIN (ID_CODE)

.id_code        0x00000000        0x0
                0x00000000                __ID_Code_Start = .
 *(.id_code*)
                0x00000000                __ID_Code_End = .
                0x00000000                __tz_ID_CODE_N = __ID_Code_End
                0x0100a100                __tz_OPTION_SETTING_S = ORIGIN (OPTION_SETTING)

.option_setting
                0x0100a100       0x38
                0x0100a100                __OPTION_SETTING_Start = .
 *(.option_setting_ofs0)
 .option_setting_ofs0
                0x0100a100        0x4 ./ra/fsp/src/bsp/mcu/all/bsp_rom_registers.o
                0x0100a104                . = PROJECT_SECURE_OR_FLAT?(__OPTION_SETTING_Start + 0x4):__OPTION_SETTING_Start
 *(.option_setting_ofs2)
                0x0100a110                . = PROJECT_SECURE_OR_FLAT?(__OPTION_SETTING_Start + 0x10):__OPTION_SETTING_Start
 *fill*         0x0100a104        0xc ff
 *(.option_setting_dualsel)
                0x0100a134                . = PROJECT_SECURE_OR_FLAT?(__OPTION_SETTING_Start + 0x34):__OPTION_SETTING_Start
 *fill*         0x0100a110       0x24 ff
 *(.option_setting_sas)
 .option_setting_sas
                0x0100a134        0x4 ./ra/fsp/src/bsp/mcu/all/bsp_rom_registers.o
                0x0100a138                __OPTION_SETTING_End = .
                0x0100a180                __tz_OPTION_SETTING_N = ABSOLUTE (OPTION_SETTING_START_NS)

.option_setting_ns
                0x0100a138        0x0
                0x0100a138                __OPTION_SETTING_NS_Start = .
 *(.option_setting_ofs1)
                0x0100a138                . = USE_OPTION_SETTING_NS?(__OPTION_SETTING_NS_Start + 0x4):__OPTION_SETTING_NS_Start
 *(.option_setting_ofs3)
                0x0100a138                . = USE_OPTION_SETTING_NS?(__OPTION_SETTING_NS_Start + 0x10):__OPTION_SETTING_NS_Start
 *(.option_setting_banksel)
                0x0100a138                . = USE_OPTION_SETTING_NS?(__OPTION_SETTING_NS_Start + 0x40):__OPTION_SETTING_NS_Start
 *(.option_setting_bps0)
                0x0100a138                . = USE_OPTION_SETTING_NS?(__OPTION_SETTING_NS_Start + 0x44):__OPTION_SETTING_NS_Start
 *(.option_setting_bps1)
                0x0100a138                . = USE_OPTION_SETTING_NS?(__OPTION_SETTING_NS_Start + 0x48):__OPTION_SETTING_NS_Start
 *(.option_setting_bps2)
                0x0100a138                . = USE_OPTION_SETTING_NS?(__OPTION_SETTING_NS_Start + 0x4c):__OPTION_SETTING_NS_Start
 *(.option_setting_bps3)
                0x0100a138                . = USE_OPTION_SETTING_NS?(__OPTION_SETTING_NS_Start + 0x60):__OPTION_SETTING_NS_Start
 *(.option_setting_pbps0)
                0x0100a138                . = USE_OPTION_SETTING_NS?(__OPTION_SETTING_NS_Start + 0x64):__OPTION_SETTING_NS_Start
 *(.option_setting_pbps1)
                0x0100a138                . = USE_OPTION_SETTING_NS?(__OPTION_SETTING_NS_Start + 0x68):__OPTION_SETTING_NS_Start
 *(.option_setting_pbps2)
                0x0100a138                . = USE_OPTION_SETTING_NS?(__OPTION_SETTING_NS_Start + 0x6c):__OPTION_SETTING_NS_Start
 *(.option_setting_pbps3)
                0x0100a138                __OPTION_SETTING_NS_End = .
                0x0100a200                __tz_OPTION_SETTING_S_S = ORIGIN (OPTION_SETTING_S)

.option_setting_s
                0x0100a200       0xd0
                0x0100a200                __OPTION_SETTING_S_Start = .
 *(.option_setting_ofs1_sec)
 .option_setting_ofs1_sec
                0x0100a200        0x4 ./ra/fsp/src/bsp/mcu/all/bsp_rom_registers.o
                0x0100a204                . = PROJECT_SECURE_OR_FLAT?(__OPTION_SETTING_S_Start + 0x4):__OPTION_SETTING_S_Start
 *(.option_setting_ofs3_sec)
                0x0100a210                . = PROJECT_SECURE_OR_FLAT?(__OPTION_SETTING_S_Start + 0x10):__OPTION_SETTING_S_Start
 *fill*         0x0100a204        0xc ff
 *(.option_setting_banksel_sec)
 .option_setting_banksel_sec
                0x0100a210        0x4 ./ra/fsp/src/bsp/mcu/all/bsp_rom_registers.o
                0x0100a240                . = PROJECT_SECURE_OR_FLAT?(__OPTION_SETTING_S_Start + 0x40):__OPTION_SETTING_S_Start
 *fill*         0x0100a214       0x2c ff
 *(.option_setting_bps_sec0)
 .option_setting_bps_sec0
                0x0100a240        0x4 ./ra/fsp/src/bsp/mcu/all/bsp_rom_registers.o
                0x0100a244                . = PROJECT_SECURE_OR_FLAT?(__OPTION_SETTING_S_Start + 0x44):__OPTION_SETTING_S_Start
 *(.option_setting_bps_sec1)
 .option_setting_bps_sec1
                0x0100a244        0x4 ./ra/fsp/src/bsp/mcu/all/bsp_rom_registers.o
                0x0100a248                . = PROJECT_SECURE_OR_FLAT?(__OPTION_SETTING_S_Start + 0x48):__OPTION_SETTING_S_Start
 *(.option_setting_bps_sec2)
 .option_setting_bps_sec2
                0x0100a248        0x4 ./ra/fsp/src/bsp/mcu/all/bsp_rom_registers.o
                0x0100a24c                . = PROJECT_SECURE_OR_FLAT?(__OPTION_SETTING_S_Start + 0x4c):__OPTION_SETTING_S_Start
 *(.option_setting_bps_sec3)
 .option_setting_bps_sec3
                0x0100a24c        0x4 ./ra/fsp/src/bsp/mcu/all/bsp_rom_registers.o
                0x0100a260                . = PROJECT_SECURE_OR_FLAT?(__OPTION_SETTING_S_Start + 0x60):__OPTION_SETTING_S_Start
 *fill*         0x0100a250       0x10 ff
 *(.option_setting_pbps_sec0)
 .option_setting_pbps_sec0
                0x0100a260        0x4 ./ra/fsp/src/bsp/mcu/all/bsp_rom_registers.o
                0x0100a264                . = PROJECT_SECURE_OR_FLAT?(__OPTION_SETTING_S_Start + 0x64):__OPTION_SETTING_S_Start
 *(.option_setting_pbps_sec1)
 .option_setting_pbps_sec1
                0x0100a264        0x4 ./ra/fsp/src/bsp/mcu/all/bsp_rom_registers.o
                0x0100a268                . = PROJECT_SECURE_OR_FLAT?(__OPTION_SETTING_S_Start + 0x68):__OPTION_SETTING_S_Start
 *(.option_setting_pbps_sec2)
 .option_setting_pbps_sec2
                0x0100a268        0x4 ./ra/fsp/src/bsp/mcu/all/bsp_rom_registers.o
                0x0100a26c                . = PROJECT_SECURE_OR_FLAT?(__OPTION_SETTING_S_Start + 0x6c):__OPTION_SETTING_S_Start
 *(.option_setting_pbps_sec3)
 .option_setting_pbps_sec3
                0x0100a26c        0x4 ./ra/fsp/src/bsp/mcu/all/bsp_rom_registers.o
                0x0100a280                . = PROJECT_SECURE_OR_FLAT?(__OPTION_SETTING_S_Start + 0x80):__OPTION_SETTING_S_Start
 *fill*         0x0100a270       0x10 ff
 *(.option_setting_ofs1_sel)
 .option_setting_ofs1_sel
                0x0100a280        0x4 ./ra/fsp/src/bsp/mcu/all/bsp_rom_registers.o
                0x0100a284                . = PROJECT_SECURE_OR_FLAT?(__OPTION_SETTING_S_Start + 0x84):__OPTION_SETTING_S_Start
 *(.option_setting_ofs3_sel)
                0x0100a290                . = PROJECT_SECURE_OR_FLAT?(__OPTION_SETTING_S_Start + 0x90):__OPTION_SETTING_S_Start
 *fill*         0x0100a284        0xc ff
 *(.option_setting_banksel_sel)
 .option_setting_banksel_sel
                0x0100a290        0x4 ./ra/fsp/src/bsp/mcu/all/bsp_rom_registers.o
                0x0100a2c0                . = PROJECT_SECURE_OR_FLAT?(__OPTION_SETTING_S_Start + 0xc0):__OPTION_SETTING_S_Start
 *fill*         0x0100a294       0x2c ff
 *(.option_setting_bps_sel0)
 .option_setting_bps_sel0
                0x0100a2c0        0x4 ./ra/fsp/src/bsp/mcu/all/bsp_rom_registers.o
                0x0100a2c4                . = PROJECT_SECURE_OR_FLAT?(__OPTION_SETTING_S_Start + 0xc4):__OPTION_SETTING_S_Start
 *(.option_setting_bps_sel1)
 .option_setting_bps_sel1
                0x0100a2c4        0x4 ./ra/fsp/src/bsp/mcu/all/bsp_rom_registers.o
                0x0100a2c8                . = PROJECT_SECURE_OR_FLAT?(__OPTION_SETTING_S_Start + 0xc8):__OPTION_SETTING_S_Start
 *(.option_setting_bps_sel2)
 .option_setting_bps_sel2
                0x0100a2c8        0x4 ./ra/fsp/src/bsp/mcu/all/bsp_rom_registers.o
                0x0100a2cc                . = PROJECT_SECURE_OR_FLAT?(__OPTION_SETTING_S_Start + 0xcc):__OPTION_SETTING_S_Start
 *(.option_setting_bps_sel3)
 .option_setting_bps_sel3
                0x0100a2cc        0x4 ./ra/fsp/src/bsp/mcu/all/bsp_rom_registers.o
                0x0100a2d0                __OPTION_SETTING_S_End = .
                0x0100a2d0                __tz_OPTION_SETTING_S_N = __OPTION_SETTING_S_End
OUTPUT(usb_bootloader.elf elf32-littlearm)
LOAD linker stubs

.rel.dyn        0x0100a2d0        0x0
 .rel.iplt      0x0100a2d0        0x0 c:/renesas/ra/e2studio_v2022-10_fsp_v4.2.0/toolchains/gcc_arm/gcc-arm-none-eabi-10.3-2021.10/bin/../lib/gcc/arm-none-eabi/10.3.1/thumb/v8-m.main+fp/hard/crtbegin.o

.ARM.attributes
                0x00000000       0x36
 .ARM.attributes
                0x00000000       0x22 c:/renesas/ra/e2studio_v2022-10_fsp_v4.2.0/toolchains/gcc_arm/gcc-arm-none-eabi-10.3-2021.10/bin/../lib/gcc/arm-none-eabi/10.3.1/thumb/v8-m.main+fp/hard/crti.o
 .ARM.attributes
                0x00000022       0x38 c:/renesas/ra/e2studio_v2022-10_fsp_v4.2.0/toolchains/gcc_arm/gcc-arm-none-eabi-10.3-2021.10/bin/../lib/gcc/arm-none-eabi/10.3.1/thumb/v8-m.main+fp/hard/crtbegin.o
 .ARM.attributes
                0x0000005a       0x3a ./src/hal_entry.o
 .ARM.attributes
                0x00000094       0x3a ./src/udp_cdc.o
 .ARM.attributes
                0x000000ce       0x3a ./src/udp_printf.o
 .ARM.attributes
                0x00000108       0x3a ./src/usb_desc.o
 .ARM.attributes
                0x00000142       0x3a ./ra_gen/common_data.o
 .ARM.attributes
                0x0000017c       0x3a ./ra_gen/hal_data.o
 .ARM.attributes
                0x000001b6       0x3a ./ra_gen/main.o
 .ARM.attributes
                0x000001f0       0x3a ./ra_gen/pin_data.o
 .ARM.attributes
                0x0000022a       0x3a ./ra_gen/vector_data.o
 .ARM.attributes
                0x00000264       0x3a ./ra/fsp/src/r_usb_pcdc/src/r_usb_pcdc_driver.o
 .ARM.attributes
                0x0000029e       0x3a ./ra/fsp/src/r_usb_basic/src/hw/r_usb_creg_abs.o
 .ARM.attributes
                0x000002d8       0x3a ./ra/fsp/src/r_usb_basic/src/hw/r_usb_creg_access.o
 .ARM.attributes
                0x00000312       0x3a ./ra/fsp/src/r_usb_basic/src/hw/r_usb_mcu.o
 .ARM.attributes
                0x0000034c       0x3a ./ra/fsp/src/r_usb_basic/src/hw/r_usb_preg_abs.o
 .ARM.attributes
                0x00000386       0x3a ./ra/fsp/src/r_usb_basic/src/hw/r_usb_preg_access.o
 .ARM.attributes
                0x000003c0       0x3a ./ra/fsp/src/r_usb_basic/src/driver/r_usb_cdataio.o
 .ARM.attributes
                0x000003fa       0x3a ./ra/fsp/src/r_usb_basic/src/driver/r_usb_clibusbip.o
 .ARM.attributes
                0x00000434       0x3a ./ra/fsp/src/r_usb_basic/src/driver/r_usb_pcontrolrw.o
 .ARM.attributes
                0x0000046e       0x3a ./ra/fsp/src/r_usb_basic/src/driver/r_usb_pdriver.o
 .ARM.attributes
                0x000004a8       0x3a ./ra/fsp/src/r_usb_basic/src/driver/r_usb_pintfifo.o
 .ARM.attributes
                0x000004e2       0x3a ./ra/fsp/src/r_usb_basic/src/driver/r_usb_pinthandler_usbip0.o
 .ARM.attributes
                0x0000051c       0x3a ./ra/fsp/src/r_usb_basic/src/driver/r_usb_plibusbip.o
 .ARM.attributes
                0x00000556       0x3a ./ra/fsp/src/r_usb_basic/src/driver/r_usb_psignal.o
 .ARM.attributes
                0x00000590       0x3a ./ra/fsp/src/r_usb_basic/src/driver/r_usb_pstdfunction.o
 .ARM.attributes
                0x000005ca       0x3a ./ra/fsp/src/r_usb_basic/src/driver/r_usb_pstdrequest.o
 .ARM.attributes
                0x00000604       0x3a ./ra/fsp/src/r_usb_basic/r_usb_basic.o
 .ARM.attributes
                0x0000063e       0x3a ./ra/fsp/src/r_rtc/r_rtc.o
 .ARM.attributes
                0x00000678       0x3a ./ra/fsp/src/r_ioport/r_ioport.o
 .ARM.attributes
                0x000006b2       0x3a ./ra/fsp/src/r_flash_hp/r_flash_hp.o
 .ARM.attributes
                0x000006ec       0x3a ./ra/fsp/src/bsp/mcu/all/bsp_clocks.o
 .ARM.attributes
                0x00000726       0x3a ./ra/fsp/src/bsp/mcu/all/bsp_common.o
 .ARM.attributes
                0x00000760       0x3a ./ra/fsp/src/bsp/mcu/all/bsp_delay.o
 .ARM.attributes
                0x0000079a       0x3a ./ra/fsp/src/bsp/mcu/all/bsp_group_irq.o
 .ARM.attributes
                0x000007d4       0x3a ./ra/fsp/src/bsp/mcu/all/bsp_io.o
 .ARM.attributes
                0x0000080e       0x3a ./ra/fsp/src/bsp/mcu/all/bsp_irq.o
 .ARM.attributes
                0x00000848       0x3a ./ra/fsp/src/bsp/mcu/all/bsp_register_protection.o
 .ARM.attributes
                0x00000882       0x3a ./ra/fsp/src/bsp/mcu/all/bsp_rom_registers.o
 .ARM.attributes
                0x000008bc       0x3a ./ra/fsp/src/bsp/cmsis/Device/RENESAS/Source/startup.o
 .ARM.attributes
                0x000008f6       0x3a ./ra/fsp/src/bsp/cmsis/Device/RENESAS/Source/system.o
 .ARM.attributes
                0x00000930       0x22 c:/renesas/ra/e2studio_v2022-10_fsp_v4.2.0/toolchains/gcc_arm/gcc-arm-none-eabi-10.3-2021.10/bin/../lib/gcc/arm-none-eabi/10.3.1/thumb/v8-m.main+fp/hard\libgcc.a(_arm_addsubdf3.o)
 .ARM.attributes
                0x00000952       0x22 c:/renesas/ra/e2studio_v2022-10_fsp_v4.2.0/toolchains/gcc_arm/gcc-arm-none-eabi-10.3-2021.10/bin/../lib/gcc/arm-none-eabi/10.3.1/thumb/v8-m.main+fp/hard\libgcc.a(_arm_muldivdf3.o)
 .ARM.attributes
                0x00000974       0x22 c:/renesas/ra/e2studio_v2022-10_fsp_v4.2.0/toolchains/gcc_arm/gcc-arm-none-eabi-10.3-2021.10/bin/../lib/gcc/arm-none-eabi/10.3.1/thumb/v8-m.main+fp/hard\libgcc.a(_arm_cmpdf2.o)
 .ARM.attributes
                0x00000996       0x22 c:/renesas/ra/e2studio_v2022-10_fsp_v4.2.0/toolchains/gcc_arm/gcc-arm-none-eabi-10.3-2021.10/bin/../lib/gcc/arm-none-eabi/10.3.1/thumb/v8-m.main+fp/hard\libgcc.a(_arm_unorddf2.o)
 .ARM.attributes
                0x000009b8       0x22 c:/renesas/ra/e2studio_v2022-10_fsp_v4.2.0/toolchains/gcc_arm/gcc-arm-none-eabi-10.3-2021.10/bin/../lib/gcc/arm-none-eabi/10.3.1/thumb/v8-m.main+fp/hard\libgcc.a(_arm_fixdfsi.o)
 .ARM.attributes
                0x000009da       0x38 c:/renesas/ra/e2studio_v2022-10_fsp_v4.2.0/toolchains/gcc_arm/gcc-arm-none-eabi-10.3-2021.10/bin/../lib/gcc/arm-none-eabi/10.3.1/../../../../arm-none-eabi/lib/thumb/v8-m.main+fp/hard\libg_nano.a(lib_a-aeabi_memcpy.o)
 .ARM.attributes
                0x00000a12       0x38 c:/renesas/ra/e2studio_v2022-10_fsp_v4.2.0/toolchains/gcc_arm/gcc-arm-none-eabi-10.3-2021.10/bin/../lib/gcc/arm-none-eabi/10.3.1/../../../../arm-none-eabi/lib/thumb/v8-m.main+fp/hard\libg_nano.a(lib_a-memcpy-stub.o)
 .ARM.attributes
                0x00000a4a       0x38 c:/renesas/ra/e2studio_v2022-10_fsp_v4.2.0/toolchains/gcc_arm/gcc-arm-none-eabi-10.3-2021.10/bin/../lib/gcc/arm-none-eabi/10.3.1/../../../../arm-none-eabi/lib/thumb/v8-m.main+fp/hard\libg_nano.a(lib_a-memset.o)
 .ARM.attributes
                0x00000a82       0x17 c:/renesas/ra/e2studio_v2022-10_fsp_v4.2.0/toolchains/gcc_arm/gcc-arm-none-eabi-10.3-2021.10/bin/../lib/gcc/arm-none-eabi/10.3.1/../../../../arm-none-eabi/lib/thumb/v8-m.main+fp/hard\libg_nano.a(lib_a-strlen.o)
 .ARM.attributes
                0x00000a99       0x38 c:/renesas/ra/e2studio_v2022-10_fsp_v4.2.0/toolchains/gcc_arm/gcc-arm-none-eabi-10.3-2021.10/bin/../lib/gcc/arm-none-eabi/10.3.1/thumb/v8-m.main+fp/hard/crtend.o
 .ARM.attributes
                0x00000ad1       0x22 c:/renesas/ra/e2studio_v2022-10_fsp_v4.2.0/toolchains/gcc_arm/gcc-arm-none-eabi-10.3-2021.10/bin/../lib/gcc/arm-none-eabi/10.3.1/thumb/v8-m.main+fp/hard/crtn.o

.comment        0x00000000       0x49
 .comment       0x00000000       0x49 ./src/hal_entry.o
                                 0x4a (size before relaxing)
 .comment       0x00000049       0x4a ./src/udp_cdc.o
 .comment       0x00000049       0x4a ./src/udp_printf.o
 .comment       0x00000049       0x4a ./src/usb_desc.o
 .comment       0x00000049       0x4a ./ra_gen/common_data.o
 .comment       0x00000049       0x4a ./ra_gen/hal_data.o
 .comment       0x00000049       0x4a ./ra_gen/main.o
 .comment       0x00000049       0x4a ./ra_gen/pin_data.o
 .comment       0x00000049       0x4a ./ra_gen/vector_data.o
 .comment       0x00000049       0x4a ./ra/fsp/src/r_usb_pcdc/src/r_usb_pcdc_driver.o
 .comment       0x00000049       0x4a ./ra/fsp/src/r_usb_basic/src/hw/r_usb_creg_abs.o
 .comment       0x00000049       0x4a ./ra/fsp/src/r_usb_basic/src/hw/r_usb_creg_access.o
 .comment       0x00000049       0x4a ./ra/fsp/src/r_usb_basic/src/hw/r_usb_mcu.o
 .comment       0x00000049       0x4a ./ra/fsp/src/r_usb_basic/src/hw/r_usb_preg_abs.o
 .comment       0x00000049       0x4a ./ra/fsp/src/r_usb_basic/src/hw/r_usb_preg_access.o
 .comment       0x00000049       0x4a ./ra/fsp/src/r_usb_basic/src/driver/r_usb_cdataio.o
 .comment       0x00000049       0x4a ./ra/fsp/src/r_usb_basic/src/driver/r_usb_clibusbip.o
 .comment       0x00000049       0x4a ./ra/fsp/src/r_usb_basic/src/driver/r_usb_pcontrolrw.o
 .comment       0x00000049       0x4a ./ra/fsp/src/r_usb_basic/src/driver/r_usb_pdriver.o
 .comment       0x00000049       0x4a ./ra/fsp/src/r_usb_basic/src/driver/r_usb_pintfifo.o
 .comment       0x00000049       0x4a ./ra/fsp/src/r_usb_basic/src/driver/r_usb_pinthandler_usbip0.o
 .comment       0x00000049       0x4a ./ra/fsp/src/r_usb_basic/src/driver/r_usb_plibusbip.o
 .comment       0x00000049       0x4a ./ra/fsp/src/r_usb_basic/src/driver/r_usb_psignal.o
 .comment       0x00000049       0x4a ./ra/fsp/src/r_usb_basic/src/driver/r_usb_pstdfunction.o
 .comment       0x00000049       0x4a ./ra/fsp/src/r_usb_basic/src/driver/r_usb_pstdrequest.o
 .comment       0x00000049       0x4a ./ra/fsp/src/r_usb_basic/r_usb_basic.o
 .comment       0x00000049       0x4a ./ra/fsp/src/r_rtc/r_rtc.o
 .comment       0x00000049       0x4a ./ra/fsp/src/r_ioport/r_ioport.o
 .comment       0x00000049       0x4a ./ra/fsp/src/r_flash_hp/r_flash_hp.o
 .comment       0x00000049       0x4a ./ra/fsp/src/bsp/mcu/all/bsp_clocks.o
 .comment       0x00000049       0x4a ./ra/fsp/src/bsp/mcu/all/bsp_common.o
 .comment       0x00000049       0x4a ./ra/fsp/src/bsp/mcu/all/bsp_delay.o
 .comment       0x00000049       0x4a ./ra/fsp/src/bsp/mcu/all/bsp_group_irq.o
 .comment       0x00000049       0x4a ./ra/fsp/src/bsp/mcu/all/bsp_io.o
 .comment       0x00000049       0x4a ./ra/fsp/src/bsp/mcu/all/bsp_irq.o
 .comment       0x00000049       0x4a ./ra/fsp/src/bsp/mcu/all/bsp_register_protection.o
 .comment       0x00000049       0x4a ./ra/fsp/src/bsp/mcu/all/bsp_rom_registers.o
 .comment       0x00000049       0x4a ./ra/fsp/src/bsp/cmsis/Device/RENESAS/Source/startup.o
 .comment       0x00000049       0x4a ./ra/fsp/src/bsp/cmsis/Device/RENESAS/Source/system.o

.debug_info     0x00000000    0x73e57
 .debug_info    0x00000000     0x6af1 ./src/hal_entry.o
 .debug_info    0x00006af1     0x1c13 ./src/udp_cdc.o
 .debug_info    0x00008704      0x917 ./src/udp_printf.o
 .debug_info    0x0000901b      0x2af ./src/usb_desc.o
 .debug_info    0x000092ca     0x1207 ./ra_gen/common_data.o
 .debug_info    0x0000a4d1     0x25c9 ./ra_gen/hal_data.o
 .debug_info    0x0000ca9a       0xaa ./ra_gen/main.o
 .debug_info    0x0000cb44      0xa07 ./ra_gen/pin_data.o
 .debug_info    0x0000d54b      0x65f ./ra_gen/vector_data.o
 .debug_info    0x0000dbaa     0x35a7 ./ra/fsp/src/r_usb_pcdc/src/r_usb_pcdc_driver.o
 .debug_info    0x00011151     0x3f90 ./ra/fsp/src/r_usb_basic/src/hw/r_usb_creg_abs.o
 .debug_info    0x000150e1     0x48bb ./ra/fsp/src/r_usb_basic/src/hw/r_usb_creg_access.o
 .debug_info    0x0001999c     0x54d1 ./ra/fsp/src/r_usb_basic/src/hw/r_usb_mcu.o
 .debug_info    0x0001ee6d     0x3c4b ./ra/fsp/src/r_usb_basic/src/hw/r_usb_preg_abs.o
 .debug_info    0x00022ab8     0x2756 ./ra/fsp/src/r_usb_basic/src/hw/r_usb_preg_access.o
 .debug_info    0x0002520e     0x3d8a ./ra/fsp/src/r_usb_basic/src/driver/r_usb_cdataio.o
 .debug_info    0x00028f98     0x3a83 ./ra/fsp/src/r_usb_basic/src/driver/r_usb_clibusbip.o
 .debug_info    0x0002ca1b     0x36a6 ./ra/fsp/src/r_usb_basic/src/driver/r_usb_pcontrolrw.o
 .debug_info    0x000300c1     0x5030 ./ra/fsp/src/r_usb_basic/src/driver/r_usb_pdriver.o
 .debug_info    0x000350f1     0x34c6 ./ra/fsp/src/r_usb_basic/src/driver/r_usb_pintfifo.o
 .debug_info    0x000385b7     0x1290 ./ra/fsp/src/r_usb_basic/src/driver/r_usb_pinthandler_usbip0.o
 .debug_info    0x00039847     0x44d2 ./ra/fsp/src/r_usb_basic/src/driver/r_usb_plibusbip.o
 .debug_info    0x0003dd19     0x376a ./ra/fsp/src/r_usb_basic/src/driver/r_usb_psignal.o
 .debug_info    0x00041483     0x3cd8 ./ra/fsp/src/r_usb_basic/src/driver/r_usb_pstdfunction.o
 .debug_info    0x0004515b     0x484e ./ra/fsp/src/r_usb_basic/src/driver/r_usb_pstdrequest.o
 .debug_info    0x000499a9     0x5a06 ./ra/fsp/src/r_usb_basic/r_usb_basic.o
 .debug_info    0x0004f3af     0x86ca ./ra/fsp/src/r_rtc/r_rtc.o
 .debug_info    0x00057a79     0x7373 ./ra/fsp/src/r_ioport/r_ioport.o
 .debug_info    0x0005edec     0x8535 ./ra/fsp/src/r_flash_hp/r_flash_hp.o
 .debug_info    0x00067321     0x469e ./ra/fsp/src/bsp/mcu/all/bsp_clocks.o
 .debug_info    0x0006b9bf      0x916 ./ra/fsp/src/bsp/mcu/all/bsp_common.o
 .debug_info    0x0006c2d5      0x1d1 ./ra/fsp/src/bsp/mcu/all/bsp_delay.o
 .debug_info    0x0006c4a6     0x13d8 ./ra/fsp/src/bsp/mcu/all/bsp_group_irq.o
 .debug_info    0x0006d87e       0xa3 ./ra/fsp/src/bsp/mcu/all/bsp_io.o
 .debug_info    0x0006d921     0x1c82 ./ra/fsp/src/bsp/mcu/all/bsp_irq.o
 .debug_info    0x0006f5a3     0x3cb8 ./ra/fsp/src/bsp/mcu/all/bsp_register_protection.o
 .debug_info    0x0007325b      0x1cc ./ra/fsp/src/bsp/mcu/all/bsp_rom_registers.o
 .debug_info    0x00073427      0x154 ./ra/fsp/src/bsp/cmsis/Device/RENESAS/Source/startup.o
 .debug_info    0x0007357b      0x8dc ./ra/fsp/src/bsp/cmsis/Device/RENESAS/Source/system.o

.debug_abbrev   0x00000000     0x783b
 .debug_abbrev  0x00000000      0x50d ./src/hal_entry.o
 .debug_abbrev  0x0000050d      0x41f ./src/udp_cdc.o
 .debug_abbrev  0x0000092c      0x237 ./src/udp_printf.o
 .debug_abbrev  0x00000b63       0xae ./src/usb_desc.o
 .debug_abbrev  0x00000c11      0x150 ./ra_gen/common_data.o
 .debug_abbrev  0x00000d61      0x23b ./ra_gen/hal_data.o
 .debug_abbrev  0x00000f9c       0x66 ./ra_gen/main.o
 .debug_abbrev  0x00001002       0xdc ./ra_gen/pin_data.o
 .debug_abbrev  0x000010de       0xa7 ./ra_gen/vector_data.o
 .debug_abbrev  0x00001185      0x2c4 ./ra/fsp/src/r_usb_pcdc/src/r_usb_pcdc_driver.o
 .debug_abbrev  0x00001449      0x4af ./ra/fsp/src/r_usb_basic/src/hw/r_usb_creg_abs.o
 .debug_abbrev  0x000018f8      0x4ba ./ra/fsp/src/r_usb_basic/src/hw/r_usb_creg_access.o
 .debug_abbrev  0x00001db2      0x5f1 ./ra/fsp/src/r_usb_basic/src/hw/r_usb_mcu.o
 .debug_abbrev  0x000023a3      0x419 ./ra/fsp/src/r_usb_basic/src/hw/r_usb_preg_abs.o
 .debug_abbrev  0x000027bc      0x1d7 ./ra/fsp/src/r_usb_basic/src/hw/r_usb_preg_access.o
 .debug_abbrev  0x00002993      0x495 ./ra/fsp/src/r_usb_basic/src/driver/r_usb_cdataio.o
 .debug_abbrev  0x00002e28      0x409 ./ra/fsp/src/r_usb_basic/src/driver/r_usb_clibusbip.o
 .debug_abbrev  0x00003231      0x346 ./ra/fsp/src/r_usb_basic/src/driver/r_usb_pcontrolrw.o
 .debug_abbrev  0x00003577      0x582 ./ra/fsp/src/r_usb_basic/src/driver/r_usb_pdriver.o
 .debug_abbrev  0x00003af9      0x2e1 ./ra/fsp/src/r_usb_basic/src/driver/r_usb_pintfifo.o
 .debug_abbrev  0x00003dda      0x334 ./ra/fsp/src/r_usb_basic/src/driver/r_usb_pinthandler_usbip0.o
 .debug_abbrev  0x0000410e      0x513 ./ra/fsp/src/r_usb_basic/src/driver/r_usb_plibusbip.o
 .debug_abbrev  0x00004621      0x32e ./ra/fsp/src/r_usb_basic/src/driver/r_usb_psignal.o
 .debug_abbrev  0x0000494f      0x404 ./ra/fsp/src/r_usb_basic/src/driver/r_usb_pstdfunction.o
 .debug_abbrev  0x00004d53      0x4e4 ./ra/fsp/src/r_usb_basic/src/driver/r_usb_pstdrequest.o
 .debug_abbrev  0x00005237      0x533 ./ra/fsp/src/r_usb_basic/r_usb_basic.o
 .debug_abbrev  0x0000576a      0x59a ./ra/fsp/src/r_rtc/r_rtc.o
 .debug_abbrev  0x00005d04      0x449 ./ra/fsp/src/r_ioport/r_ioport.o
 .debug_abbrev  0x0000614d      0x5cc ./ra/fsp/src/r_flash_hp/r_flash_hp.o
 .debug_abbrev  0x00006719      0x376 ./ra/fsp/src/bsp/mcu/all/bsp_clocks.o
 .debug_abbrev  0x00006a8f      0x172 ./ra/fsp/src/bsp/mcu/all/bsp_common.o
 .debug_abbrev  0x00006c01      0x111 ./ra/fsp/src/bsp/mcu/all/bsp_delay.o
 .debug_abbrev  0x00006d12      0x254 ./ra/fsp/src/bsp/mcu/all/bsp_group_irq.o
 .debug_abbrev  0x00006f66       0x5e ./ra/fsp/src/bsp/mcu/all/bsp_io.o
 .debug_abbrev  0x00006fc4      0x251 ./ra/fsp/src/bsp/mcu/all/bsp_irq.o
 .debug_abbrev  0x00007215      0x277 ./ra/fsp/src/bsp/mcu/all/bsp_register_protection.o
 .debug_abbrev  0x0000748c       0x4d ./ra/fsp/src/bsp/mcu/all/bsp_rom_registers.o
 .debug_abbrev  0x000074d9       0xe6 ./ra/fsp/src/bsp/cmsis/Device/RENESAS/Source/startup.o
 .debug_abbrev  0x000075bf      0x27c ./ra/fsp/src/bsp/cmsis/Device/RENESAS/Source/system.o

.debug_loc      0x00000000    0x14de5
 .debug_loc     0x00000000     0x11ea ./src/hal_entry.o
 .debug_loc     0x000011ea      0x43d ./src/udp_cdc.o
 .debug_loc     0x00001627     0x1978 ./src/udp_printf.o
 .debug_loc     0x00002f9f      0x112 ./ra/fsp/src/r_usb_pcdc/src/r_usb_pcdc_driver.o
 .debug_loc     0x000030b1      0x84d ./ra/fsp/src/r_usb_basic/src/hw/r_usb_creg_abs.o
 .debug_loc     0x000038fe     0x2579 ./ra/fsp/src/r_usb_basic/src/hw/r_usb_creg_access.o
 .debug_loc     0x00005e77      0x61b ./ra/fsp/src/r_usb_basic/src/hw/r_usb_mcu.o
 .debug_loc     0x00006492      0x81a ./ra/fsp/src/r_usb_basic/src/hw/r_usb_preg_abs.o
 .debug_loc     0x00006cac       0x25 ./ra/fsp/src/r_usb_basic/src/hw/r_usb_preg_access.o
 .debug_loc     0x00006cd1      0x7eb ./ra/fsp/src/r_usb_basic/src/driver/r_usb_cdataio.o
 .debug_loc     0x000074bc      0x4d8 ./ra/fsp/src/r_usb_basic/src/driver/r_usb_clibusbip.o
 .debug_loc     0x00007994      0x216 ./ra/fsp/src/r_usb_basic/src/driver/r_usb_pcontrolrw.o
 .debug_loc     0x00007baa     0x140e ./ra/fsp/src/r_usb_basic/src/driver/r_usb_pdriver.o
 .debug_loc     0x00008fb8      0x27f ./ra/fsp/src/r_usb_basic/src/driver/r_usb_pintfifo.o
 .debug_loc     0x00009237       0x54 ./ra/fsp/src/r_usb_basic/src/driver/r_usb_pinthandler_usbip0.o
 .debug_loc     0x0000928b     0x1085 ./ra/fsp/src/r_usb_basic/src/driver/r_usb_plibusbip.o
 .debug_loc     0x0000a310      0x1a5 ./ra/fsp/src/r_usb_basic/src/driver/r_usb_psignal.o
 .debug_loc     0x0000a4b5      0x12b ./ra/fsp/src/r_usb_basic/src/driver/r_usb_pstdfunction.o
 .debug_loc     0x0000a5e0      0xf5a ./ra/fsp/src/r_usb_basic/src/driver/r_usb_pstdrequest.o
 .debug_loc     0x0000b53a     0x2292 ./ra/fsp/src/r_usb_basic/r_usb_basic.o
 .debug_loc     0x0000d7cc     0x1ef9 ./ra/fsp/src/r_rtc/r_rtc.o
 .debug_loc     0x0000f6c5     0x1b9f ./ra/fsp/src/r_ioport/r_ioport.o
 .debug_loc     0x00011264     0x333e ./ra/fsp/src/r_flash_hp/r_flash_hp.o
 .debug_loc     0x000145a2      0x2d5 ./ra/fsp/src/bsp/mcu/all/bsp_clocks.o
 .debug_loc     0x00014877       0x3c ./ra/fsp/src/bsp/mcu/all/bsp_common.o
 .debug_loc     0x000148b3      0x178 ./ra/fsp/src/bsp/mcu/all/bsp_delay.o
 .debug_loc     0x00014a2b       0xc7 ./ra/fsp/src/bsp/mcu/all/bsp_group_irq.o
 .debug_loc     0x00014af2      0x121 ./ra/fsp/src/bsp/mcu/all/bsp_irq.o
 .debug_loc     0x00014c13      0x105 ./ra/fsp/src/bsp/mcu/all/bsp_register_protection.o
 .debug_loc     0x00014d18       0xcd ./ra/fsp/src/bsp/cmsis/Device/RENESAS/Source/system.o

.debug_aranges  0x00000000      0xe50
 .debug_aranges
                0x00000000       0x40 ./src/hal_entry.o
 .debug_aranges
                0x00000040       0x78 ./src/udp_cdc.o
 .debug_aranges
                0x000000b8       0x20 ./src/udp_printf.o
 .debug_aranges
                0x000000d8       0x18 ./src/usb_desc.o
 .debug_aranges
                0x000000f0       0x20 ./ra_gen/common_data.o
 .debug_aranges
                0x00000110       0x20 ./ra_gen/hal_data.o
 .debug_aranges
                0x00000130       0x20 ./ra_gen/main.o
 .debug_aranges
                0x00000150       0x18 ./ra_gen/pin_data.o
 .debug_aranges
                0x00000168       0x18 ./ra_gen/vector_data.o
 .debug_aranges
                0x00000180       0x28 ./ra/fsp/src/r_usb_pcdc/src/r_usb_pcdc_driver.o
 .debug_aranges
                0x000001a8       0x58 ./ra/fsp/src/r_usb_basic/src/hw/r_usb_creg_abs.o
 .debug_aranges
                0x00000200      0x220 ./ra/fsp/src/r_usb_basic/src/hw/r_usb_creg_access.o
 .debug_aranges
                0x00000420       0x68 ./ra/fsp/src/r_usb_basic/src/hw/r_usb_mcu.o
 .debug_aranges
                0x00000488       0x80 ./ra/fsp/src/r_usb_basic/src/hw/r_usb_preg_abs.o
 .debug_aranges
                0x00000508       0x70 ./ra/fsp/src/r_usb_basic/src/hw/r_usb_preg_access.o
 .debug_aranges
                0x00000578       0x58 ./ra/fsp/src/r_usb_basic/src/driver/r_usb_cdataio.o
 .debug_aranges
                0x000005d0       0x80 ./ra/fsp/src/r_usb_basic/src/driver/r_usb_clibusbip.o
 .debug_aranges
                0x00000650       0x30 ./ra/fsp/src/r_usb_basic/src/driver/r_usb_pcontrolrw.o
 .debug_aranges
                0x00000680      0x100 ./ra/fsp/src/r_usb_basic/src/driver/r_usb_pdriver.o
 .debug_aranges
                0x00000780       0x30 ./ra/fsp/src/r_usb_basic/src/driver/r_usb_pintfifo.o
 .debug_aranges
                0x000007b0       0x20 ./ra/fsp/src/r_usb_basic/src/driver/r_usb_pinthandler_usbip0.o
 .debug_aranges
                0x000007d0       0xa0 ./ra/fsp/src/r_usb_basic/src/driver/r_usb_plibusbip.o
 .debug_aranges
                0x00000870       0x38 ./ra/fsp/src/r_usb_basic/src/driver/r_usb_psignal.o
 .debug_aranges
                0x000008a8       0x38 ./ra/fsp/src/r_usb_basic/src/driver/r_usb_pstdfunction.o
 .debug_aranges
                0x000008e0       0x80 ./ra/fsp/src/r_usb_basic/src/driver/r_usb_pstdrequest.o
 .debug_aranges
                0x00000960      0x108 ./ra/fsp/src/r_usb_basic/r_usb_basic.o
 .debug_aranges
                0x00000a68       0x90 ./ra/fsp/src/r_rtc/r_rtc.o
 .debug_aranges
                0x00000af8       0x90 ./ra/fsp/src/r_ioport/r_ioport.o
 .debug_aranges
                0x00000b88      0x120 ./ra/fsp/src/r_flash_hp/r_flash_hp.o
 .debug_aranges
                0x00000ca8       0x60 ./ra/fsp/src/bsp/mcu/all/bsp_clocks.o
 .debug_aranges
                0x00000d08       0x30 ./ra/fsp/src/bsp/mcu/all/bsp_common.o
 .debug_aranges
                0x00000d38       0x28 ./ra/fsp/src/bsp/mcu/all/bsp_delay.o
 .debug_aranges
                0x00000d60       0x28 ./ra/fsp/src/bsp/mcu/all/bsp_group_irq.o
 .debug_aranges
                0x00000d88       0x18 ./ra/fsp/src/bsp/mcu/all/bsp_io.o
 .debug_aranges
                0x00000da0       0x20 ./ra/fsp/src/bsp/mcu/all/bsp_irq.o
 .debug_aranges
                0x00000dc0       0x28 ./ra/fsp/src/bsp/mcu/all/bsp_register_protection.o
 .debug_aranges
                0x00000de8       0x18 ./ra/fsp/src/bsp/mcu/all/bsp_rom_registers.o
 .debug_aranges
                0x00000e00       0x28 ./ra/fsp/src/bsp/cmsis/Device/RENESAS/Source/startup.o
 .debug_aranges
                0x00000e28       0x28 ./ra/fsp/src/bsp/cmsis/Device/RENESAS/Source/system.o

.debug_ranges   0x00000000     0x2d00
 .debug_ranges  0x00000000      0x2a8 ./src/hal_entry.o
 .debug_ranges  0x000002a8      0x2d0 ./src/udp_cdc.o
 .debug_ranges  0x00000578      0x1c0 ./src/udp_printf.o
 .debug_ranges  0x00000738       0x10 ./ra_gen/common_data.o
 .debug_ranges  0x00000748       0x10 ./ra_gen/hal_data.o
 .debug_ranges  0x00000758       0x10 ./ra_gen/main.o
 .debug_ranges  0x00000768       0x18 ./ra/fsp/src/r_usb_pcdc/src/r_usb_pcdc_driver.o
 .debug_ranges  0x00000780       0x78 ./ra/fsp/src/r_usb_basic/src/hw/r_usb_creg_abs.o
 .debug_ranges  0x000007f8      0x468 ./ra/fsp/src/r_usb_basic/src/hw/r_usb_creg_access.o
 .debug_ranges  0x00000c60      0x318 ./ra/fsp/src/r_usb_basic/src/hw/r_usb_mcu.o
 .debug_ranges  0x00000f78       0x70 ./ra/fsp/src/r_usb_basic/src/hw/r_usb_preg_abs.o
 .debug_ranges  0x00000fe8       0x60 ./ra/fsp/src/r_usb_basic/src/hw/r_usb_preg_access.o
 .debug_ranges  0x00001048       0x78 ./ra/fsp/src/r_usb_basic/src/driver/r_usb_cdataio.o
 .debug_ranges  0x000010c0       0x70 ./ra/fsp/src/r_usb_basic/src/driver/r_usb_clibusbip.o
 .debug_ranges  0x00001130       0x20 ./ra/fsp/src/r_usb_basic/src/driver/r_usb_pcontrolrw.o
 .debug_ranges  0x00001150      0x278 ./ra/fsp/src/r_usb_basic/src/driver/r_usb_pdriver.o
 .debug_ranges  0x000013c8       0x20 ./ra/fsp/src/r_usb_basic/src/driver/r_usb_pintfifo.o
 .debug_ranges  0x000013e8       0x60 ./ra/fsp/src/r_usb_basic/src/driver/r_usb_pinthandler_usbip0.o
 .debug_ranges  0x00001448       0xc8 ./ra/fsp/src/r_usb_basic/src/driver/r_usb_plibusbip.o
 .debug_ranges  0x00001510       0x28 ./ra/fsp/src/r_usb_basic/src/driver/r_usb_psignal.o
 .debug_ranges  0x00001538       0x28 ./ra/fsp/src/r_usb_basic/src/driver/r_usb_pstdfunction.o
 .debug_ranges  0x00001560      0x1b8 ./ra/fsp/src/r_usb_basic/src/driver/r_usb_pstdrequest.o
 .debug_ranges  0x00001718      0x240 ./ra/fsp/src/r_usb_basic/r_usb_basic.o
 .debug_ranges  0x00001958      0x628 ./ra/fsp/src/r_rtc/r_rtc.o
 .debug_ranges  0x00001f80      0x240 ./ra/fsp/src/r_ioport/r_ioport.o
 .debug_ranges  0x000021c0      0x890 ./ra/fsp/src/r_flash_hp/r_flash_hp.o
 .debug_ranges  0x00002a50      0x128 ./ra/fsp/src/bsp/mcu/all/bsp_clocks.o
 .debug_ranges  0x00002b78       0x20 ./ra/fsp/src/bsp/mcu/all/bsp_common.o
 .debug_ranges  0x00002b98       0x18 ./ra/fsp/src/bsp/mcu/all/bsp_delay.o
 .debug_ranges  0x00002bb0       0x58 ./ra/fsp/src/bsp/mcu/all/bsp_group_irq.o
 .debug_ranges  0x00002c08       0x68 ./ra/fsp/src/bsp/mcu/all/bsp_irq.o
 .debug_ranges  0x00002c70       0x48 ./ra/fsp/src/bsp/mcu/all/bsp_register_protection.o
 .debug_ranges  0x00002cb8       0x18 ./ra/fsp/src/bsp/cmsis/Device/RENESAS/Source/startup.o
 .debug_ranges  0x00002cd0       0x30 ./ra/fsp/src/bsp/cmsis/Device/RENESAS/Source/system.o

.debug_line     0x00000000    0x14b02
 .debug_line    0x00000000     0x14bc ./src/hal_entry.o
 .debug_line    0x000014bc      0xa92 ./src/udp_cdc.o
 .debug_line    0x00001f4e      0xcdc ./src/udp_printf.o
 .debug_line    0x00002c2a      0x19f ./src/usb_desc.o
 .debug_line    0x00002dc9      0x324 ./ra_gen/common_data.o
 .debug_line    0x000030ed      0x3b8 ./ra_gen/hal_data.o
 .debug_line    0x000034a5       0x5e ./ra_gen/main.o
 .debug_line    0x00003503      0x1f8 ./ra_gen/pin_data.o
 .debug_line    0x000036fb       0xf9 ./ra_gen/vector_data.o
 .debug_line    0x000037f4      0x47c ./ra/fsp/src/r_usb_pcdc/src/r_usb_pcdc_driver.o
 .debug_line    0x00003c70      0x695 ./ra/fsp/src/r_usb_basic/src/hw/r_usb_creg_abs.o
 .debug_line    0x00004305     0x1b5a ./ra/fsp/src/r_usb_basic/src/hw/r_usb_creg_access.o
 .debug_line    0x00005e5f      0xb6c ./ra/fsp/src/r_usb_basic/src/hw/r_usb_mcu.o
 .debug_line    0x000069cb      0xa11 ./ra/fsp/src/r_usb_basic/src/hw/r_usb_preg_abs.o
 .debug_line    0x000073dc      0x4cc ./ra/fsp/src/r_usb_basic/src/hw/r_usb_preg_access.o
 .debug_line    0x000078a8      0x749 ./ra/fsp/src/r_usb_basic/src/driver/r_usb_cdataio.o
 .debug_line    0x00007ff1      0x63e ./ra/fsp/src/r_usb_basic/src/driver/r_usb_clibusbip.o
 .debug_line    0x0000862f      0x48e ./ra/fsp/src/r_usb_basic/src/driver/r_usb_pcontrolrw.o
 .debug_line    0x00008abd     0x11dd ./ra/fsp/src/r_usb_basic/src/driver/r_usb_pdriver.o
 .debug_line    0x00009c9a      0x42f ./ra/fsp/src/r_usb_basic/src/driver/r_usb_pintfifo.o
 .debug_line    0x0000a0c9      0x42e ./ra/fsp/src/r_usb_basic/src/driver/r_usb_pinthandler_usbip0.o
 .debug_line    0x0000a4f7      0xe1d ./ra/fsp/src/r_usb_basic/src/driver/r_usb_plibusbip.o
 .debug_line    0x0000b314      0x4bf ./ra/fsp/src/r_usb_basic/src/driver/r_usb_psignal.o
 .debug_line    0x0000b7d3      0x5b7 ./ra/fsp/src/r_usb_basic/src/driver/r_usb_pstdfunction.o
 .debug_line    0x0000bd8a      0xf45 ./ra/fsp/src/r_usb_basic/src/driver/r_usb_pstdrequest.o
 .debug_line    0x0000cccf     0x125e ./ra/fsp/src/r_usb_basic/r_usb_basic.o
 .debug_line    0x0000df2d     0x1af7 ./ra/fsp/src/r_rtc/r_rtc.o
 .debug_line    0x0000fa24      0xe9c ./ra/fsp/src/r_ioport/r_ioport.o
 .debug_line    0x000108c0     0x1eae ./ra/fsp/src/r_flash_hp/r_flash_hp.o
 .debug_line    0x0001276e      0x83c ./ra/fsp/src/bsp/mcu/all/bsp_clocks.o
 .debug_line    0x00012faa      0x2c9 ./ra/fsp/src/bsp/mcu/all/bsp_common.o
 .debug_line    0x00013273      0x2e4 ./ra/fsp/src/bsp/mcu/all/bsp_delay.o
 .debug_line    0x00013557      0x34d ./ra/fsp/src/bsp/mcu/all/bsp_group_irq.o
 .debug_line    0x000138a4      0x1af ./ra/fsp/src/bsp/mcu/all/bsp_io.o
 .debug_line    0x00013a53      0x473 ./ra/fsp/src/bsp/mcu/all/bsp_irq.o
 .debug_line    0x00013ec6      0x3ea ./ra/fsp/src/bsp/mcu/all/bsp_register_protection.o
 .debug_line    0x000142b0      0x161 ./ra/fsp/src/bsp/mcu/all/bsp_rom_registers.o
 .debug_line    0x00014411      0x233 ./ra/fsp/src/bsp/cmsis/Device/RENESAS/Source/startup.o
 .debug_line    0x00014644      0x4be ./ra/fsp/src/bsp/cmsis/Device/RENESAS/Source/system.o

.debug_str      0x00000000     0xe4a1
 .debug_str     0x00000000     0x4de2 ./src/hal_entry.o
                               0x4f4f (size before relaxing)
 .debug_str     0x00004de2      0xbf0 ./src/udp_cdc.o
                               0x280b (size before relaxing)
 .debug_str     0x000059d2       0xf2 ./src/udp_printf.o
                                0x2d5 (size before relaxing)
 .debug_str     0x00005ac4      0x127 ./src/usb_desc.o
                                0x353 (size before relaxing)
 .debug_str     0x00005beb      0x26e ./ra_gen/common_data.o
                               0x3257 (size before relaxing)
 .debug_str     0x00005e59      0xcf4 ./ra_gen/hal_data.o
                               0x36f8 (size before relaxing)
 .debug_str     0x00006b4d       0x16 ./ra_gen/main.o
                                0x1bb (size before relaxing)
 .debug_str     0x00006b63      0x648 ./ra_gen/pin_data.o
                               0x1d3d (size before relaxing)
 .debug_str     0x000071ab     0x149e ./ra_gen/vector_data.o
                               0x1633 (size before relaxing)
 .debug_str     0x00008649      0xd38 ./ra/fsp/src/r_usb_pcdc/src/r_usb_pcdc_driver.o
                               0x31eb (size before relaxing)
 .debug_str     0x00009381      0x3d4 ./ra/fsp/src/r_usb_basic/src/hw/r_usb_creg_abs.o
                               0x31fe (size before relaxing)
 .debug_str     0x00009755      0x3b0 ./ra/fsp/src/r_usb_basic/src/hw/r_usb_creg_access.o
                               0x33ca (size before relaxing)
 .debug_str     0x00009b05      0x937 ./ra/fsp/src/r_usb_basic/src/hw/r_usb_mcu.o
                               0x3bec (size before relaxing)
 .debug_str     0x0000a43c      0x2d1 ./ra/fsp/src/r_usb_basic/src/hw/r_usb_preg_abs.o
                               0x32f3 (size before relaxing)
 .debug_str     0x0000a70d       0xc6 ./ra/fsp/src/r_usb_basic/src/hw/r_usb_preg_access.o
                               0x10e4 (size before relaxing)
 .debug_str     0x0000a7d3      0x3c7 ./ra/fsp/src/r_usb_basic/src/driver/r_usb_cdataio.o
                               0x36b2 (size before relaxing)
 .debug_str     0x0000ab9a      0x162 ./ra/fsp/src/r_usb_basic/src/driver/r_usb_clibusbip.o
                               0x3433 (size before relaxing)
 .debug_str     0x0000acfc       0x6d ./ra/fsp/src/r_usb_basic/src/driver/r_usb_pcontrolrw.o
                               0x2ff8 (size before relaxing)
 .debug_str     0x0000ad69      0x63b ./ra/fsp/src/r_usb_basic/src/driver/r_usb_pdriver.o
                               0x3da6 (size before relaxing)
 .debug_str     0x0000b3a4       0x8e ./ra/fsp/src/r_usb_basic/src/driver/r_usb_pintfifo.o
                               0x2f26 (size before relaxing)
 .debug_str     0x0000b432       0x40 ./ra/fsp/src/r_usb_basic/src/driver/r_usb_pinthandler_usbip0.o
                               0x247d (size before relaxing)
 .debug_str     0x0000b472       0xca ./ra/fsp/src/r_usb_basic/src/driver/r_usb_plibusbip.o
                               0x3387 (size before relaxing)
 .debug_str     0x0000b53c       0x77 ./ra/fsp/src/r_usb_basic/src/driver/r_usb_psignal.o
                               0x3185 (size before relaxing)
 .debug_str     0x0000b5b3       0x78 ./ra/fsp/src/r_usb_basic/src/driver/r_usb_pstdfunction.o
                               0x378d (size before relaxing)
 .debug_str     0x0000b62b      0x284 ./ra/fsp/src/r_usb_basic/src/driver/r_usb_pstdrequest.o
                               0x38fd (size before relaxing)
 .debug_str     0x0000b8af      0x2a6 ./ra/fsp/src/r_usb_basic/r_usb_basic.o
                               0x3e77 (size before relaxing)
 .debug_str     0x0000bb55      0x708 ./ra/fsp/src/r_rtc/r_rtc.o
                               0x4608 (size before relaxing)
 .debug_str     0x0000c25d      0x8bf ./ra/fsp/src/r_ioport/r_ioport.o
                               0x5643 (size before relaxing)
 .debug_str     0x0000cb1c      0x8eb ./ra/fsp/src/r_flash_hp/r_flash_hp.o
                               0x472e (size before relaxing)
 .debug_str     0x0000d407      0x597 ./ra/fsp/src/bsp/mcu/all/bsp_clocks.o
                               0x1fa4 (size before relaxing)
 .debug_str     0x0000d99e      0x10b ./ra/fsp/src/bsp/mcu/all/bsp_common.o
                               0x1b6b (size before relaxing)
 .debug_str     0x0000daa9       0xbc ./ra/fsp/src/bsp/mcu/all/bsp_delay.o
                                0x2e4 (size before relaxing)
 .debug_str     0x0000db65      0x1de ./ra/fsp/src/bsp/mcu/all/bsp_group_irq.o
                               0x2076 (size before relaxing)
 .debug_str     0x0000dd43       0x23 ./ra/fsp/src/bsp/mcu/all/bsp_io.o
                                0x1e4 (size before relaxing)
 .debug_str     0x0000dd66      0x36f ./ra/fsp/src/bsp/mcu/all/bsp_irq.o
                               0x1ee3 (size before relaxing)
 .debug_str     0x0000e0d5       0x88 ./ra/fsp/src/bsp/mcu/all/bsp_register_protection.o
                               0x19ba (size before relaxing)
 .debug_str     0x0000e15d      0x185 ./ra/fsp/src/bsp/mcu/all/bsp_rom_registers.o
                                0x32e (size before relaxing)
 .debug_str     0x0000e2e2       0x89 ./ra/fsp/src/bsp/cmsis/Device/RENESAS/Source/startup.o
                                0x235 (size before relaxing)
 .debug_str     0x0000e36b      0x136 ./ra/fsp/src/bsp/cmsis/Device/RENESAS/Source/system.o
                                0x610 (size before relaxing)

.debug_frame    0x00000000     0x29f0
 .debug_frame   0x00000000       0xd4 ./src/hal_entry.o
 .debug_frame   0x000000d4      0x168 ./src/udp_cdc.o
 .debug_frame   0x0000023c       0x70 ./src/udp_printf.o
 .debug_frame   0x000002ac       0x20 ./ra_gen/common_data.o
 .debug_frame   0x000002cc       0x20 ./ra_gen/hal_data.o
 .debug_frame   0x000002ec       0x28 ./ra_gen/main.o
 .debug_frame   0x00000314       0x50 ./ra/fsp/src/r_usb_pcdc/src/r_usb_pcdc_driver.o
 .debug_frame   0x00000364      0x118 ./ra/fsp/src/r_usb_basic/src/hw/r_usb_creg_abs.o
 .debug_frame   0x0000047c      0x488 ./ra/fsp/src/r_usb_basic/src/hw/r_usb_creg_access.o
 .debug_frame   0x00000904      0x10c ./ra/fsp/src/r_usb_basic/src/hw/r_usb_mcu.o
 .debug_frame   0x00000a10      0x180 ./ra/fsp/src/r_usb_basic/src/hw/r_usb_preg_abs.o
 .debug_frame   0x00000b90       0xc0 ./ra/fsp/src/r_usb_basic/src/hw/r_usb_preg_access.o
 .debug_frame   0x00000c50       0xf8 ./ra/fsp/src/r_usb_basic/src/driver/r_usb_cdataio.o
 .debug_frame   0x00000d48      0x148 ./ra/fsp/src/r_usb_basic/src/driver/r_usb_clibusbip.o
 .debug_frame   0x00000e90       0x88 ./ra/fsp/src/r_usb_basic/src/driver/r_usb_pcontrolrw.o
 .debug_frame   0x00000f18      0x384 ./ra/fsp/src/r_usb_basic/src/driver/r_usb_pdriver.o
 .debug_frame   0x0000129c       0x8c ./ra/fsp/src/r_usb_basic/src/driver/r_usb_pintfifo.o
 .debug_frame   0x00001328       0x2c ./ra/fsp/src/r_usb_basic/src/driver/r_usb_pinthandler_usbip0.o
 .debug_frame   0x00001354      0x214 ./ra/fsp/src/r_usb_basic/src/driver/r_usb_plibusbip.o
 .debug_frame   0x00001568       0xa8 ./ra/fsp/src/r_usb_basic/src/driver/r_usb_psignal.o
 .debug_frame   0x00001610       0x88 ./ra/fsp/src/r_usb_basic/src/driver/r_usb_pstdfunction.o
 .debug_frame   0x00001698      0x22c ./ra/fsp/src/r_usb_basic/src/driver/r_usb_pstdrequest.o
 .debug_frame   0x000018c4      0x3bc ./ra/fsp/src/r_usb_basic/r_usb_basic.o
 .debug_frame   0x00001c80      0x230 ./ra/fsp/src/r_rtc/r_rtc.o
 .debug_frame   0x00001eb0      0x1b4 ./ra/fsp/src/r_ioport/r_ioport.o
 .debug_frame   0x00002064      0x498 ./ra/fsp/src/r_flash_hp/r_flash_hp.o
 .debug_frame   0x000024fc       0xd4 ./ra/fsp/src/bsp/mcu/all/bsp_clocks.o
 .debug_frame   0x000025d0       0x40 ./ra/fsp/src/bsp/mcu/all/bsp_common.o
 .debug_frame   0x00002610       0x44 ./ra/fsp/src/bsp/mcu/all/bsp_delay.o
 .debug_frame   0x00002654       0x3c ./ra/fsp/src/bsp/mcu/all/bsp_group_irq.o
 .debug_frame   0x00002690       0x30 ./ra/fsp/src/bsp/mcu/all/bsp_irq.o
 .debug_frame   0x000026c0       0x48 ./ra/fsp/src/bsp/mcu/all/bsp_register_protection.o
 .debug_frame   0x00002708       0x38 ./ra/fsp/src/bsp/cmsis/Device/RENESAS/Source/startup.o
 .debug_frame   0x00002740       0x44 ./ra/fsp/src/bsp/cmsis/Device/RENESAS/Source/system.o
 .debug_frame   0x00002784       0xac c:/renesas/ra/e2studio_v2022-10_fsp_v4.2.0/toolchains/gcc_arm/gcc-arm-none-eabi-10.3-2021.10/bin/../lib/gcc/arm-none-eabi/10.3.1/thumb/v8-m.main+fp/hard\libgcc.a(_arm_addsubdf3.o)
 .debug_frame   0x00002830       0x50 c:/renesas/ra/e2studio_v2022-10_fsp_v4.2.0/toolchains/gcc_arm/gcc-arm-none-eabi-10.3-2021.10/bin/../lib/gcc/arm-none-eabi/10.3.1/thumb/v8-m.main+fp/hard\libgcc.a(_arm_muldivdf3.o)
 .debug_frame   0x00002880       0xc4 c:/renesas/ra/e2studio_v2022-10_fsp_v4.2.0/toolchains/gcc_arm/gcc-arm-none-eabi-10.3-2021.10/bin/../lib/gcc/arm-none-eabi/10.3.1/thumb/v8-m.main+fp/hard\libgcc.a(_arm_cmpdf2.o)
 .debug_frame   0x00002944       0x20 c:/renesas/ra/e2studio_v2022-10_fsp_v4.2.0/toolchains/gcc_arm/gcc-arm-none-eabi-10.3-2021.10/bin/../lib/gcc/arm-none-eabi/10.3.1/thumb/v8-m.main+fp/hard\libgcc.a(_arm_unorddf2.o)
 .debug_frame   0x00002964       0x24 c:/renesas/ra/e2studio_v2022-10_fsp_v4.2.0/toolchains/gcc_arm/gcc-arm-none-eabi-10.3-2021.10/bin/../lib/gcc/arm-none-eabi/10.3.1/thumb/v8-m.main+fp/hard\libgcc.a(_arm_fixdfsi.o)
 .debug_frame   0x00002988       0x20 c:/renesas/ra/e2studio_v2022-10_fsp_v4.2.0/toolchains/gcc_arm/gcc-arm-none-eabi-10.3-2021.10/bin/../lib/gcc/arm-none-eabi/10.3.1/../../../../arm-none-eabi/lib/thumb/v8-m.main+fp/hard\libg_nano.a(lib_a-aeabi_memcpy.o)
 .debug_frame   0x000029a8       0x28 c:/renesas/ra/e2studio_v2022-10_fsp_v4.2.0/toolchains/gcc_arm/gcc-arm-none-eabi-10.3-2021.10/bin/../lib/gcc/arm-none-eabi/10.3.1/../../../../arm-none-eabi/lib/thumb/v8-m.main+fp/hard\libg_nano.a(lib_a-memcpy-stub.o)
 .debug_frame   0x000029d0       0x20 c:/renesas/ra/e2studio_v2022-10_fsp_v4.2.0/toolchains/gcc_arm/gcc-arm-none-eabi-10.3-2021.10/bin/../lib/gcc/arm-none-eabi/10.3.1/../../../../arm-none-eabi/lib/thumb/v8-m.main+fp/hard\libg_nano.a(lib_a-memset.o)
